:020000040000FA
:100000000C9426070C9457070C9457070C94570729
:100010000C9457070C9457070C9457070C945707E8
:100020000C9457070C9457070C9457070C945707D8
:100030000C9457070C94B17D0C9457070C945707F8
:100040000C9457070C94F57B0C9457070C945707A6
:100050000C9457070C9457070C9457070C94217B6A
:100060000C9457070C9402780C94D8770C9457078B
:100070000C9457070C9457070C9457070C94570788
:100080000C94C77B0C9457070C9457070C94570794
:100090000C9457070C9457070C9457070C945980ED
:1000A0000C9457070C9457070C94997B0C945707A2
:1000B0000C9457070C9457070C9457070C946B7BC0
:1000C0000C9457070C9457070C9457070C94570738
:1000D0000C9457070C9457070C94A2770C947877DC
:1000E0000C9457070C9459070C94E06D0C948E0FE8
:1000F0000C9429890C94456F0C94C9070C94E01456
:100100000C94168D0C94B6070C94D56F0C94580F64
:100110000C94960C0C94F76F0C941F6E0C94E007E3
:100120000C94020E0C94A0070C94E16D0C94566F85
:100130000C9489070C94D46F0C94E58E0C94000FEA
:100140000C9481070C94C00F0C9474140C94907050
:100150000C94106E0C94416E0C945A6F0C94860D96
:100160000C94EC070C94EF070C94726F0C94AE0C8B
:100170000C94EE5A0C949D150C94F2070C94766F27
:100180000C944D6F0C94908A0C94FE6F0C94836EBB
:100190000C942B700C94C1070C94B00D0C949B7FA5
:1001A0000C947A700C94350F0C94D06E0C94E46F10
:1001B0000C94581A0C9478200C947B6F0C941116A4
:1001C0000C945A700C9400960C946E0E0C94506F14
:1001D0000C94F68E0C94496F0C943B6F0C94E36D69
:1001E0000C9499070C94416F0C9480120C946B073B
:1001F0000C94A8950C94646F0C947C6F0C94606FB5
:100200000C94EA070C94686F0C94F10C0C94670D35
:100210000C94DF0E0C94F3120C94CA070C94806FAC
:100220000C9433890C94060E0C947F160C9441198F
:100230000C9451610C94336E0C94AA760C9485073F
:100240000C947C160C946E6F0C94E26D0C94E98CFB
:100250004E414E494E495459494E46CDCCCC3D0AAB
:10026000D7233C17B7D13877CC2B329595E6241F8E
:10027000B14F0A000020410000C84200401C462047
:10028000BCBE4CCA1B0E5AAEC59D7400407A10F31A
:100290005A00A0724E18090010A5D4E80000E876B4
:1002A00048170000E40B54020000CA9A3B0000000B
:1002B000E1F505000080969800000040420F000024
:1002C00000A08601000000102700000000E80300E5
:1002D0000000006400000000000A000000000001AF
:1002E00000000000002C76D888DC674F0823DFC1AF
:1002F000DFAE59E1B1B796E5E3E453C63AE651996A
:100300007696E8E6C28426EB898C9B62ED407C6F92
:10031000FCEFBC9C9F40F2BAA56FA5F490055A2A49
:10032000F75C936B6CF9676DC11BFCE0E40D47FE55
:10033000F520E6B500D0ED902E030094357705004A
:1003400080841E080000204E0A000000C80C3333D1
:1003500033330F986E12831141EF8D2114893BE6E0
:100360005516CFFEE6DB18D1844B381BF77C1D9069
:100370001DA4BBE424203284725E228100C9F124D2
:10038000ECA1E53D27485454502F312E3020343015
:10039000302042616420526571756573740D0A5393
:1003A00065727665723A205765626475696E6F2F63
:1003B000312E370D0A436F6E74656E742D5479704B
:1003C000653A20746578742F68746D6C0D0A0D0A97
:1003D0003C68313E45504943204641494C3C2F68DA
:1003E000313E00485454502F312E302032303020CE
:1003F0004F4B0D0A5365727665723A2057656264F9
:1004000075696E6F2F312E370D0A41636365737303
:100410002D436F6E74726F6C2D416C6C6F772D4F26
:10042000726967696E3A202A0D0A436F6E74656EB1
:10043000742D547970653A2000436F6E6E65637455
:10044000696F6E3A20636C6F73650D0A436F6E744B
:10045000656E742D547970653A206170706C6963B3
:100460006174696F6E2F782D7777772D666F726D57
:100470002D75726C656E636F64656400506F737484
:10048000206661696C65640055706C6F616420461C
:1004900061696C65643A2000234E6F2073656E734A
:1004A0006F7220666F722074656D702026206875EB
:1004B0006D696469747921004E6F2053656E736FA6
:1004C00072210020666F722074656D70202620688E
:1004D000756D696469747921002353656E736F7259
:1004E000204572726F72200053656E736F722045E3
:1004F00072726F7221002357726F6E672073656E80
:10050000736F7220666F722074656D70202620688C
:10051000756D6964697479210057726F6E67205335
:10052000656E736F7221004320483D00543D0020EA
:1005300020202020202020202020202020202000DB
:1005400020202020202020202020202020202000CB
:1005500020202020202020202020202020202000BB
:1005600054696D657374616D702075706C6F616432
:10057000206661696C65640053657474696E6720F8
:10058000636C6F636B2074696D6500495020616412
:1005900064726573733A2000416E676C6540004970
:1005A0006E76616C696420534D207374657073209E
:1005B00070657220616E676C653D00534D207374E9
:1005C0006570732070657220616E676C653D003CDC
:1005D000703E4C616D7020616E64204F746865726E
:1005E00020537461747573EFBC9A3C2F703E003CCD
:1005F000703E54696D653A20003C2F68333E0A0016
:100600003C62723E4254206E616D653D003C6272F8
:100610003E506174683D003C68333E5379737465A5
:100620006D3A2056657273696F6E3D003C21646FB0
:1006300063747970652068746D6C3E3C68746D6C91
:100640003E3C686561643E3C6D6574612063686131
:10065000727365743D227574662D38223E3C746950
:10066000746C653E4F6E6C696E652065787065725E
:10067000696D656E74202D20506F6C6172697A61AE
:1006800074696F6E2065666665637473206F66209B
:100690006C696768743C2F7469746C653E3C2F68A4
:1006A0006561643E3C626F64793E3C68313E4F6EEA
:1006B0006C696E65206578706572696D656E742011
:1006C0002D20506F6C6172697A6174696F6E20655C
:1006D000666665637473206F66206C696768743C36
:1006E0002F68313E003C68343E436F707972696711
:1006F00068742843293230323020456455484B20F5
:100700004861732043656E7472652E3C2F68343ED9
:100710003C2F626F64793E3C2F68746D6C3E003CE8
:1007200068313E43616E6E6F742067657420736537
:100730006E736F722072656164696E6773213C2FFE
:1007400068313E00506172616D657465727320722C
:100750006573657420646F6E6521007365737573CE
:1007600065722F736D6C69676874706F2F73312FAA
:1007700000616E676C6520646972656374696F6E91
:100780003A200043757272656E7420534D20697370
:10079000202300534D3A5461626C65207374657078
:1007A000732070657220616E676C653D00534D3A31
:1007B000506F6C6172697A65722073746570732012
:1007C00070657220616E676C653D00234448543D3E
:1007D00000236E65743D424C4500236E65743D57A1
:1007E00069466900236E65743D4254002366747047
:1007F00020757365726E616D653A003A0023486F2B
:1008000073742073657276657220495020616E643E
:1008100020506F72743A002352656C6179206465D0
:1008200076696365733A002352656C61792073744D
:1008300061747573206C6162656C733A2000235299
:10084000656C6179207374617465733A0023526535
:100850006C61792070696E733A00234E6F2E206FA1
:10086000662072656C6179733D0046696E64696EDD
:10087000672057694669204950004E45543D426CF7
:100880007565746F6F7468204C45004E45543D4249
:100890006C7565746F6F7468004E45543D576946BA
:1008A00069005344206F70656E206661696C004E6C
:1008B0006577206461746120636F6C6C6563746933
:1008C0006F6E207374617274656400437572726533
:1008D0006E742073657474696E67733A005379732C
:1008E00074656D2072657365742061742000234403
:1008F0005320546865726D6F6D6574657220636115
:100900006C6962726174656420666F7220230049AD
:100910006E76616C696420616E676C6520666F72CB
:1009200020002073746570732070657220616E679B
:100930006C653D0020737465707320706572206172
:100940006E676C653D005461626C65205365742070
:100950003000235475726E7461626C652053657447
:10096000203000506F6C6172697A65722053657433
:1009700020300023506F6C6172697A657220536574
:10098000742030005461626C65205365742030001F
:10099000235475726E7461626C65205365742030E7
:1009A00000506F6C6172697A6572205365742030F3
:1009B0000023506F6C6172697A65722053657420F0
:1009C0003000576946692049503A004C6F676765A7
:1009D00072204E616D653A20005265626F6F7469D6
:1009E0006E672E2E2E0053657276657220506F72E0
:1009F0007420757064617465640053504F52543DA7
:100A00000049502075706461746564005349503D1D
:100A10000074696D6520696E74657276616C3D0065
:100A200054494D455354414D503D0054494D455353
:100A300054414D500023776562736572766572206C
:100A4000626567696E73005461626C6520536574FA
:100A5000203000235475726E7461626C652053659A
:100A600074203000506F6C6172697A657220536532
:100A70007420300023506F6C6172697A6572205364
:100A8000657420300053797374656D2072657374DA
:100A9000617274656421002053797374656D2072EE
:100AA0006573746172746564210023436F6D6D61B9
:100AB0006E64400054657374204C616D70732F46F2
:100AC000616E7300444843502053756363657373CC
:100AD0000044484350204641494C45440053657406
:100AE00074696E6720446576696365204950202EDD
:100AF0002E2E006572726F72206F70656E696E6760
:100B00002066696C653A20004C616D70204F7468F6
:100B10006572002354696D652020202020204461E7
:100B2000746520202020205365636F6E647320500D
:100B30006F6C6172697A6572205461626C652054D1
:100B4000286F43292048282529202000646F6E65DE
:100B50002100696E69742E20646F6E652E00534407
:100B600020696E69742E206661696C656421006974
:100B70006E69742E206661696C65642100232320F0
:100B80004F452057656C636F6D6520232300496EC8
:100B9000697469616C697A696E6720534420636186
:100BA00072642E2E2E0075706C6F61642062792045
:100BB000465450206661696C6564210075706C6FE5
:100BC000616420627920465450204F4B21007C3CC8
:100BD0003E5E2B3D3F2F5B5D3B2C2A225C000000DC
:100BE0002100240027002A002D00300033000101DD
:100BF0000000040107010A0100002200250028006E
:100C00002B002E0031003400020100000501080114
:100C10000B01000020002300260029002C002F00DB
:100C20003200000100000301060109010505050568
:100C3000070508080808020202020A0A0808040454
:100C40000404010101010101010103030303030382
:100C50000303040707070C0C0C0C0C0C0C0C020211
:100C6000020206060606060606060B0B0B0B0B0B0E
:100C70000B0B01021020200808102040102040809B
:100C80000201020108040201010204081020408050
:100C900080402010080402018004020180402010DE
:100CA0000804020108040201010204081020408027
:100CB000010204081020408000000A0B02090C0DFC
:100CC0000E080703040100000000000000000000FF
:100CD0000000000000000000000000000000000014
:100CE00000000000121110000000000000000000D1
:100CF00000000000000000000000000000000000F4
:100D0000010001001010020001000100B00000000D
:100D10001600000028000000100000002000000065
:100D200001000100000000000000000000000000C1
:100D300000000000000000000000000000000000B3
:100D4000FF000000FFFF0000FFFF0000FFFF0000AA
:100D5000CFBF0000C7BF0000C3BF0000C1BF00007D
:100D6000C0BF000000000000C0BF0000C1BF000005
:100D7000C3BF0000C7BF0000CFBF0000FFFF0000DF
:100D8000FFFF000000000000000000000000000065
:100D90000000000000000000000000000000000053
:100DA0000000000000000000000000000000000043
:100DB0000000000000000000000000000000000033
:100DC00000000000557365722D6167656E743A20EE
:100DD0002A0D0A446973616C6C6F773A202F0D0AF3
:100DE000004E6574776F726B206D61696E74616916
:100DF0006E65642061742000417070656E64206DC2
:100E00006561732E200053696E676C65206D6561A6
:100E1000732E200053617665206D65617375726570
:100E200020746F3A00202020202020202020202025
:100E300020202020200020202020202020202020D2
:100E400020202020202000000096A89511241FBEFD
:100E5000CFEFD1E2DEBFCDBF00E00CBF1AE0A0E0D3
:100E6000B2E0E6E9FFE501E00BBF02C007900D929A
:100E7000AE33B107D9F725E1AEE3BAE001C01D9268
:100E8000AC3DB207E1F717E0C5E2D7E000E006C0ED
:100E900021970109802FFE010E942CAAC432D1079C
:100EA00080E00807A9F70E947A990C94B9AF0C94D6
:100EB0000000CF93DF93EC01898D9A8D892B41F04F
:100EC000E881F9810284F385E02DCE011995F4CFF4
:100ED000DF91CF910895CF93DF931F92CDB7DEB707
:100EE0006983DC01ED91FC910280F381E02D41E00A
:100EF00050E0BE016F5F7F4F19950F90DF91CF914A
:100F00000895FC01818D928D0895FC018489958955
:100F1000089521E034E0FC0131832083FB01408906
:100F2000518962897389FC01428353836483758389
:100F30000895DC01ED91FC91048CF58DE02D199460
:100F4000CF93DF931F92CDB7DEB76983DC01ED91BC
:100F5000FC910280F381E02D41E050E0BE016F5F23
:100F60007F4F19950F90DF91CF910895FC019485E3
:100F7000FB018485981303C081E0943009F480E07C
:100F8000089521E0FC018485843009F420E0822F5B
:100F900008950895CF93DF931F92CDB7DEB769838D
:100FA000DC01ED91FC910280F381E02D41E050E005
:100FB000BE016F5F7F4F19950F90DF91CF9108951C
:100FC000DC01ED91FC91068CF78DE02D199591E0F7
:100FD00089270895862F089581E0862708950A9627
:100FE0000C94CA0790E080E0089590E0982F88273D
:100FF00044E050E0845F9B4F0C946292DF92EF924A
:10100000FF920F931F93CF93DF93D82E0AED1BE02F
:10101000E801EE24E394F12C22968091A8029091AD
:10102000A9028E159F059CF061E088810E94557988
:101030006091D50B88810E94387864EF71E080E080
:1010400090E00E94AB798FEFE81AF80AE5CFDD2037
:1010500009F45EC0CAEDDBE0EE24E394F12C2296A5
:101060008091A8029091A902E816F9062CF56091EA
:10107000D70B88810E94387868EE73E080E090E0BA
:101080000E94AB79AFEFEA1AFA0A6091D70B8A8116
:101090000E94387868EE73E080E090E00E94AB79BF
:1010A0006091D50B88810E94387868EE73E080E00B
:1010B00090E00E94AB79D3CF68EE73E080E090E0DF
:1010C0000E94AB7993E4E92E92E0F92EC1E0D0E0E2
:1010D000B2E0EB0EF11C0E5F1F4F8091A8029091C1
:1010E000A9028C179D07A4F0D701ED91FC91EE0F9A
:1010F000FF1FEB52F44F6081F80180810E94387825
:1011000068EC70E080E090E00E94AB792196E0CF3F
:10111000DF91CF911F910F91FF90EF90DF90089595
:101120009F92AF92BF92CF92DF92EF92FF920F9376
:101130001F93CF93DF935C017B018B01D0E0C0E074
:10114000F80191908F016501CC0EDD1EC6010E9451
:1011500064A8981621F0692DC6010E946CA82196FA
:10116000CA32F1E0DF0761F7C701DF91CF911F912C
:101170000F91FF90EF90DF90CF90BF90AF909F9036
:10118000089581E08093DD028091DE02882341F0A2
:1011900088E08093E61160E08BED91E10C946E7F26
:1011A0000895CF93DF93EC01FB01248135810E94E8
:1011B000EC75CE01DF91CF9108958091DE028823F6
:1011C000F9F08091DD028823D9F081E00E94B27F9E
:1011D0008BE39FE10197F1F760E080E00E94C37F1D
:1011E00060E575E08BED91E10E94487761E080E079
:1011F0000E94C37F60E475E08BED91E10C94487729
:1012000008958F929F92AF92BF92CF92DF92EF920A
:10121000FF920F931F93CF93DF938C01862F0B3098
:10122000110509F09FC090916411992309F0F89479
:1012300062E10E94DE79EC0180916411882309F05B
:101240007894209701F180E090ECA9E7B4EC8093CA
:10125000571190935811A0935911B0935A1180933C
:101260005B1190935C11A0935D11B0935E11CE3F22
:101270008FEFD80709F4A9C0CF3FDC0709F462C09B
:10128000CCEFDFEF30C1C0915F11E09060116E2DA7
:1012900070E090E080E00E9447A72DEC3CEC4CEC25
:1012A0005DE30E94A6A74B015C016C2F70E090E00B
:1012B00080E00E9447A79B01AC01C501B4010E94D8
:1012C000EEA8609357117093581180935911909321
:1012D0005A11D0916111F09062116D2F6F7770E00B
:1012E00090E080E00E9447A74B015C016F2D70E009
:1012F00090E080E00E9447A72DEC3CEC4CEC5DE3D5
:101300000E94A6A79B01AC01C501B4010E94EEA8F2
:10131000D7FD26C060935B1170935C1180935D11C3
:1013200090935E11CE0DCD0FCF0D81E090E0209116
:101330006311C21302C090E080E0892B09F493C0CE
:10134000CFEFDFEFCE01DF91CF911F910F91FF9093
:10135000EF90DF90CF90BF90AF909F908F900895C7
:101360009058D8CFCFEFDFEF0631110509F0BBC0A1
:1013700090916411992309F0F89461E00E94DE795C
:10138000EC0180916411882309F07894209701F191
:1013900080E090ECA9E7B4EC80935711909358113A
:1013A000A0935911B0935A1180935B1190935C11E3
:1013B000A0935D11B0935E11CF3FDC0719F2209727
:1013C00009F451C0229609F05BCFCEEFDFEF8BC05E
:1013D000C0916011D0915F1160915F1170916011A7
:1013E00076276727762790E080E00E9445A72DECBE
:1013F0003CEC4CEC5DE30E94A6A760935711709300
:1014000058118093591190935A11E0906211F09005
:1014100061116F2D6F77762F6E2D90E080E00E9426
:1014200045A72DEC3CEC4CEC5DE30E94A6A7F7FC35
:1014300018C060935B1170935C1180935D11909361
:101440005E118C2F8D0F8E0D8F0DC1E0D0E090912D
:101450006311891302C0D0E0C0E0D195C195D109D4
:10146000ABCF9058E6CFC0905711D0905811E09074
:101470005911F0905A1120E030E048EC52E4C701D5
:10148000B6010E9402AAD0E0C0E0181614F4CBEF17
:10149000DFEF20E030E0A901C701B6010E9440A7BC
:1014A00087FF02C0CAEFDFEFC0905B11D0905C11E4
:1014B000E0905D11F0905E1120E030E048EC52ECDD
:1014C000C701B6010E9440A787FF02C0C9EFDFEF46
:1014D00020E030E040EF52E4C701B6010E9402AACA
:1014E00018160CF483C00C30110509F02BCF81E0E5
:1014F0008093B80C8CE58093BA0C1092B90C1092C2
:10150000BB0C60E086EF9DE00E942B7081E00E94A2
:101510007E7E0E9486796B017C018091B20C8111E4
:1015200068C081E08093B20C8093B10C9FEF9093E0
:10153000B00C1092AF0C94E09093AE0C80938D0C95
:1015400080918D0C886B80938D0C80918C0C8130F8
:1015500009F028C110928C0C0E9486796B017C01E5
:1015600080918D0C8093BB008091B40C9091B50C50
:10157000A091B60CB091B70C892B8A2B8B2BA1F0C4
:101580000E9486790091B40C1091B50C2091B60C94
:101590003091B70C6C197D098E099F090617170742
:1015A0002807390708F446C08091BC0083FDD8CFD6
:1015B00085EC8093BC000E9486796B017C01809150
:1015C000B20C813009F4F0C08091AF0C853008F086
:1015D0000DC18091AF0CAEE8BCE0E1E2FCE090E030
:1015E000981769F12D9121939F5FFACFC8EFDFEF34
:1015F0007ACF8091B40C9091B50CA091B60CB091BB
:10160000B70C892B8A2B8B2B09F487CF0E94867904
:101610000091B40C1091B50C2091B60C3091B70C20
:101620006C197D098E099F090617170728073907C6
:1016300008F073CF8091B30C0E945D7E80E0109221
:10164000720C8093710C082F10E0CEEFDFEF88232F
:1016500009F478CECDEFDFEF053011050CF472CE32
:10166000CEEFDAE086EF9DE00E94E46F8887219656
:10167000CE018E5F9A4080179107A4F3C091060BAC
:101680000091070B602F70E090E080E00E9447A778
:101690002DEC3CEC4CEC5DE30E94A6A76B017C01B9
:1016A0006C2F70E090E080E00E9447A79B01AC01A6
:1016B000C701B6010E94EEA86B017C01C092FE0A30
:1016C000D092FF0AE092000BF092010BD091080B30
:1016D0001091090B6D2F6F7770E090E080E00E9411
:1016E00047A74B015C01612F70E090E080E00E9411
:1016F00047A72DEC3CEC4CEC5DE30E94A6A79B01B8
:10170000AC01C501B4010E94EEA8D7FD71C0609381
:10171000020B7093030B8093040B9093050BC00F87
:10172000CD0FC10F80910A0BC8130ACE20E030E024
:1017300048EC52E4C701B6010E9402AAD0E0C0E022
:10174000181614F4CBEFDFEF20E030E040EA50E46D
:10175000C701B6010E9440A787FF02C0CAEFDFEFB2
:10176000C090020BD090030BE090040BF090050B9F
:1017700020E030E040EF51ECC701B6010E9440A7E5
:1017800087FF02C0C9EFDFEF20E030E040EF52E416
:10179000C701B6010E9402AA18160CF0D3CDC8EFFB
:1017A000DFEFD0CD85EE05CF8091B40C9091B50CD4
:1017B000A091B60CB091B70C892B8A2B8B2B09F416
:1017C000FECE0E9486790091B40C1091B50C209148
:1017D000B60C3091B70C6C197D098E099F0906175C
:1017E00017072807390708F0EACE24CF85E0F3CEA3
:1017F00090588DCF2C9A08952C9808958EBD000096
:101800000DB407FEFDCF8EB508959B0190E00496C0
:10181000982F8827642F820F931F0C94F192CF93F7
:10182000DF93C82FD62F472F60E170E00E94050C90
:101830004D2F61E170E08C2FDF91CF910C94050C5E
:10184000CF93DF93C82FD0E02496DC2FCC27C60F90
:10185000D71F0E94FC0B8FE00E94FE0B8D2F0E9471
:10186000FE0B8C2F0E94FE0B80E00E94FE0BC82F07
:101870000E94FA0B8C2FDF91CF9108951F93CF9385
:10188000DF93182F66E270E00E94200CC82F67E2F9
:1018900070E0812F0E94200C9C2FDF91CF911F912F
:1018A00008951F93CF93DF93182F60E270E00E949A
:1018B000200CC82F61E270E0812F0E94200C9C2F29
:1018C000DF91CF911F91089544E050E0BC018FE07B
:1018D00090E00C94629208958CBD9DBD0895EF92A6
:1018E000FF920F931F93CF93C82F7B0180E590E069
:1018F0000E946C0C68E270E08C2F0E94200C082F74
:1019000069E270E08C2F0E94200C282F302FB90143
:1019100021E030E0A7018C2F0E94C17281E090E0AD
:10192000CF911F910F91FF90EF900895CF93DF9388
:101930001F92CDB7DEB7FC01218D328D8FEF9FEF67
:10194000232B41F0BE016F5F7F4F808D0E946F0C93
:10195000898190E00F90DF91CF9108950F931F93AD
:10196000CF93DF931F92CDB7DEB78C01DC01ED91F1
:10197000FC910084F185E02D1995892B79F0BE0149
:101980006F5F7F4FF80184850E946F0C898190E022
:101990000F90DF91CF911F910F9108958FEF9FEFDF
:1019A000F7CFFF920F931F93CF93DF93F82E80E52D
:1019B00090E00E946C0C10E000E08F2D0E943E0C25
:1019C000EC01892B21F08F2D0E943E0C8C01C01759
:1019D000D10799F7CE01DF91CF911F910F91FF9021
:1019E0000895FC018485843011F00C94D10C90E0B2
:1019F00080E00895AF92BF92CF92DF92EF92FF9274
:101A00001F93CF93DF93182F6B017A0180E590E04D
:101A10000E946C0CB12CA12C812F0E943E0CEC0179
:101A2000892B21F0812F0E943E0C5C01CA15DB0539
:101A300099F72097E9F463E070E0812F0E94200C71
:101A4000843159F0882349F0C1E0D0E08C3111F4A1
:101A5000D0E0C0E0D195C195D109CE01DF91CF9101
:101A60001F91FF90EF90DF90CF90BF90AF900895BF
:101A7000EC16FD060CF4E7011C161D0674F768E26F
:101A800070E0812F0E94200CE82E69E270E0812F27
:101A90000E94200C282F3E2D79019E01A601B7013E
:101AA000812F0E94C172EC0EFD1E4F2D68E270E086
:101AB000812F0E94050C4E2D69E270E0812F0E945B
:101AC000050C60E470E0812F0E948D71C6CFCF932A
:101AD000DF93FC01218D328D2115310529F48FEF23
:101AE0009FEFDF91CF910895EC01808D421753074E
:101AF00008F0A9010E94FA0C1816190684F7298D1E
:101B00003A8D281B390B3A8F298FEBCF0F931F93F8
:101B1000CF93DF931F92CDB7DEB7FC01218D328DBD
:101B2000232B41F48FEF9FEF0F90DF91CF911F9107
:101B30000F9108958C0141E050E0BE016F5F7F4F2F
:101B4000FC01808D0E94FA0C181619065CF7F8014A
:101B5000818D928D0197928F818F898190E0E4CF62
:101B60000F931F93CF93DF9300D000D01F921F924B
:101B7000CDB7DEB78C01DC01ED91FC910680F781D9
:101B8000E02D1995F801808D0E94D10C18161906C8
:101B9000B4F548E050E0BE016F5F7F4FD801589622
:101BA0008C910E94FA0C18161906F4F4D80150967C
:101BB00084E0FE01319601900D928A95E1F78D81C6
:101BC00090E0982F88272E81820F911DF801958B28
:101BD000848B8F81282F30E0322F22278885820F37
:101BE000932F911D928F818F28960FB6F894DEBFA8
:101BF0000FBECDBFDF91CF911F910F91089590E05F
:101C000080E0F2CFFC0184850C94FA0CCF93DF9333
:101C10001F92CDB7DEB741E050E0BE016F5F7F4F4E
:101C2000FC0184850E94FA0C1816190634F4898187
:101C300090E00F90DF91CF9108958FEF9FEFF9CF54
:101C4000CF93C82F80E590E00E946C0C60E170E0BB
:101C50008C2F0E948D714FEF62E070E08C2FCF913E
:101C60000C94050CFF920F931F93CF93DF93C82F13
:101C7000D62F8A01F22E0E94200E80E590E00E946D
:101C80006C0C4D2F4F2970E060E08C2F0E94050CEA
:101C900001151105C1F0412F64E070E08C2F0E9406
:101CA000050C402F65E070E08C2F0E94050C61E070
:101CB00070E08C2F0E948D7181E0DF91CF911F9198
:101CC0000F91FF90089500911F0C1091200C0F5F51
:101CD0001F4F1093200C00931F0CDDCFBF92CF92AB
:101CE000DF92EF92FF920F931F93CF93DF9300D079
:101CF00000D0CDB7DEB7FC01208D243009F05DC0E7
:101D00006A017B018C01B12C63E070E08B2D0E9495
:101D1000200C81114AC0F801B08EF801808D84300A
:101D200009F44BC096E0E9EEF2E0DE011196019075
:101D30000D929A95E1F7F70193819F779C839481A7
:101D40009D8395819E83B7016E5F7F4F0E94F5074B
:101D5000B601F801808D0E940F0CF801808D90E093
:101D6000982F882746E050E0BE016F5F7F4F8A5F63
:101D70009B4F0E946292F801128E118E20E8A601FC
:101D800062E0808D0E94320E81E026960FB6F894B4
:101D9000DEBF0FBECDBFDF91CF911F910F91FF909E
:101DA000EF90DF90CF90BF900895883109F4B3CFC2
:101DB000B394F4E0BF12A8CFB0CF80E0E6CFCF93CA
:101DC000DF93EC01888D843061F00E94200EE88D55
:101DD000F0E0EE0FFF1FE25BF34F1182108284E010
:101DE000888FDF91CF910895CF93C82F80E590E041
:101DF0000E946C0C63E070E08C2FCF910C94200C4F
:101E0000EF92FF921F93CF93DF93FC01208D24303C
:101E100039F080E0DF91CF911F91FF90EF9008950E
:101E20007B01EC0110E0812F0E94F40E81110FC0A4
:101E3000188F888D843069F3FD86EC861A8E198E92
:101E400020E0A70162E00E94320E81E0E3CF8831FA
:101E500079F31F5F143039F7ECCFFC0184858430AF
:101E600011F00C94F40E80E00895CF93DF93FC0101
:101E700024852430D9F0EC010E942D0F843189F0A3
:101E8000882379F0883169F021E08C3159F4E881B8
:101E9000F9810084F185E02DCE01199521E0892B8F
:101EA00009F420E0822FDF91CF91089580E0FBCFED
:101EB000AF92BF92CF92DF92FF920F931F93CF9377
:101EC000DF938C015B01EA01FC01C688D788F08CA6
:101ED00080E590E00E946C0C8F2D0E949D718C1704
:101EE0009D0720F48F2D0E949D71EC019E01A5019C
:101EF000B6018F2D0E949192F801868997898C0FE7
:101F00009D1F978B868BCE01DF91CF911F910F91F3
:101F1000FF90DF90CF90BF90AF900895CF93FC01DA
:101F2000C08D80E590E00E946C0C60E270E08C2F28
:101F30000E948D7162E070E08C2F0E94200C84FD65
:101F400016C062E070E08C2F0E94200C83FF0AC054
:101F500048E162E070E08C2F0E94050C90E080E088
:101F6000CF91089580E590E00E946C0CE3CF40E1B2
:101F700062E070E08C2F0E94050C81E090E0F0CFD1
:101F8000FF920F931F93CF93DF93EB01FC01178A0E
:101F9000168A2A81211109C02B81211106C02C81AA
:101FA000211103C02D812223E1F041155105C9F013
:101FB0008A01FC01F08C80E590E00E946C0CBE016F
:101FC0006E5F7F4F8F2D0E94F507B8018F2D0E9405
:101FD0000F0C81E090E0DF91CF911F910F91FF9066
:101FE000089590E080E0F7CF4F925F926F927F92DA
:101FF0008F929F92AF92BF92CF92DF92EF92FF9219
:102000000F931F93CF93DF93CDB7DEB763970FB6D0
:10201000F894DEBF0FBECDBF7C016B013A01FB011E
:1020200020E090E080E06AE03191332309F461C060
:1020300040ED430F4A3008F04DC0689FA001699FF2
:10204000500D1124CA01C097830F911D37FD9A9539
:102050008F3F910549F340F3F70142815381648139
:1020600075818091570E9091580EA091590EB091A4
:102070005A0E481759076A077B0709F439C28701C6
:10208000085F1F4F0E94697A6F7077277C5FC801D5
:102090000E94000F813009F030C281E094E09A8301
:1020A0008983F70182819381A481B5818B839C838D
:1020B000AD83BE8345E350E0BE016F5F7F4FC80133
:1020C0000E94C00F892BA9F5D12CC12CC8010E94F8
:1020D000DF0E17C03E3209F0BFCF233009F4BCCF6A
:1020E000D301A20FB11D12968C932F5F90E080E078
:1020F0009BCF233009F0B0CFF3018583CC24C39468
:10210000D12CC60163960FB6F894DEBF0FBECDBFCB
:10211000DF91CF911F910F91FF90EF90DF90CF90C3
:10212000BF90AF909F908F907F906F905F904F90F7
:1021300008950E94697AF701778366837627672777
:1021400076277A83698342E050E0BE016F5F7F4F5C
:10215000C8010E94580F81E090E09E878D8742E081
:1021600050E0BE01635F7F4FC8010E94580F80E0BE
:1021700091E09E878D8742E050E0BE01635F7F4F14
:10218000C8010E94580F1E861D8642E050E0BE0125
:10219000635F7F4FC8010E94580F42E050E0BE01CC
:1021A000635F7F4FC8010E94580F42E050E0BE01BC
:1021B000635F7F4FC8010E94580F5601F60180816E
:1021C000882301F16501F60181912F01882311F027
:1021D0008E32B1F446018A189B081814190474F45D
:1021E0008F8641E050E0BE01615F7F4FC8010E94D1
:1021F000580FA401B501C8010E94580F5201DECF4B
:102200006201E1CF1F8641E050E0BE01615F7F4F78
:10221000C8010E94580FC12CDD24D394DE86CD86E0
:1022200042E050E0BE01635F7F4FC8010E94580F3B
:10223000DE86CD8642E050E0BE01635F7F4FC8017D
:102240000E94580FC8010E948E0F892B09F43CCFC1
:10225000F3E0AF2EB12C230122E0420E511C5EC0F0
:10226000F7014281538164817581808D918DA28DAA
:10227000B38D481759076A077B0709F02FC1848D72
:10228000958DC59709F02AC181A192A10C970CF4F4
:102290002AC14CE050E0BE016F5F7F4FC8010E9431
:1022A000670D8B819C819827892798279A8B898B2A
:1022B00029813A81322723273227F7014681578126
:1022C00042175307D1F497FF18C08F709270892B73
:1022D00009F042C06F807884762467247624D12C5C
:1022E000C12C6114710409F051C0C8010E94590742
:1022F0006AEFC62EDD24DA9407C0C8010E94590790
:10230000ECEFCE2EDD24DA9481E0A81AB10809F4AE
:10231000DDCEFFEFCF16DF0609F0D8CE0E94697A36
:102320003B014C01C8010E94B00D181619060CF4AF
:1023300097CF0E94697A66197709880999096938DF
:1023400073418105910508F0C5C062E370E080E04B
:1023500090E00E94AB79E6CFC8010E9459077BEF5D
:10236000C72EDD24DA94D0CF8D85811117C0C80126
:102370000E94860DC8010E94860DC8010E94860D2C
:10238000C8010E94860DFFEFCF1ADF0A8D819E8162
:10239000982789279827C816D906A8F441E050E065
:1023A000BE01635F7F4FC8010E94670D8D85882342
:1023B000D9F28D859FEF980F9D878823A9F2C801D8
:1023C0000E94860DF6CF912C812C41E050E0BE0199
:1023D0006D5E7F4FC8010E94670D8B89982F907C9E
:1023E00061F4882389F08B899FEF980F9B8B88235A
:1023F00041F0C8010E94860DF6CFC8010E94860DEB
:102400001B8A8B898111E1CF42E050E0BE01615F00
:102410007F4FC8010E94670D42E050E0BE01635F3C
:102420007F4FC8010E94670DC8010E94860DC80138
:102430000E94860DC8010E94860DC8010E94860D6B
:1024400042E050E0BE016F5E7F4FC8010E94670D01
:102450008F85988981159140E9F4CD84DE84DC2450
:10246000CD24DC2481E0C816D104A1F489899A899D
:102470008115944041F0C8010E94590757EFC52EBD
:10248000DD24DA9441CF44E050E0B201C8010E945B
:10249000670D3ACFD12CC12C89899A899827892731
:1024A0009827C816D90638F4C8010E94860DFFEF98
:1024B000CF1ADF0AF1CF2FEF821A920A681479043B
:1024C00009F083CFC8010E94590746EFC42EDD24CE
:1024D000DA941ACFCC24CA94DC2C16CF2EEFC22E5D
:1024E000DD24DA9411CF9DEFC92EDD24DA940CCFD0
:1024F0008EEFC82EDD24DA9404CED12CC12C01CE6F
:10250000CF92DF92EF92FF920F931F93CF93DF93BF
:10251000CDB7DEB7AF970FB6F894DEBF0FBECDBF15
:102520007C016A0101E014E01A8309831C861B8682
:1025300088EE93E0A0E0B0E08D879E87AF87B88BF0
:1025400085E993E09A878987188F0F8B198E1A8EE9
:102550001B8E1C8E84E089A31BA70AA71CA61DA6A0
:102560001EA61FA680914F0E9091500EA091510E65
:10257000B091520E8EA39FA3A8A7B9A78B839C836B
:10258000AD83BE8318861F82AE01465D5F4FCE01CC
:1025900001960E94F40F81309105B1F4D701ED91BD
:1025A000FC910488F589E02D1DA30CA38CA59DA5A5
:1025B000AEA5BFA58EA39FA3A8A7B9A7A601BE01DC
:1025C0006C5D7F4FC7011995AF960FB6F894DEBFCB
:1025D0000FBECDBFDF91CF911F910F91FF90EF9074
:1025E000DF90CF900895CF92DF92EF92FF920F93FA
:1025F0001F93CF93DF93CDB7DEB7AF970FB6F894A5
:10260000DEBF0FBECDBF7C016A0101E014E01A837A
:1026100009831C861B8688EE93E0A0E0B0E08D87DE
:102620009E87AF87B88B85E993E09A878987188F53
:102630000F8B198E1A8E1B8E1C8E84E089A31BA70C
:102640000AA71CA61DA61EA61FA680914F0E90913C
:10265000500EA091510EB091520E8EA39FA3A8A729
:10266000B9A78B839C83AD83BE8318861F82AE017E
:10267000465D5F4FCE0101960E94F40F81309105B7
:10268000B1F4D701ED91FC910684F785E02D1DA3EF
:102690000CA38CA59DA5AEA5BFA58EA39FA3A8A79F
:1026A000B9A7A601BE016C5D7F4FC7011995AF9612
:1026B0000FB6F894DEBF0FBECDBFDF91CF911F9153
:1026C0000F91FF90EF90DF90CF9008957F928F92BF
:1026D0009F92AF92BF92CF92DF92EF92FF920F93B1
:1026E0001F93CF93DF93CDB7DEB7A6970FB6F894BD
:1026F000DEBF0FBECDBF8C01762E942E852E20E23C
:10270000A22ECE0101967C01DC01EA2D1D92EA95F4
:10271000E9F76801F3E4CF0ED11C81E094E09AA3BD
:1027200089A38FEF8BA38CA38DA38EA343E450E0EA
:10273000BE016F5D7F4FC6010E94C00F019609F474
:10274000BFC081E089838A8386E0B82EBB821C8269
:10275000D80114966D917D918D919C9117970E944F
:1027600034AA6D837E838F83988789869A8680E8D2
:1027700090E09C878B874CE150E0B701C6010E9436
:10278000580FFE0137968AE1DF011D928A95E9F71D
:102790004801B8E08B0E911CF401D70101900D9215
:1027A000BA94E1F740E150E0B701C6010E94580F2A
:1027B000F7011192AA94E9F796E0A92EB12C40E214
:1027C00050E0B701C6010E94580FF1E0AF1AB108FE
:1027D000B1F783E6898392E89A8393E59B838C83A0
:1027E00085E38D8381E08E837F829DE3988797E0E8
:1027F00099878A8786E0F401DE011B9601900D928D
:102800008A95E1F78CE0898B8A8B63E074E0CE01D6
:1028100043960E94A5ACD8011B966C91CE014996B7
:102820000E940973F8016485CE014B960E940973DA
:10283000D8011D966C91CE014D960E9409734EE110
:1028400050E0B701C6010E94580FB3E07B121EC0D2
:1028500082E3898384E08A83F80196859B83978548
:102860009C8390899D8391899E8396E39F8388872B
:10287000828D8987838D8A87848D8B87858D8C87D0
:102880004CE050E0B701C6010E94580F87E38983EE
:1028900086E08A8391E09B8393E09C838D838FE025
:1028A0008E838AE38F838BE388878FEF898749E064
:1028B00050E0B701C6010E94580FC6010E948E0F5A
:1028C000A6960FB6F894DEBF0FBECDBFDF91CF91B5
:1028D0001F910F91FF90EF90DF90CF90BF90AF903E
:1028E0009F908F907F9008958F929F92AF92BF920A
:1028F000CF92DF92EF92FF920F931F93CF93DF93CC
:10290000CDB7DEB72D970FB6F894DEBF0FBECDBFA3
:102910007C0110E000E038EE832E33E0932EA12CF2
:10292000B12C4DEBC42E43E0D42E1C821B828D8231
:102930009E82AF82B886DA82C9820D87CE01019667
:102940000E942D0F811135C0F7014481558120E08F
:1029500061E0802F0E94320E80E590E00E946C0CB6
:1029600063E070E0802F0E94200C833129F462E044
:1029700070E0802F0E948D71F70184819581000F96
:10298000111FF801E25BF34F918380832D960FB600
:10299000F894DEBF0FBECDBFDF91CF911F910F9195
:1029A000FF90EF90DF90CF90BF90AF909F908F906F
:1029B00008950F5F1F4F0430110509F0B6CFE6CF21
:1029C000CF92DF92EF92FF921F93CF93DF93FC01A0
:1029D0001485143089F1EC0180E590E00E946C0CC4
:1029E00068E070E0812F0E948D710E94697A6B010E
:1029F0007C01CE010E942D0F8823A1F061E070E0E0
:102A000080E090E00E94AB790E94697A6C197D09A0
:102A10008E099F09683E73408105910550F38C85AE
:102A20000E94200EEC85F0E0EE0FFF1FE25BF34FFB
:102A30001182108284E08C87DF91CF911F91FF90EB
:102A4000EF90DF90CF9008954F925F926F927F92B8
:102A50008F929F92AF92BF92CF92DF92EF92FF92AE
:102A60001F93CF93DF93CDB7DEB72D970FB6F894B2
:102A7000DEBF0FBECDBF7C019EE4A92E9CE0B92E27
:102A800010E0D12CC12C28EE422E23E0522E612CD6
:102A9000712C3DEB832E33E0932E1C821B824D82E2
:102AA0005E826F8278869A8289821D87D5012D91F8
:102AB0003D915D01F7018481958128173907B1F4B3
:102AC000CE0101960E942D0F843199F1CE0101961D
:102AD0000E942D0F8C3151F4CE0101960E94F10C11
:102AE000892B21F4CE0101960E94E0141F5F14305F
:102AF000A1F6CD2841F4D701ED91FC910084F18538
:102B0000E02DC70119952D960FB6F894DEBF0FBEC4
:102B1000CDBFDF91CF911F91FF90EF90DF90CF90CD
:102B2000BF90AF909F908F907F906F905F904F90ED
:102B30000895CC24C394D12CD9CF8F929F92AF9279
:102B4000BF92CF92DF92EF92FF920F931F93CF939A
:102B50006C015B017A01FC01C485C430A1F481E001
:102B600090E0F60193838283F12CE12CC701CF9191
:102B70001F910F91FF90EF90DF90CF90BF90AF909B
:102B80009F908F9008958A014130584010F000E0E6
:102B900018E080E590E00E946C0C8C2F0E949D71E3
:102BA0004C0163E070E08C2F0E94200C873111F003
:102BB0008C3129F58016910660F380E590E00E9443
:102BC0006C0C9801A50170E060E08C2F0E9491923E
:102BD00060E270E08C2F0E948D7162E070E08C2FBB
:102BE0000E94200C84FD13C063E070E08C2F0E94D3
:102BF000200C811107C08C2F0E94200EB0CF10E056
:102C000000E0DBCF80E590E00E946C0CE6CF40E175
:102C100062E070E08C2F0E94050C012B09F0A6CF1A
:102C20009ECF3F924F925F926F927F928F929F9230
:102C3000AF92BF92CF92DF92EF92FF920F931F93CA
:102C4000CF93DF93CDB7DEB72D970FB6F894DEBFE5
:102C50000FBECDBF6C015B014A010E9424158EE4BA
:102C6000E82E8CE0F82E312C10E000E098EE492E92
:102C700093E0592E612C712C1C821B824D825E8246
:102C80006F8278868DEB93E09A8389833D86F70186
:102C9000219131917F01F6018481958128173907AF
:102CA00071F4CE0101960E942D0F873141F4A401E9
:102CB000B501CE0101960E949D15080F191F33948E
:102CC000F4E03F12D9CFC8012D960FB6F894DEBFBD
:102CD0000FBECDBFDF91CF911F910F91FF90EF906D
:102CE000DF90CF90BF90AF909F908F907F906F902C
:102CF0005F904F903F9008950A960C949D15CF9247
:102D0000DF92FF920F931F93CF93DF93FC012485F3
:102D1000243051F090E080E0DF91CF911F910F912E
:102D2000FF90DF90CF9008956A01EB018C01F12CA8
:102D30008F2D0E94F40E811129C0F801F486F8014C
:102D40008485843039F320919C0230919D022F5F5D
:102D50003F4F21F130939D0220939C0240919C02B1
:102D600050919D0220E061E00E94320E8A818F3FE7
:102D7000C1F48B818F3F01F58C818F3FE9F48D8108
:102D80008F3FD1F484E0F8018487C4CF8B7F8831F2
:102D9000A1F2F394F4E0FF12CBCFD1CF20E030ECDE
:102DA000D9CF811109C08B81811106C08C8181111D
:102DB00003C08D81882331F3C114D10419F3F801C4
:102DC000F48480E590E00E946C0CBE016E5F7F4F42
:102DD0008F2D0E94F507B6018F2D0E940F0C64E025
:102DE00070E08F2D0E948D71C8010E942D0F8731D8
:102DF00061F061E070E080E090E00E94AB79C80192
:102E00000E942D0F8111F0CFBDCF81E090E084CFE3
:102E1000CF93CFB7F89480911E0C811127C0E1E6C3
:102E2000FCE08491E7EAFCE09491E82FF0E0EE0FFB
:102E3000FF1FE252F44FA591B491EC91E92321F4E4
:102E400061E085E30E94387861E085E30E9455796E
:102E50008CB580618CBD8CB580648CBD61E084E3F1
:102E60000E94557961E083E30E94557980911E0CA0
:102E70008F5F80931E0CCFBFCF9108954F925F92CA
:102E80006F927F928F929F92AF92BF92CF92DF927A
:102E9000EF92FF920F931F93CF93DF93EC018090FB
:102EA000A8029090A902E5E4F2E081E090E0512CC4
:102EB000412C8816990654F0219131912130310529
:102EC00019F42FEF421A520A0196F3CF1C161D0671
:102ED0000CF04AC08C169D060CF446C04E018E01C3
:102EE000000F111F7E01EE0CFF1CEE0CFF1C8C1658
:102EF0009D060CF4D9C0C701895C9D4F6C01FC0193
:102F000080819181A281B3819701215B3D4F59015D
:102F1000181619061A061B0654F50E94487CF5017E
:102F20002081318142815381621B730B840B950B8D
:102F3000F6012081318142815381261737074807E6
:102F4000590758F410821182128213820E94487C21
:102F5000F501608371838283938321960E5F1F4FF7
:102F6000F4E0EF0EF11CC3CFC1E0D0E0B8CF980180
:102F70002E553D4F3901F9018081918198012D5BDA
:102F80003D4F6901F9012081318182179307F1F0EA
:102F9000F3E04F16510414F00097C1F4880F991F05
:102FA000FC01EB52F44F6081F801E652F44F80814E
:102FB0000E943878F30180819181F60191838083AA
:102FC0006CE271E080E090E00E94AB79F5018081D5
:102FD0009181A281B381181619061A061B060CF0FE
:102FE000BCCF0E94487CF501208131814281538110
:102FF000621B730B840B950BF701E55AFD4F208183
:10300000318142815381261737074807590708F055
:10301000A4CFF50110821182128213829801275BDE
:103020003D4F5901F90180819181F6012081318163
:103030008217930709F491CF6091A8027091A902B9
:10304000E5E4F2E041E050E030E020E0641775078D
:103050004CF0A191B191119711F42F5F3F4F4F5F49
:103060005F4FF4CF233031051CF0009709F075CF86
:10307000880F991FFC01EB52F44F6081F801E65272
:10308000F44F80810E943878F50180819181F601AA
:1030900091838083F301918380836CE271E080E00F
:1030A00090E00E94AB7959CFDF91CF911F910F91A2
:1030B000FF90EF90DF90CF90BF90AF909F908F9058
:1030C0007F906F905F904F900895CF93DF93FC01B6
:1030D00024813581232B69F0EC01BC0189E59DE059
:1030E0000E943477BE018CEB9CE0DF91CF910C9471
:1030F0003477DF91CF910895CF93DF93FC01248142
:103100003581232B69F0EC01BC0189E59DE00E942B
:103110002677BE018CEB9CE0DF91CF910C94267753
:10312000DF91CF910895CF93DF93FB01228133810B
:10313000DC0113963C932E9312974481558166814E
:10314000778114964D935D936D937C93179740858B
:1031500051856285738518964D935D936D937C932D
:103160001B971C96EF012C969C01275E3F4F4991BF
:103170004D93A217B307D9F7218D328DFC01328F01
:10318000218FDF91CF910895CF92DF92EF92FF923E
:103190000F931F93CF93DF93CDB7DEB7A0970FB6F2
:1031A000F894DEBF0FBECDBF7C018B0150E040E044
:1031B0006C018AE0C80ED11CCA010196F801249165
:1031C000E1E0F0E0EC0FFD1FE40FF51F2083222368
:1031D00089F08032910551F440E250E0BE016F5F0A
:1031E0007F4FC6010E949D1590E080E00F5F1F4F4A
:1031F000AC01E2CF029738F0BE016F5F7F4FC7018D
:103200000A960E949D15A0960FB6F894DEBF0FBED9
:10321000CDBFDF91CF911F910F91FF90EF90DF9085
:10322000CF900895EF92FF920F931F93CF93DF9368
:10323000EC018B017A0163EE73E00E94C418B801BF
:10324000CE010E941E778E01065F1F4F42E050E0C4
:1032500067EE79E0C8010E949D15E114F10421F0A8
:10326000B701CE010E941E7742E050E067EE79E0A0
:10327000C801DF91CF911F910F91FF90EF900C94B7
:103280009D1565E873E00C94C418CF92DF92EF921D
:10329000FF920F931F93CF93DF9300D000D0CDB751
:1032A000DEB77C01FB01848195818A01081B190B23
:1032B000101611069CF0C7010E94BC75C701269626
:1032C0000FB6F894DEBF0FBECDBFDF91CF911F9137
:1032D0000F91FF90EF90DF90CF900895CE0101966F
:1032E0000E94CE75CC24C394D12C6CED75E0CE0138
:1032F00001960E94B274FFEFCF1ADF0A0C151D056C
:10330000A4F7BE016F5F7F4FC7010E94BC75CE015D
:1033100001960E943875D2CFDF92EF92FF920F9301
:103320001F93CF93DF93CDB7DEB762970FB6F894B4
:10333000DEBF0FBECDBF2091DE02222379F12091A6
:10334000DD02222359F17A018C016F3F7F4FA1F5F5
:1033500060E080E00E94C37FD12CB8018BED91E149
:103360000E9426776FE275E08BED91E10E9448772D
:10337000F801848160E08D0D0E94C37F0E94697A0C
:103380006093780C7093790C80937A0C90937B0CFB
:10339000B701FF0C880B990B0E94AB7962960FB6B0
:1033A000F894DEBF0FBECDBFDF91CF911F910F917B
:1033B000FF90EF90DF90089560E080E00E94C37F6F
:1033C0000E94697A28EE33E040E050E00E948AA82B
:1033D000CA01B90120E831E541E050E00E94ACA803
:1033E000AB01BC0120E0CE0101960E947675BE01C2
:1033F0006F5F7F4FCE0107960E94CE7566E778E03B
:10340000CE0107960E943D74BC01CE010D960E942C
:10341000CE75CE0107960E943875CE0101960E94A6
:103420003875BE01635F7F4F8BED91E10E94267777
:10343000D98860E08D2D0E94C37FCE010D960E9439
:1034400038758BCFEF92FF920F931F93CF93DF933B
:1034500000D000D0CDB7DEB78C017B0163ED78E002
:103460000E94D7758AE0E816F1042CF462E976E050
:10347000C8010E94B274B701CE0101960E94257363
:10348000BE016F5F7F4FC8010E94BC74CE010196E0
:103490000E943875C80126960FB6F894DEBF0FBE9D
:1034A000CDBFDF91CF911F910F91FF90EF900895C5
:1034B000CF92DF92EF92FF920F931F93CF93DF9300
:1034C000CDB7DEB7C455D1090FB6F894DEBF0FBE35
:1034D000CDBF65965FAF4EAF65972091570C309189
:1034E000580C2F5F3F4F3093580C2093570C20916E
:1034F000560C2111C1C08B016C0181E08093560CE8
:103500001092580C1092570C63ED78E0CE01895B55
:103510009F4F0E94D77563ED78E0CE01835B9F4F8C
:103520000E94D77550E040E06AE074E0C6010E9456
:1035300012190130110509F08EC063ED78E08BEFB0
:103540009FE00E941B7363ED78E087ED9FE00E948F
:103550001B736596EEADFFAD65978081882309F4F6
:1035600074C000E210E09E012F5F3F4F40E250E048
:10357000BE016F5D7F4FCE018D5A9F4F0E94B97182
:10358000049739F3BE016F5D7F4FCE018F5B9F4F74
:103590000E94D775BE016F5B7F4FCE01895B9F4F45
:1035A0000E94FF74CE018F5B9F4F0E943875BE0151
:1035B0006F5F7F4FCE018F5B9F4F0E94D775BE011B
:1035C0006F5B7F4FCE01835B9F4F0E94FF74CE01E4
:1035D0008F5B9F4F0E9438752D968EAD9FAD2D97B6
:1035E0000297029730F463E274E087ED9FE00E9457
:1035F0001B73BE01695B7F4F8BEF9FE00E94BC7421
:1036000063968EAD9FAD6397892B09F4A2CF6FEDC2
:1036100075E0CE018F5B9F4F0E94D775BE01635B43
:103620007F4FCE018F5B9F4F0E9453746CED75E00E
:103630000E943D74BC018BEF9FE00E94BC74CE01E0
:103640008F5B9F4F0E94387584CF6BEF7FE087EDD3
:103650009FE00E94BC741092560CCE01835B9F4F7A
:103660000E943875CE01895B9F4F0E9438750FB656
:10367000F894DEBF0FBECDBFCC5ADF4F0FB6F89423
:10368000DEBF0FBECDBFDF91CF911F910F91FF9095
:10369000EF90DF90CF9008950F931F93CF93DF9318
:1036A000CDB7DEB72C970FB6F894DEBF0FBECDBFF7
:1036B0002C893D893093A9022093A802FE017496BB
:1036C000AAEDBBE090E080E032962817390734F08D
:1036D000408151814D935D930196F6CF8C8D9D8DE8
:1036E0009093D60B8093D50B8E8D9F8D9093D80B96
:1036F0008093D70BAD968FADAD97BE0164597F4FC8
:103700008F3209F0BAC1CE0107960E94D7756AE2DE
:1037100074E0CE0101960E94D775BE01695F7F4FAC
:10372000CE0101960E945374BC0183E891E10E948E
:10373000E874CE0101960E943875CE0107960E946A
:10374000387563E871E1CE0101960E94CE75CE0115
:1037500001960E946518CE0101960E94387560E4BA
:1037600074E0CE0101960E94D775BE016F5F7F4F56
:1037700083E891E10E940274182FCE0101960E9405
:1037800038754091871150918811112309F47CC13B
:10379000BA016250710983E891E10E94F173682FC8
:1037A000CE0101960E94A375BE016F5F7F4F85E633
:1037B00091E10E94FF74CE0101960E9438756DE57B
:1037C00070E1CE0107960E94D77562E474E0CE01E5
:1037D00001960E94D775BE01695F7F4FCE010196A9
:1037E0000E945374BC018DE791E10E94E874CE0100
:1037F00001960E943875CE0107960E94387524966E
:103800008FAD24971F928F9323968FAD23971F928E
:103810008F9322968FAD22971F928F9321968FAD13
:1038200021971F928F9388E494E09F938F938CE06D
:103830009CE09F938F930E94E3ACCE52DF4F888130
:103840009981C25DD0409093840280938302BE012F
:103850006C527F4FCE0101960E94D775BE016F5FFB
:103860007F4F87E791E10E94FF74CE0101960E948D
:103870003875BE0161527F4FCE0101960E94D77507
:10388000BE016F5F7F4F81E791E10E94FF74CE011F
:1038900001960E94387540917511509176114250F1
:1038A000510961E771E1CE0101960E94D108CE0174
:1038B00001960E9489736C596093B502CE010196FE
:1038C0000E943875CC5EDE4F688179818A819B8148
:1038D000C451D1400E9447A70FB6F894DEBF0FBE77
:1038E000CDBF9B01AC010E9407AA882389F08CE31D
:1038F00090E0A0E0B0E0CC5EDE4F88839983AA839D
:10390000BB83C451D140CD5EDE4F1882C351D1403C
:10391000CD5EDE4F8881C351D140882399F0CC5EC3
:10392000DE4F88819981AA81BB81C451D1408093A7
:10393000AC029093AD02A093AE02B093AF0281E0CF
:103940008093750CC85EDE4F688179818A819B8186
:10395000C851D1409B01AC010E9407AA882361F0A5
:1039600080E090E0A0E7B2E4C85EDE4F88839983F0
:10397000AA83BB83C851D140C45EDE4F6881798180
:10398000CC51D140072E000C880B990B0E9447A701
:103990009B01AC010E9407AA882341F082E090E0DD
:1039A000C45EDE4F99838883CC51D140C45CDE4F26
:1039B00008811981CC53D140B801012E000C880B2D
:1039C000990B0E9447A79B01AC010E9407AA811195
:1039D00003C01016110644F080E590E0C45CDE4F91
:1039E00099838883CC53D140C45CDE4F8881998110
:1039F000CC53D140909336028093350288E2FE0189
:103A0000E551FF4FA0EEBBE001900D928A95E1F7E2
:103A1000CE5CDE4F88819981AA81BB81C253D1409F
:103A20008093200290932102A0932202B09323025C
:103A3000CA5CDE4F88819981AA81BB81C653D1407F
:103A400080931C0290931D02A0931E02B0931F024C
:103A5000C65CDE4F88819981CA53D1409093680239
:103A6000809367022C960FB6F894DEBF0FBECDBFD1
:103A7000DF91CF911F910F910895CE0107960E947B
:103A8000D7756FE274E045CE4150510963E871E1AA
:103A9000CE0101960E94D108BE016F5F7F4F85E67F
:103AA00091E10E94FF74CE0101960E94387563E88F
:103AB00071E1CE0101960E94CE7560E474E0CE0102
:103AC00001960E943D74BC0183E891E10E94E87474
:103AD00072CE0F931F93CF93DF9300D000D0CDB75A
:103AE000DEB72091D90B2223A9F08C016CE877E096
:103AF000CE0101960E94D775B801CE0101960E94B1
:103B00005374BC0189E59DE00E943477CE01019693
:103B10000E94387526960FB6F894DEBF0FBECDBF53
:103B2000DF91CF911F910F910895DF92EF92FF9255
:103B30000F931F93CF93DF93CDB7DEB762970FB686
:103B4000F894DEBF0FBECDBF8C0110920B0B63ED5E
:103B500078E0CE010D960E94D775FF24F39489E595
:103B60009DE00E94416E20910B0B181619067CF502
:103B700021112DC089E59DE00E941F6E8A3009F059
:103B80007EC089899A89892B09F481C0F0920B0B38
:103B900064E574E0CE0101960E94D775BE01635FB3
:103BA0007F4FCE0101960E945374BC01CE0107964F
:103BB0000E94CE75CE0107960E94691DCE01079620
:103BC0000E943875CE0101960E94387560C0F12CB4
:103BD000E12CDD24D394222309F460C089899A89D9
:103BE000019709F045C06BEC74E0CE0107960E9486
:103BF000D775BE01695F7F4FCE010D960E9422747A
:103C0000F12C811115C064E674E0CE0101960E948A
:103C1000D775BE016F5F7F4FCE010D960E94227453
:103C2000FF24F3948111F12CCE0101960E94387586
:103C3000CE0107960E943875FF20A1F050E040E0C9
:103C4000BE01635F7F4FCE0101960E94D108BE0185
:103C50006F5F7F4F8EE99FE00E94FF74CE01019657
:103C60000E94387564E170E080E090E00E94AB79DA
:103C7000BE01635F7F4FC8010E94BC758EC08D304E
:103C800009F47FCF682FCE010D960E9490746AE0F0
:103C900070E080E090E00E94AB7961CF8CEB9CE01B
:103CA0000E94416E1816190614F58CEB9CE00E94D8
:103CB0001F6E8A30A9F08D3099F090910B0B911105
:103CC0000FC0682FCE010D960E9490748FEFE81AF6
:103CD000F80A65E070E080E090E00E94AB79DECF0A
:103CE00089899A89892BA9F3D0920B0BF2CF64E1D1
:103CF00070E080E090E00E94AB79EF2809F43FC0CB
:103D000089899A89892BD9F18091D90B882389F1E6
:103D10006CE877E0CE0101960E94D775BE016F5F17
:103D20007F4FCE010D960E942274F82ECE0101968F
:103D30000E943875F1101DC06DE574E0CE0101964A
:103D40000E94D775CE0101960E947C18CE01019683
:103D50000E943875BE01635F7F4FCE0101960E94BD
:103D6000CE75CE0101960E946518CE0101960E9483
:103D7000387564E170E080E090E00E94AB79898959
:103D80009A8920910B0B21112BCF009709F028CF96
:103D900063ED78E0C8010E94D775CE010D960E94B0
:103DA0003875C80162960FB6F894DEBF0FBECDBF5E
:103DB000DF91CF911F910F91FF90EF90DF900895C9
:103DC0000F931F93CF93DF93CDB7DEB72C970FB62A
:103DD000F894DEBF0FBECDBF8C010E94A97DBC014F
:103DE000C8010E94221A0E94A17DBC01CE01079643
:103DF0000E94221A60EC76E0CE0101960E94D775EF
:103E0000BE01695F7F4FCE0101960E945374BC01D1
:103E1000C8010E94BC74CE0101960E943875CE0183
:103E200007960E9438756CED75E0C8010E94B27467
:103E30000E94997DBC01CE0101960E94221ABE010A
:103E40006F5F7F4FC8010E94BC74CE0101960E9433
:103E5000387566E674E0C8010E94B2740E94917DD4
:103E6000BC01CE0101960E94221ABE016F5F7F4FF6
:103E7000C8010E94BC74CE0101960E94387566E6A6
:103E800074E0C8010E94B2740E94877DBC01CE011B
:103E900001960E94221ABE016F5F7F4FC8010E94E7
:103EA000BC74CE0101960E943875C8012C960FB6DD
:103EB000F894DEBF0FBECDBFDF91CF911F910F9160
:103EC0000895CF93DF9300D000D0CDB7DEB70E9426
:103ED000DD08CE0101960E94E01E4AE050E06FEF3F
:103EE0007FEFCE0101960E948C19CE0101960E94AF
:103EF000387561E080E00E94C37FCE0101960E9488
:103F00007D726BED71E1CE0101960E94AA7668E6A2
:103F100074E08BED91E10E941E770E94697A6093B4
:103F2000610C7093620C8093630C9093640C2696E2
:103F30000FB6F894DEBF0FBECDBFDF91CF910895CD
:103F40000F931F93CF93DF9300D000D0CDB7DEB790
:103F50008C01CE0101960E94E01E4AE050E06FEF16
:103F60007FEFCE0101960E948C19CE0101960E942E
:103F70003875B801CE0101960E94CE756AE070E0F6
:103F8000CE0101960E94F07FCE0101960E94387505
:103F900026960FB6F894DEBF0FBECDBFDF91CF914E
:103FA0001F910F9108950F931F93CF93DF93CDB778
:103FB000DEB72C970FB6F894DEBF0FBECDBF8C01D5
:103FC0000E94A97DBC01C8010E94221A0E94A17D05
:103FD000BC01CE0107960E94221A60EC76E0CE0169
:103FE00001960E94D775BE01695F7F4FCE01019691
:103FF0000E945374BC01C8010E94BC74CE0101969A
:104000000E943875CE0107960E9438750E94487C40
:104010000E948E7C6091410C70E0CE0107960E9458
:10402000221A60EC76E0CE0101960E94D775BE019F
:10403000695F7F4FCE0101960E945374BC01C80195
:104040000E94BC74CE0101960E943875CE0107967D
:104050000E9438756CED75E0C8010E94B2740E9430
:10406000997DBC01CE0101960E94221ABE016F5FAC
:104070007F4FC8010E94BC74CE0101960E94387522
:1040800066E674E0C8010E94B2740E94917DBC0192
:10409000CE0101960E94221ABE016F5F7F4FC801B8
:1040A0000E94BC74CE0101960E94387566E674E0E9
:1040B000C8010E94B2740E94877DBC01CE010196A6
:1040C0000E94221ABE016F5F7F4FC8010E94BC741C
:1040D000CE0101960E943875C8012C960FB6F8944F
:1040E000DEBF0FBECDBFDF91CF911F910F9108951D
:1040F0006115710519F00A960C94387690E080E00D
:1041000008952F923F924F925F926F927F928F927B
:104110009F92AF92BF92DF92EF92FF920F931F9305
:10412000CF93DF93CDB7DEB7E4970FB6F894DEBF39
:104130000FBECDBF7C014A015B0119010E94697A63
:104140002B013C0187010D5B1F4FC8010E94B00D80
:10415000181619069CF00E94697A64197509860977
:10416000970986169706A806B90608F490C162E377
:1041700070E080E090E00E94AB79E7CF42E250E04F
:10418000BE016F5F7F4FC8010E94670D8981823039
:1041900009F078C1F801848995898334910509F083
:1041A00071C16D817E818F8198850E9434AA2B0117
:1041B0003C01F101408251826282738246E050E00C
:1041C000B701685F7F4FCE014D960E9462AC892B8C
:1041D00099F4F70180819181A281B3814816590633
:1041E0006A067B0648F084819581A681B781841593
:1041F0009505A605B705E8F4C8010E945907D12C1A
:104200008D2DE4960FB6F894DEBF0FBECDBFDF91C3
:10421000CF911F910F91FF90EF90DF90BF90AF90E3
:104220009F908F907F906F905F904F903F902F90D6
:10423000089589899A89AB89BC8986879787A08BDD
:10424000B18B8EECA82EB12CC8010E94860DF1E036
:10425000AF1AB108C9F7D12CC70182969AA789A7CE
:10426000F701B696FCA7EBA708969EA78DA73C97EB
:104270004F01899698AB8FA73897FAABE9AB170136
:10428000F6E12F0E311CC5979CAB8BABF801818DED
:10429000928D181619060CF0F6C0C8010E94860D02
:1042A0008333910509F4D4C0A4F58130910509F454
:1042B00074C074F4892B51F3C8010E94860DB82E86
:1042C000BA94FFEFBF1611F3C8010E94860DF8CF14
:1042D0008330910509F46CC0069771F7C8010E94FC
:1042E000860DA82E44E050E06BA97CA9C8010E946D
:1042F000670D712C612CEA2DE450FF0B5F016A14ED
:104300007B0424F6C8010E94860DFFEF6F1A7F0A16
:10431000F6CF8A33910509F46FC074F585339105A2
:10432000A1F1C69749F6C8010E94860DB82EF70183
:10433000828D811109C0838D811106C0848D811108
:1043400003C0858D8823A1F0EFA5F8A94080518096
:1043500062807380B401CE0183960E946C778DA138
:104360009EA1AFA1B8A584159505A605B705D9F5F9
:1043700044E050E0B40118C08B33910509F452C0F9
:104380008F3F910509F482CF97CFC8010E94860D17
:10439000C8010E94860DD82E79CFC8010E94860DD3
:1043A00044E050E069A97AA9C8010E94670D6ECF68
:1043B000C8010E94860DA82E44E050E0B101C8015A
:1043C0000E94670D712C612C8A2D8450990B5C0121
:1043D0006A147B040CF05ACFC8010E94860D9FEF2F
:1043E000691A790AF5CFBA94FFEFBF1609F44ECFD8
:1043F000C8010E94860DF7CFC8010E94860D44E0D7
:1044000050E06BA57CA5C8010E94670DF70166A16D
:1044100077A180A591A50E9434AA66A377A380A75F
:1044200091A734CFC8010E94860D44E050E06DA5ED
:104430007EA5C8010E94670DF70162A573A584A53A
:1044400095A50E9434AA62A773A784A795A71ECF3B
:10445000C8010E94860D44E050E069A57AA5C80114
:104460000E94670DF70162A173A184A195A10E942A
:1044700034AA62A373A384A395A366A777A780AB8E
:1044800091AB04CFD12CC8010E945907B9CEDD24CD
:10449000DA94B6CE2F923F924F925F926F927F92B4
:1044A0008F929F92AF92BF92CF92DF92EF92FF9244
:1044B0000F931F93CF93DF9300D000D0CDB7DEB71B
:1044C0008C010E9451A12FEC37E040E050E00E94A7
:1044D000ACA8DC01CB010196A11DB11DF8018483BC
:1044E0009583A683B78380839183A283B383580186
:1044F000F3E4AF0EB11CC5010E94DF0E64E470E06E
:10450000C5010E94000F882309F445C10E94697A01
:104510002B013C01480182E4880E911C48EEC42E18
:1045200043E0D42EE12CF12C52E0252E1E821D8278
:10453000D4018C918330B1F1811166C0F80184817E
:104540009581A681B7810196A11DB11D84839583B4
:10455000A683B7830E94697A641975098609970949
:10456000A70196010E948AA8A90161E0C8010E94E2
:10457000661381E0D4018C938D819E810197C1F2F5
:104580000E94697A6419750986099709D801D69637
:104590002D913D914D915C91D9972617370748078A
:1045A000590720F6C5010E94DF0EF801848195812C
:1045B000A681B7810196A11DB11D84839583A68331
:1045C000B7830E94697AF801FE96608371838283C3
:1045D00093838D819E8126960FB6F894DEBF0FBE21
:1045E000CDBFDF91CF911F910F91FF90EF90DF90A2
:1045F000CF90BF90AF909F908F907F906F905F9083
:104600004F903F902F9008958430F1F4F801848109
:104610009581A681B7810196A11DB11D84839583E3
:10462000A683B7830E94697A641975098609970978
:10463000A70196010E948AA8A90163E0C8010E940F
:104640006613D4012C9298CF813051F5F80142AD18
:1046500053AD64AD75AD9E012F5F3F4FC8010E9401
:104660008120382EF2E08F1390C089819A81AB812E
:10467000BC81F80184839583A683B7830E94697AFD
:104680006419750986099709A70196010E948AA8ED
:10469000A90163E0C8010E946613D4013C926CCF6B
:1046A000823009F069CFF80142AD53AD64AD75AD0C
:1046B0009E012F5F3F4FC8010E948120382EF5E0F8
:1046C0008F135DC0E3E0D401EC93F80182A193A1C4
:1046D000A4A1B5A1892B8A2B8B2B41F484E893E00C
:1046E000A0E0B0E082A393A3A4A3B5A3F80186A1A0
:1046F00097A1A0A5B1A5892B8A2B8B2B61F482A150
:1047000093A1A4A1B5A1B695A7959795879586A3E2
:1047100097A3A0A7B1A7F80182A593A5A4A5B5A5C5
:10472000892B8A2B8B2BA9F482A193A1A4A1B5A1DB
:10473000AC01BD0123E076956795579547952A957D
:10474000D1F7841B950BA60BB70B82A793A7A4A741
:10475000B5A7F80186A197A1A0A5B1A586A797A79F
:10476000A0ABB1AB82A593A5A4A5B5A582AB93AB35
:10477000A4ABB5AB81E090E09E838D83FDCE96E047
:10478000891303C0D4011C92F7CEBFEF3B12F4CEC5
:10479000F4011082F1CE1E821D821BCFEF92FF9298
:1047A0000F931F93CF93DF93CDB7DEB7E8970FB684
:1047B000F894DEBF0FBECDBF63ED78E0CE018796E3
:1047C0000E94D77563ED78E0CE018D960E94D77573
:1047D00082E0E82EF12C2496FFAEEEAE249786E020
:1047E000EFEEF2E0DE01D39601900D928A95E1F7AB
:1047F00086E0FE01F396DE01AC5BBF4F01900D92A7
:104800008A95E1F72C961FAE1EAE2C9701E010E0C2
:104810002E961FAF0EAF2E9788E0E5EFF2E0DE0197
:10482000599601900D928A95E1F788E0FE017996FC
:10483000DE01A25BBF4F01900D928A95E1F788E1FE
:10484000EDEFF2E0DE01119601900D928A95E1F70D
:1048500088E1FE013196DE01AA5ABF4F01900D9208
:104860008A95E1F78091150390911603A0911703A3
:10487000B0911803E2968CAF9DAFAEAFBFAFE29799
:104880006CE674E0CE0187960E941B7360E0CE0157
:1048900087960E9490744BA55CA5BE016E587F4F11
:1048A000CE0187960E949B726BE577E0CE018D96D4
:1048B0000E94C37462EC74E085E691E10E941B7370
:1048C00060E0CE018D960E94907449A95AA9BE015C
:1048D00066567F4FCE018D960E949B7263ED78E005
:1048E000CE0187960E941B7363ED78E0CE018D9612
:1048F0000E941B73C250DF4F19821882CE5FD040D6
:104900008091830290918402C050DF4F9983888305
:10491000C050D14080E090E0A0E7B2E4CA5BDE4F37
:1049200088839983AA83BB83C654D140C65BDE4F7C
:10493000F982E882CA54D14080E090E0A0E2B2E47B
:10494000C45BDE4F88839983AA83BB83CC54D14058
:1049500080E090E0A4E3B2E4C05BDE4F88839983FB
:10496000AA83BB83C055D14084EB90E0CC5ADE4F84
:1049700099838883C455D14088E790E0CA5ADE4FB6
:1049800099838883C655D1408CE291E0A0E0B0E0E5
:10499000C85ADE4F88839983AA83BB83C855D14008
:1049A000C45ADE4F19830883CC55D140C25ADE4F1A
:1049B000F982E882CE55D14060E087E791E10E941C
:1049C000907460E081E791E10E94907440917B11C6
:1049D00050917C11BE016E5F7E4F87E791E10E948E
:1049E0009B724091751150917611BE01635F7E4FAD
:1049F00081E791E10E949B7288E2E0EEFBE0DE013C
:104A0000A75EBE4F01900D928A95E1F78CE390E08E
:104A1000A0E0B0E0CE5BDE4F88839983AA83BB839E
:104A2000C254D140CF5BDE4F1882C154D14084EED6
:104A300098E3AEE8B2E4C05ADE4F88839983AA8334
:104A4000BB83C056D14084EE98E3AEE8B1E4CC59C4
:104A5000DE4F88839983AA83BB83C456D140C8594B
:104A6000DE4F19830883C856D14080E590E0C659CF
:104A7000DE4F99838883CA56D14084EF91E09093AA
:104A80009B0280939A02BE016E5B7F4F0E9490084A
:104A900064EF71E080E090E00E94AB7964E477E03D
:104AA000CE0181960E94C575CE0181960E9465183F
:104AB000CE0181960E943875CE018D960E94387580
:104AC000CE0187960E943875E8960FB6F894DEBF3F
:104AD0000FBECDBFDF91CF911F910F91FF90EF904F
:104AE00008959F92AF92BF92CF92DF92EF92FF9282
:104AF0000F931F93CF93DF93CDB7DEB7C859D1097A
:104B00000FB6F894DEBF0FBECDBF5C017B016A011A
:104B100065E870E1CE0189579F4F0E94D77560E428
:104B200074E08E010F5F1F4FC8010E94D775B80156
:104B3000CE0189579F4F0E942274982EC8010E946F
:104B40003875911014C060E474E0C8010E94D775F4
:104B5000BE0169577F4FC8010E945374BC01CE014A
:104B600089579F4F0E94E874C8010E943875B501AB
:104B7000CE0183579F4F0E94D77564E774E0E1141C
:104B8000F10471F062E874E021E0E216F10441F012
:104B90006DE874E032E0E316F10411F065E974E0C9
:104BA000CE0189579F4F0E94B27460E0CE018957B1
:104BB0009F4F0E949074B601C8010E94CE756AE0B2
:104BC000C8010E94A474BC01CE018D569F4F0E9463
:104BD000CE75C8010E943875C557DF4F488159818D
:104BE000CB58D040B801CE0189579F4F0E949B728D
:104BF0008091760C882399F16DE974E0CE018F578E
:104C00009F4F0E94D775CE018F579F4F0E947C18EF
:104C1000CE018F579F4F0E943875BE0169577F4F55
:104C2000CE018F579F4F0E94CE75CE018F579F4F59
:104C30000E947C18CE018F579F4F0E943875B80193
:104C4000CE018F579F4F0E94D775CE018F579F4F30
:104C50000E947C18CE018F579F4F0E943875CC560A
:104C6000DF4F8881C459D0408F93CD56DF4F888164
:104C7000C359D0408F93C257DF4F8881CE58D04060
:104C80008F93C357DF4F8881CD58D0408F938DEAE3
:104C900094E09F938F938EE3E82E8AE0F82EFF92A4
:104CA000EF920E94E3AC40913502509136026CE0E5
:104CB0007CE08EE090E10E94F3120FB6F894DEBF24
:104CC0000FBECDBF019709F07CC01F930F9383EBFC
:104CD00094E09F938F9300E41BE01F930F930E9437
:104CE000E3ACB8018EE090E10E940A778CE09CE092
:104CF0009F938F9384EC94E09F938F931F930F93D4
:104D00000E94E3ACB8018EE090E10E940A7769E36B
:104D100074E08EE090E10E94487767EE79E08EE0E3
:104D200090E10E943876F70101900020E9F7CF0169
:104D30008F539A409F938F938DEC94E09F938F9322
:104D40001F930F930E94E3ACB8018EE090E10E94A4
:104D50000A77B7018EE090E10E941E7762E370E06F
:104D600080E090E00E94AB798EE090E10E94E01438
:104D70000FB6F894DEBF0FBECDBF11E0CE018D5649
:104D80009F4F0E943875CE0183579F4F0E94387500
:104D9000CE0189579F4F0E943875812FC856DF4F2B
:104DA0000FB6F894DEBF0FBECDBFDF91CF911F913C
:104DB0000F91FF90EF90DF90CF90BF90AF909F90BA
:104DC00008956CE774E0CE018F579F4F0E94C57520
:104DD000CE018F579F4F0E946518CE018F579F4F6E
:104DE0000E94387568E874E0CE018F579F4F0E948B
:104DF000C575CE018F579F4F0E947C18CE018F57EB
:104E00009F4F0E9438756EE37AE0CE018F579F4F17
:104E10000E94D775CE018F579F4F0E946518CE0113
:104E20008F579F4F0E94387510E0A8CF8F929F92A6
:104E3000AF92BF92EF92FF920F931F93CF93DF93A6
:104E4000CDB7DEB76E970FB6F894DEBF0FBECDBFFD
:104E50000091530E1091540E0115110509F4D8C09C
:104E60000E94697A4B015C0178012EE3E20EF11C8D
:104E7000F70180819181A281B381A5019401281B52
:104E8000390B4A0B5B0BCA01B901683E33E073076B
:104E900081059105A0F128EE33E040E050E00E944A
:104EA0008AA8861A970AA80AB90AD7018D929D92F4
:104EB000AD92BC921397F80186A597A5A0A9B1A9B8
:104EC00049015A01880C991CAA1CBB1C881599051C
:104ED000AA05BB0508F0C2C016A617A610AA11AAFB
:104EE000F80182A993A9A4A9B5A988159905AA05CD
:104EF000BB0508F0BCC012AA13AA14AA15AAF8018F
:104F000086A597A5A0A9B1A9892B8A2B8B2B09F07F
:104F1000B7C0EE5BFF4F8081833009F0B1C084E001
:104F20008083C8010E944A220196D801D2964D91F1
:104F30005D916D917C91D597452B462B472BA1F424
:104F4000F801EE5BFF4F2081233011F021110CC0DE
:104F50001082F8013E9684E1DF011D928A95E9F7FF
:104F6000C8010E944A2203968230910519F00497E5
:104F700009F04EC080E590E00E946C0C6091530EE9
:104F80007091540E625F7F4FCE0101960E946C7744
:104F9000CE0103960E94640C6091530E7091540EE2
:104FA0006A5E7F4FCE0101960E946C7744E050E02C
:104FB000BE016D5F7F4F81E090E00E946292609140
:104FC000530E7091540E6E5E7F4FCE0101960E947B
:104FD0006C7744E050E0BE016D5F7F4F85E090E06C
:104FE0000E9462926091530E7091540E625E7F4FE8
:104FF000CE0101960E946C778B819C81AD81BE8130
:1050000080934F0E9093500EA093510EB093520E7A
:1050100060ED77E080E090E00E94AB790E940C9315
:105020007C0168EE73E080E090E00E94AB7905E1DE
:1050300010E0EF28B1F50150110929F160ED77E09A
:1050400080E090E00E94AB790E940C937C0168EEB6
:1050500073E080E090E00E94AB79EBCF821B930B72
:10506000A40BB50B86A797A7A0ABB1AB39CF821B1A
:10507000930BA40BB50B82AB93ABA4ABB5AB3FCFFB
:1050800090E080E052CF8091650C9091660CA091E9
:10509000670CB091680C892B8A2B8B2B11F0F801CF
:1050A000199585EF9EE00E9474140E94611F63EDC4
:1050B00078E0CE010D960E94D7756BE875E0CE01C1
:1050C00043960E94C575CE0149960E947D728E8DD1
:1050D0001F928F938D8D1F928F938C8D1F928F9324
:1050E0008B8D1F928F9388E494E09F938F9380E43D
:1050F0009BE09F938F930E94E3AC60E47BE0CE0142
:1051000001960E94D775BE016F5F7F4FCE010D964D
:105110000E94FF74CE0101960E943875BE016D5E3B
:105120007F4FCE0101960E94CE75BE01635F7F4F17
:10513000CE0101960E945374BC01CE0107960E94D5
:10514000CE75CE0107960E946518CE0107960E9483
:105150003875CE0101960E943875BE01635F7F4F9E
:10516000CE0101960E94CE75AE014F5F5F4F63E0A6
:1051700070E085E892E00E947125182FCE0101961B
:105180000E9438750FB6F894DEBF0FBECDBF111167
:1051900022C062EE74E0CE0101960E94D775BE0176
:1051A0006D5E7F4FCE0101960E9453746DED7FE0DE
:1051B0000E945374BC01CE0107960E94CE75CE01A9
:1051C00007960E946518CE0107960E943875CE0199
:1051D00001960E943875CE0143960E943875CE0123
:1051E0000D960E9438756E960FB6F894DEBF0FBE0E
:1051F000CDBFDF91CF911F910F91FF90EF90BF90A6
:10520000AF909F908F9008957F928F929F92AF92D0
:10521000BF92CF92DF92EF92FF920F931F93CF93A3
:10522000DF93CDB7DEB762970FB6F894DEBF0FBE3F
:10523000CDBF68E775E0CE0101960E94C575CE012D
:1052400001960E946518CE0101960E94387506E00D
:1052500010E03CE0C32E3BE0D32E40E3E42E53EEBF
:10526000B52E66E0A62E7CEE972EE1E3FE2EFEE440
:105270008F2EA4E37A2E68EB72E280EB9FE00E940F
:10528000000FF6018E2D11928A95E9F7B0920C0B62
:10529000A0920E0B90920F0BF092180B8092190BAC
:1052A000F0921A0B70921B0B60E072E0CE01019637
:1052B0000E946C774BE750E0BE016F5F7F4F80EB41
:1052C0009FE00E94C00F40E350E06CE07BE080EB89
:1052D0009FE00E94580F80EB9FE00E948E0F68EEC7
:1052E00073E080E090E00E94AB7980EB9FE00E9449
:1052F000B00D892B09F04FC00150110909F07CC095
:1053000080913C0B90913D0BA0913E0BB0913F0BD7
:10531000892B8A2B8B2B09F089C063ED78E08BEF0A
:105320009FE00E941B736BEF7FE0CE0101960E940D
:10533000CE75AE014F5F5F4F70E060E089E692E0AE
:105340000E947125182FCE0101960E943875111107
:105350000EC060E675E0CE0101960E94C575CE01D3
:1053600001960E946518CE0101960E9438756296DA
:105370000FB6F894DEBF0FBECDBFDF91CF911F9166
:105380000F91FF90EF90DF90CF90BF90AF909F90E4
:105390008F907F90089540E350E06CE07BE080EBDD
:1053A0009FE00E94670D6091340B7091350B76275A
:1053B0006727762790E080E0CB017727662700916A
:1053C000360B1091370B10270127102730E020E013
:1053D000602B712B822B932B7E508A4A93480E941C
:1053E000237C0E94487C60933C0B70933D0B809320
:1053F0003E0B90933F0B84CF68EE73E080E090E02B
:105400000E94AB7940913C0B50913D0B60913E0B5B
:1054100070913F0B2AE089E59DE00E94477667EE98
:1054200079E089E59DE00E94387625CF68EE73E04B
:1054300080E090E00E94AB790E94487C6093650C0C
:105440007093660C8093670C9093680C0E94487C64
:105450006093690C70936A0C80936B0C90936C0C46
:10546000CE0101960E94D31FBE016F5F7F4F89E579
:105470009DE00E943477CE0101960E9438750E940B
:10548000997DBC01CE0107960E94221A66E674E05F
:10549000CE0107960E94B2740E94917DBC01CE019C
:1054A00001960E94221ABE016F5F7F4FCE010796C0
:1054B0000E94BC74CE0101960E94387566E674E0C5
:1054C000CE0107960E94B2740E94877DBC01CE0176
:1054D00001960E94221ABE016F5F7F4FCE01079690
:1054E0000E94BC74CE0101960E9438756BEE74E088
:1054F000CE0101960E94D775BE01695F7F4FCE0134
:1055000001960E945374BC01CE010D960E94CE7587
:105510004AE050E06FEF7FEFCE010D960E948C19AC
:10552000CE010D960E943875CE0101960E94387505
:10553000CE0107960E94387568EE73E080E090E037
:105540000E94AB790E94A97DBC01CE010D960E94FC
:10555000221A0E94A17DBC01CE0101960E94221A4E
:1055600060EC76E0CE0107960E94D775BE016F5FB2
:105570007F4FCE0107960E945374BC01CE010D9659
:105580000E94BC74CE0107960E943875CE01019628
:105590000E9438750E94487C0E948E7C6091410C6C
:1055A00070E0CE0101960E94221A60EC76E0CE01F6
:1055B00007960E94D775BE016F5F7F4FCE01079699
:1055C0000E945374BC01CE010D960E94BC74CE01A2
:1055D00007960E943875CE0101960E94387561EFDA
:1055E00074E0CE0101960E94D775BE01635F7F4FC4
:1055F000CE0101960E945374BC01CE0107960E9411
:10560000CE754AE050E06FEF7FEFCE0107960E9423
:105610008C19CE0107960E943875CE0101960E9422
:105620003875CE010D960E94387568EE73E080E003
:1056300090E00E94AB79CE0101960E94E01E4AE004
:1056400050E06FEF7FEFCE0101960E948C198BCE58
:10565000CF92DF92EF92FF920F931F93CF93DF933E
:10566000CDB7DEB768970FB6F894DEBF0FBECDBFDB
:1056700063ED78E0CE0143960E94D7756AE578E045
:10568000CE0101960E94C575CE0101960E947C183C
:10569000CE0101960E9438756CA17DA1CE010196C4
:1056A0000E942573CE0101960E946518CE010196D5
:1056B0000E9438756DE478E0CE0101960E94C575B0
:1056C000CE0101960E947C18CE0101960E94387589
:1056D0007E0188E2E80EF11C01E010E08CA19DA1A2
:1056E000801791070CF1F701619171917F01CE0153
:1056F00001960E942573CE0101960E947C18CE016E
:1057000001960E9438756CED75E0CE0101960E94FD
:10571000D775CE0101960E947C18CE0101960E9499
:1057200038750F5F1F4FDACF6CED75E0CE01019633
:105730000E94D775CE0101960E946518CE01019690
:105740000E9438756EE378E0CE0101960E94C5751F
:10575000CE0101960E947C18CE0101960E943875F8
:105760006091D50B7091D60BCE0101960E942573E6
:10577000CE0101960E947C18CE0101960E943875D8
:105780006CED75E0CE0101960E94D775CE010196B1
:105790000E947C18CE0101960E9438756091D70B4B
:1057A0007091D80BCE0101960E942573CE0101960F
:1057B0000E946518CE0101960E94387567E278E074
:1057C000CE0101960E94C575CE0101960E947C18FB
:1057D000CE0101960E943875BE01605D7F4FCE01FB
:1057E00001960E94D775CE0101960E947C18CE01C9
:1057F00001960E9438756CED75E0CE0101960E940D
:10580000D775CE0101960E947C18CE0101960E94A8
:105810003875BE016C5C7F4FCE0101960E94D77532
:10582000CE0101960E946518CE0101960E9438753E
:1058300067E178E0CE0101960E94C575CE01019620
:105840000E946518CE0101960E9438758E010C5D8C
:105850001F4FEE24E394F12C6801F8E0CF0ED11C29
:105860008CA19DA18E159F050CF449C0B701CE01F6
:1058700007960E9425736CE877E0CE0101960E949E
:10588000D775BE01695F7F4FCE0101960E945374A8
:10589000BC01CE010D960E94CE75CE010D960E94E0
:1058A0007C18CE010D960E943875CE0101960E949B
:1058B0003875CE0107960E94387560EC76E0CE010F
:1058C00001960E94D775CE0101960E947C18CE01E8
:1058D00001960E943875B801645E7F4FCE01019633
:1058E0000E94D775CE0101960E946518CE010196DF
:1058F0000E9438758FEFE81AF80A8601ADCF6DEF78
:1059000077E0CE0101960E94C575CE0101960E94F6
:105910007C18CE0101960E9438756CE07CE0CE01C7
:1059200001960E94D775CE0101960E947C18CE0187
:1059300001960E9438756BEF77E0CE0101960E94C8
:10594000C575CE0101960E947C18CE0101960E9479
:1059500038756091350270913602CE0101960E9431
:105960002573CE0101960E946518CE0101960E9412
:1059700038756CEE77E0CE0101960E94C575CE01B8
:1059800001960E947C18CE0101960E943875BE01D6
:105990006C5A7F4FCE0101960E94D775CE010196B9
:1059A0000E946518CE0101960E94387567EF74E079
:1059B000CE0101960E94D775CE0101960E947C18F7
:1059C000CE0101960E943875BE0164587F4FCE010A
:1059D00001960E94D775CE0101960E946518CE01EE
:1059E00001960E943875C052DF4F88819981C05E50
:1059F000D040892B71F464EE77E0CE0101960E94CD
:105A0000C575CE0101960E946518CE0101960E94CF
:105A10003875C052DF4F88819981C05ED0400197B0
:105A200071F46AED77E0CE0101960E94C575CE0152
:105A300001960E946518CE0101960E943875C052E9
:105A4000DF4F88819981C05ED040029771F461ED8B
:105A500077E0CE0101960E94C575CE0101960E94A5
:105A60006518CE0101960E9438756BEC77E0CE0187
:105A700001960E94C575CE0101960E947C18CE0148
:105A800001960E943875CE51DF4F68817981C25EE0
:105A9000D040CE0101960E942573CE0101960E944E
:105AA0006518CE0101960E94387540915D0C5091A9
:105AB0005E0C60915F0C7091600C21E0CE01079646
:105AC0000E94407562E075E0CE0101960E94D77594
:105AD000BE01695F7F4FCE0101960E9453746DE055
:105AE00075E00E943D74BC01CE010D960E94CE75FA
:105AF000CE010D960E946518CE010D960E94387554
:105B0000CE0101960E943875CE0107960E94387525
:105B10004091590C50915A0C60915B0C70915C0C47
:105B200021E0CE0107960E94407562E175E0CE014A
:105B300001960E94D775BE01695F7F4FCE01019625
:105B40000E9453746DE075E00E943D74BC01CE016B
:105B50000D960E94CE75CE010D960E946518CE015D
:105B60000D960E943875CE0101960E943875CE01BF
:105B700007960E9438756DEA77E0CE0101960E9483
:105B8000C575CE0101960E947C18CE0101960E9437
:105B9000387540912002509121026091220270914B
:105BA000230225E0CE0101960E944075CE010196A8
:105BB0000E946518CE0101960E94387563E977E06E
:105BC000CE0101960E94C575CE0101960E947C18F7
:105BD000CE0101960E94387540911C0250911D0221
:105BE00060911E0270911F0225E0CE0101960E9475
:105BF0004075CE0101960E946518CE0101960E9463
:105C0000387563E877E0CE0101960E94C575CE0134
:105C100001960E947C18CE0101960E943875609111
:105C2000AA027091AB02CE0101960E942573CE01AB
:105C300001960E946518CE0101960E94387561E7B1
:105C400077E0CE0101960E94C575CE0101960E94B3
:105C50007C18CE0101960E943875C65BDE4F6881C4
:105C60007981CA54D140CE0101960E942573CE019C
:105C700001960E946518CE0101960E943875CE01EA
:105C800043960E94387568960FB6F894DEBF0FBE33
:105C9000CDBFDF91CF911F910F91FF90EF90DF90DB
:105CA000CF9008952F923F924F925F926F927F9282
:105CB0008F929F92AF92BF92CF92DF92EF92FF921C
:105CC0000F931F93CF93DF93CDB7DEB7EF970FB648
:105CD000F894DEBF0FBECDBF3C018B0170E060E0E9
:105CE0000E94F1738F8F63ED78E0CE0149960E9498
:105CF000D7758091AA029091AB028130910509F08D
:105D000092C028E030E030931B0220931A0229E071
:105D100030E030931902209318022091D30B309178
:105D2000D40B3093D20B2093D10B4091140250919D
:105D30001502609116027091170240931002509361
:105D40001102609312027093130240912C02509141
:105D50002D0260912E0270912F02409330025093D9
:105D6000310260933202709333022091D00B209362
:105D7000CF0B4091CB0B5091CC0B6091CD0B709120
:105D8000CE0B4093C70B5093C80B6093C90B709315
:105D9000CA0B2AE330E030930F0220930E024091A9
:105DA0005D0C50915E0C60915F0C7091600C4093A3
:105DB000080C5093090C60930A0C70930B0C209103
:105DC0000C0230910D0230930B0220930A02409195
:105DD000200250912102609122027091230240938F
:105DE00024025093250260932602709327022F8D80
:105DF000233509F08AC01092D20B1092D10B8091FA
:105E0000D90B882371F069E175E0CE0101960E94FB
:105E1000D775CE0101960E946518CE0101960E94A9
:105E20003875E12C5AC18230910509F72AE030E03B
:105E300030931B0220931A022BE030E030931902BA
:105E4000209318022091C50B3091C60B3093D20BD2
:105E50002093D10B409106025091070260910802F5
:105E60007091090240931002509311026093120244
:105E700070931302409128025091290260912A02E6
:105E800070912B02409330025093310260933202A2
:105E9000709333022091C40B2093CF0B4091C00B21
:105EA0005091C10B6091C20B7091C30B4093C70B13
:105EB0005093C80B6093C90B7093CA0B2BE330E06F
:105EC00030930F0220930E024091590C50915A0CBE
:105ED00060915B0C70915C0C4093080C5093090C22
:105EE00060930A0C70930B0C209104023091050210
:105EF00030930B0220930A0240911C0250911D0224
:105F000060911E0270911F026ACF980121503109E1
:105F10002230310508F001C281E090E0A0E0B0E05D
:105F20008093100290931102A0931202B093130277
:105F3000D30114968D919C91029748F141E050E075
:105F4000B301CE0101960E94D108BE016F5F7F4F61
:105F5000CE0149960E94FF74CE0101960E943875C9
:105F6000CE0149960130110581F50E947E7320E033
:105F700030E040E251E40E94A6A70E94CCA96093C1
:105F80001002709311028093120290931302BF8D3E
:105F900081E090E09093D20B8093D10BB13401F566
:105FA0008091D90B882309F43CCF6EE175E0CE01D6
:105FB00001960E94D775CE0101960E946518CE0108
:105FC00001960E943875E12C55C00E947E73209185
:105FD0002402309125024091260250912702CBCF16
:105FE000EF8DE63409F054C161E080911A020E94FD
:105FF000387864E670E080E090E00E94AB7961E080
:1060000080911A020E94387864E670E080E090E0A7
:106010000E94AB7902301105C1F4CE0149960E946D
:106020007E739B01AC016091080C7091090C80910A
:106030000A0C90910B0C0E94EDA86093080C7093D1
:10604000090C80930A0C90930B0C8091D90B882338
:1060500071F067E275E0CE0101960E94D775CE011E
:1060600001960E947C18CE0101960E943875EE249C
:10607000E394F12C8091D90B882379F1409110029F
:106080005091110260911202709113022AE0CE0128
:1060900001960E947675BE016F5F7F4FCE01079615
:1060A0000E94CE756BE375E0CE0107960E943D74A9
:1060B000BC01CE010D960E94CE75CE010D960E94B8
:1060C0006518CE010D960E943875CE0107960E9484
:1060D0003875CE0101960E9438758091100290911A
:1060E0001102A0911202B0911302181619061A0695
:1060F0001B060CF0D8C55F8D563409F4E0C4523548
:1061000009F4E1C46E2D80911A020E94387864E689
:1061100070E080E090E00E94AB796091D10B8091BB
:1061200018020E94387861E070E080E090E00E9400
:10613000AB7960E0809118020E94387868EC70E0DA
:1061400080E090E00E94AB79C12CD12C7601C39401
:106150008091100290911102A0911202B09113024D
:10616000C816D906EA06FB060CF0AFC46091D10B45
:10617000809118020E94387861E070E080E090E041
:106180000E94AB7960E0809118020E94387860919B
:1061900030027091310280913202909133020E945C
:1061A000AB798091300290913102A0913202B0918E
:1061B00033020B97A105B1050CF464C06091240271
:1061C0007091250280912602909127029B01AC01DB
:1061D0000E94EEA80E94CCA99B01AC01C701B601A8
:1061E0000E94ACA8672B682B692B09F04BC00230CA
:1061F00011050CF447C068E975E082E99FE00E9450
:10620000C374C701B6010E9447A7209124023091B0
:10621000250240912602509127020E945AA9AB0103
:10622000BC0120E0CE0107960E94407562E97FE044
:10623000CE0101960E94CE75BE01695F7F4FCE01EF
:1062400001960E9453746DE075E00E943D74BC019C
:1062500082E99FE00E94E874CE0101960E943875A1
:10626000CE0107960E94387562E97FE0CE01019663
:106270000E94CE75CE0101960E94A01FCE0101960C
:106280000E9438758FEFC81AD80AE80AF80A60CF5A
:10629000FF8DF23509F097CE60E080911A020E94DE
:1062A000387864E670E080E090E00E94AB7960E0CE
:1062B00080911A020E94387864E670E080E090E0F5
:1062C0000E94AB7902301105C1F4CE0149960E94BB
:1062D0007E739B01AC016091080C7091090C809158
:1062E0000A0C90910B0C0E94EEA86093080C70931E
:1062F000090C80930A0C90930B0C8091D90B882386
:1063000009F48FCD61E375E0CE0101960E94D77547
:10631000CE0101960E947C1852CE0115110521F084
:106320000330110509F07DCD20E137E240E050E077
:106330008130910521F420E43CE940E050E029ABB4
:106340003AAB4BAB5CAB21E030E03093D20B209307
:10635000D10B3093680220936702029759F40330FF
:10636000110541F48091531190915411909368025A
:1063700080936702409167025091680258AB4FA723
:10638000551F5527551F5DAB81E090E09093680243
:1063900080936702652F80911A020E94387864E624
:1063A00070E080E090E00E94AB796DA980911A02C4
:1063B0000E94387864E670E080E090E00E94AB795B
:1063C0008FEF9FEF90930B0280930A02812C912C08
:1063D00054011BA61CA61DA61EA61FA218A619A620
:1063E0001AA61BA21CA21DA21EA2212C312C210127
:1063F0001AAE1BAE1CAE1DAE1EAA1FAA18AE19AE59
:1064000061E0809118020E94387861E070E080E0DD
:1064100090E00E94AB7960E0809118020E94387889
:1064200061E070E080E090E00E94AB79C501B401CA
:1064300026E030E040E050E00E94ACA8672B682BDB
:10644000692B09F0F8C0A2E0B0E0BFAFAEAFC12C3D
:10645000D12C760180910E02863308F0865320916C
:106460007B00982F9870277F922B90937B008770EA
:10647000806480937C0080917A00806480937A00AD
:1064800080917A0086FDFCCF809178006091790040
:10649000762F682F072E000C880B990B0E9447A7B8
:1064A0009B01AC01C701B6010E94EEA86B017C0103
:1064B00062E070E080E090E00E94AB792EAD3FADED
:1064C0002130310509F0ADC020E030EC4FEF54E44D
:1064D000C701B6010E945AA96B017C018091D90BBA
:1064E000882399F12DEC3CEC4CE45EE3C701B60146
:1064F0000E9402AA87FD29C022E0B701A601CE01B1
:1065000007960E94407562E475E0CE0101960E94F4
:10651000D775BE01695F7F4FCE0101960E9453740B
:10652000BC01CE010D960E94CE75CE010D960E9443
:106530006518CE010D960E943875CE0101960E9415
:106540003875CE0107960E9438752AE939E949E97C
:106550005EE3C701B6010E9402AA87FD13C02114A1
:1065600031044104510411F4140125018FA198A5AF
:10657000A9A5BAA5892B8A2B8B2B21F48FA298A6CB
:10658000A9A6BAA62DEC3CEC4CE45EE3C701B6012B
:106590000E9440A718160CF449C02114310441048C
:1065A000510409F448C02BA13CA14DA15EA1232BAD
:1065B000242B252B69F48BA59CA5ADA5BEA5892B05
:1065C0008A2B8B2B09F401C18BA29CA2ADA2BEA287
:1065D0002BA13CA14DA15EA122163306440655060F
:1065E00054F580910A0290910B0297FFF3C010922C
:1065F0000B0210920A02220E331E441E551ED201B7
:10660000C101B595A795979587958AAF9BAFACAF1C
:10661000BDAF1BA21CA21DA21EA2212C312C210148
:106620000AC0E1E0F0E0FFAFEEAF14CF2114310477
:106630004104510469F6E0900A02F0900B0292E0E6
:10664000E916F10434F4F7FCE1C00330110509F058
:10665000DDC089A89AA8ABA8BCA8AAE08A0E911CA4
:10666000A11CB11C89A99AA9ABA9BCA98816990635
:10667000AA06BB060CF4C4CEE2E0EE16F1040CF45C
:1066800079C06EA97FA988AD99AD2AAD3BAD4CAD5F
:106690005DAD621B730B840B950B0E9447A74B01EA
:1066A0005C01B701FF0C880B990B0E9447A79B0167
:1066B000AC01C501B4010E945AA920E030E044EBCE
:1066C00053E40E945AA96B017C01C0922402D0922B
:1066D0002502E0922602F092270220E030E040E816
:1066E0005FE30E9402AA87FDABC08091AA0290914D
:1066F000AB028130910509F08FC0C0924B11D0924E
:106700004C11E0924D11F0924E11C0922002D092A5
:106710002102E0922202F09223026BEB75E0CE019F
:1067200001960E94C575CE0101960E947C18CE018B
:1067300001960E9438754091240250912502609183
:1067400026027091270225E0CE0101960E94407535
:10675000CE0101960E946518CE0101960E943875FF
:1067600084EF91E090939B0280939A026DE270E136
:106770000E9490080330110531F03DA9E32E011568
:10678000110509F0AACCC3010E947E736B017C0144
:10679000C092080CD092090CE0920A0CF0920B0CFB
:1067A00020E030E044EB53E4C701B6010E9402AAA6
:1067B00087FD6AC020E030E044EB53E4C701B60136
:1067C0000E94EDA86B017C01EBCF8BA69CA6ADA629
:1067D000BEA6FACE0115110509F02DCF01969093B2
:1067E0000B0280930A022BA13CA14DA15EA1220EB7
:1067F000331E441E551ED201C101B595A79597952C
:1068000087958EAB9FABA8AFB9AF03CFBFEF8B1A05
:106810009B0AAB0ABB0A26CF029709F07ECFC09233
:106820004F11D0925011E0925111F0925211C0923A
:106830001C02D0921D02E0921E02F0921F026DCF48
:106840006FE975E0CE0101960E94C575CE010196F3
:106850000E947C18CE0101960E9438754091240256
:1068600050912502609126027091270225E0CE0109
:1068700001960E944075CE0101960E946518CE01D6
:1068800001960E94387576CF20E030E0A901C7015B
:10689000B6010E9440A787FF0BC020E030E044EB28
:1068A00053E4C701B6010E94EEA86B017C01ECCF56
:1068B000C092C70BD092C80BE092C90BF092CA0BE2
:1068C0004BA45CA46DA47EA48FA198A5A9A5BAA58C
:1068D000481A590A6A0A7B0A01151105D9F410925F
:1068E000C70B1092C80B1092C90B1092CA0BAFA520
:1068F000B8A9812C912C54018394C12CD12C760100
:10690000B7FF26C0C12CD12C760188248A94982CFC
:1069100054011EC0EFA5F8A9812C912C5401839439
:10692000F7FF04C088248A94982C5401C090C70BA8
:10693000D090C80BE090C90BF090CA0B20E030E07B
:1069400044E353E4C701B6010E9440A787FF92C009
:10695000C701B60190582091240230912502409140
:106960002602509127020E94A6A76B017C01A30179
:106970009201C501B4010E947AA80E9447A720E0B5
:1069800030E040E05FE30E94A6A79B01AC01C70195
:10699000B6010E94EDA80E94CCA9609310027093EA
:1069A000110280931202909313028091D90B8823D5
:1069B00009F441C02AE04BA55CA56DA57EA5CE01DA
:1069C0000D960E9476752AE04FA158A569A57AA573
:1069D000CE0107960E94767569E475E0CE010196B6
:1069E0000E94D775BE01695F7F4FCE0101960E945C
:1069F00053746CED75E00E943D74BE01635F7F4F80
:106A00000E945374BC01CE0143960E94CE75CE0104
:106A100043960E946518CE0143960E943875CE01B8
:106A200001960E943875CE0107960E943875CE01F6
:106A30000D960E9438758091100290911102A091DC
:106A40001202B0911302B7FF36C0B095A095909591
:106A500081959F4FAF4FBF4F8093100290931102CB
:106A6000A0931202B0931302EE24E394F12C36E4C7
:106A70003F8F33CB20912402309125024091260292
:106A8000509127022F8F38A349A35AA3A70196013B
:106A900060E070E084EB93E40E94EDA86093C70B84
:106AA0007093C80B8093C90B9093CA0B2F8D38A19C
:106AB00049A15AA158CFE12C42E54F8F0ECBEE24CD
:106AC000E394F12C1FCBE12C1DCB0230110524F4F3
:106AD0000115110509F0DFC061E080E00E94C37F6D
:106AE0000230110524F40115110509F09CC0C09075
:106AF000080CD090090CE0900A0CF0900B0C20E0F0
:106B000030E044EB53E4C701B6010E9402AA87FDBE
:106B10000BC020E030E044EB53E4C701B6010E9413
:106B2000EDA86B017C01EBCF20E030E0A901C701AB
:106B3000B6010E9440A787FF0BC020E030E044EB85
:106B400053E4C701B6010E94EEA86B017C01ECCFB3
:106B5000C092080CD092090CE0920A0CF0920B0C37
:106B60008091AA029091AB020197B1F462E075E0C6
:106B700082E99FE00E941B738091080C9091090CA0
:106B8000A0910A0CB0910B0C80935D0C90935E0C5D
:106B9000A0935F0CB093600C8091AA029091AB021D
:106BA0000297B1F462E175E082E99FE00E941B73F5
:106BB0008091080C9091090CA0910A0CB0910B0CDB
:106BC0008093590C90935A0CA0935B0CB0935C0C7F
:106BD0004091080C5091090C60910A0C70910B0CBB
:106BE00020E0CE0107960E94407562E97FE0CE0169
:106BF00001960E94CE75BE01695F7F4FCE0101965E
:106C00000E9453746EE075E00E943D74BC0182E9FD
:106C10009FE00E94E874CE0101960E943875CE0173
:106C200007960E9438750130110539F54091100220
:106C300050911102609112027091130221E0CE0175
:106C400007960E94767561E575E0CE0101960E9477
:106C5000D775BE01695F7F4FCE0101960E945374C4
:106C6000BC0182E99FE00E94E874CE0101960E9477
:106C70003875CE0107960E94387562E97FE0CE0133
:106C800001960E94CE75CE0101960E94A01FCE01F2
:106C900001960E9438751092100210921102109203
:106CA0001202109213028091AA029091AB028130DD
:106CB000910509F083C08091D10B9091D20B9093F4
:106CC000D40B8093D30B8091100290911102A0916C
:106CD0001202B09113028093140290931502A093B4
:106CE0001602B09317028091300290913102A09168
:106CF0003202B091330280932C0290932D02A09324
:106D00002E02B0932F028091CF0B8093D00B8091F5
:106D1000C70B9091C80BA091C90BB091CA0B80937F
:106D2000CB0B9093CC0BA093CD0BB093CE0B80915B
:106D3000080C9091090CA0910A0CB0910B0C809357
:106D40005D0C90935E0CA0935F0CB093600C8091EF
:106D50000A0290910B0290930D0280930C02012B7A
:106D600081F48091240290912502A0912602B09195
:106D700027028093200290932102A0932202B093D5
:106D80002302CE0149960E943875EF960FB6F8940B
:106D9000DEBF0FBECDBFDF91CF911F910F91FF904E
:106DA000EF90DF90CF90BF90AF909F908F907F90AB
:106DB0006F905F904F903F902F900895029709F742
:106DC0008091D10B9091D20B9093C60B8093C50B01
:106DD0008091100290911102A0911202B0911302C1
:106DE0008093060290930702A0930802B0930902D1
:106DF0008091300290913102A0913202B091330221
:106E00008093280290932902A0932A02B0932B0228
:106E10008091CF0B8093C40B8091C70B9091C80BCE
:106E2000A091C90BB091CA0B8093C00B9093C10B7A
:106E3000A093C20BB093C30B8091080C9091090CE6
:106E4000A0910A0CB0910B0C8093590C90935A0CA2
:106E5000A0935B0CB0935C0C80910A0290910B02A2
:106E60009093050280930402012B09F08ACF809150
:106E7000240290912502A0912602B09127028093CE
:106E80001C0290931D02A0931E02B0931F0279CFA3
:106E90004F925F926F927F928F929F92AF92BF922A
:106EA000CF92DF92EF92FF920F931F93CF93DF93D6
:106EB000CDB7DEB7ED970FB6F894DEBF0FBECDBFEE
:106EC0006AEA7FE0CE01C4960E94CE750CA91DA986
:106ED0000115110571F0F80181918F01882349F0A6
:106EE000082E000C990B0E945AACF8013197808350
:106EF000F2CF68E575E0CE0101960E94D775BE011C
:106F00006F5F7F4FCE01C4960E942274182FCE016E
:106F100001960E943875112309F4FFC045E050E046
:106F20006AEA7FE0CE0101960E94D108BE016F5F40
:106F30007F4F8CE89FE00E94FF74CE0101960E9473
:106F400038758CE89FE00E94947360E08CE89FE0C5
:106F50000E9490744091900F5091910F65E870E1FC
:106F60008CE89FE00E949B7260E474E0CE01019681
:106F70000E94D775BE016F5F7F4F8CE89FE00E9433
:106F80002274182FCE0101960E9438756AE274E0CF
:106F9000111102C06FE274E0CE0101960E94D77514
:106FA0006CE87FE0CE0101960E945374BC0183E837
:106FB00091E10E94E874CE0101960E94387583E841
:106FC00091E10E9494734091871150918811415032
:106FD000510963E871E1CE0101960E94D108BE011A
:106FE0006F5F7F4F85E691E10E94FF74CE010196AD
:106FF0000E94387585E691E10E9489730E9447A737
:107000009B01AC010E9407AA882309F448C0609143
:107010008711709188116250710983E891E10E9493
:10702000F173682FCE0101960E94A375BE016F5FB8
:107030007F4F85E691E10E94FF74CE0101960E9488
:10704000387560E474E0CE0101960E94D775BE01E8
:107050006F5F7F4F85E691E10E942274182FCE0169
:1070600001960E9438751123D1F0609187117091BB
:1070700088116350710983E891E10E94F173682FD0
:10708000CE0101960E94A375BE016F5F7F4F85E61A
:1070900091E10E94FF74CE0101960E94387584EF41
:1070A00091E090939B0280939A026DE270E10E94BE
:1070B000900864E670E080E090E00E94AB798091F7
:1070C0003402882371F06AEA7FE0CE0101960E94C3
:1070D000CE75CE0101960E94691DCE0101960E94D7
:1070E0003875CE01C4960E94387581E0ED960FB6D2
:1070F000F894DEBF0FBECDBFDF91CF911F910F91EE
:10710000FF90EF90DF90CF90BF90AF909F908F90C7
:107110007F906F905F904F9008956EE575E0CE017F
:1071200001960E94D775BE016F5F7F4FCE01C49656
:107130000E942274182FCE0101960E9438751123E7
:1071400009F447C045E050E06AEA7FE0CE010196CD
:107150000E94D108BE016F5F7F4F8CE89FE00E94C4
:10716000FF74CE0101960E9438758CE89FE00E9462
:10717000947360E08CE89FE00E9490744091900FBF
:107180005091910F6DE570E18CE89FE00E949B7239
:107190006DE570E1CE014C960E94D77562E474E013
:1071A000CE0101960E94D775BE01645E7F4FCE016D
:1071B00001960E945374BC018DE791E10E94E8742E
:1071C000CE0101960E943875CE014C960E9438750A
:1071D00066CF64E675E0CE0101960E94D775BE01C8
:1071E0006F5F7F4FCE01C4960E942274182FCE018C
:1071F00001960E9438751123E1F043E050E06AEAFD
:107200007FE0CE0101960E94D108BE016F5F7F4FE3
:107210008CE89FE00E94FF74CE0101960E943875B1
:107220006CE87FE0CE0101960E94CE75CE010196FA
:10723000CDCF68E675E0CE0101960E94D775BE01FC
:107240006F5F7F4FCE01C4960E942274182FCE012B
:1072500001960E943875112301F144E050E06AEA7A
:107260007FE0CE0101960E94D108BE016F5F7F4F83
:107270008CE89FE00E94FF74CE0101960E94387551
:107280008CE89FE00E9489737093EC106093EB1080
:10729000709384026093830202CF6DE675E0CE01A5
:1072A00001960E94D775BE016F5F7F4FCE01C496D5
:1072B0000E942274182FCE0101960E943875112366
:1072C00009F449C045E050E06AEA7FE0CE0101964A
:1072D0000E94D108BE016F5F7F4F8CE89FE00E9443
:1072E000FF74CE0101960E9438758CE89FE00E94E1
:1072F0008973709348116093471184EF91E09093E4
:107300009B0280939A026DE270E10E94900864E60D
:1073100070E080E090E00E94AB796CE877E0CE010D
:1073200001960E94D7756AEA7FE0CE0101960E941D
:107330005374BC01CE014C960E94CE75CE014C9682
:107340000E946518CE014C960E943875CE010196B8
:107350000E943875B4CE63E775E0CE0101960E94B5
:10736000D775BE016F5F7F4FCE01C4960E94227415
:10737000182FCE0101960E9438751123E1F044E0E8
:1073800050E06AEA7FE0CE0101960E94D108BE017A
:107390006F5F7F4F8CE89FE00E94FF74CE010196E3
:1073A0000E9438758CE89FE00E94897370934A119F
:1073B00060934911A2CF68E775E0CE0101960E9463
:1073C000D775BE016F5F7F4FCE01C4960E942274B5
:1073D000182FCE0101960E9438751123A1F044E0C8
:1073E00050E06AEA7FE0CE0101960E94D108BE011A
:1073F0006F5F7F4F8CE89FE00E94FF74CE01019683
:107400000E94387584CF6DE775E0CE0101960E9429
:10741000D775BE016F5F7F4FCE01C4960E94227464
:10742000182FCE0101960E9438751123A1F047E074
:1074300050E06AEA7FE0CE0101960E94D108BE01C9
:107440006F5F7F4F8CE89FE00E94FF74CE01019632
:107450000E9438752ECE65E875E0CE0101960E9437
:10746000D775BE016F5F7F4FCE01C4960E94227414
:10747000182FCE0101960E9438751111D8CF6DE8F2
:1074800075E0CE0101960E94D775BE016F5F7F4FF8
:10749000CE01C4960E942274182FCE0101960E943C
:1074A0003875112321F081E00E94FE0702CE67E9C2
:1074B00075E0CE0101960E94D775BE016F5F7F4FC8
:1074C000CE01C4960E942274182FCE0101960E940C
:1074D0003875112319F00E941627EBCD6BE27AE084
:1074E000CE0101960E94C575BE016F5F7F4FCE0130
:1074F000C4960E942274182FCE0101960E943875FE
:10750000112309F485C060E27AE0CE0101960E9461
:10751000C575BE016F5F7F4FCE01C4960E94227475
:10752000182FCE0101960E943875112309F454C01A
:107530004AE050E06AEA7FE0CE0101960E94D1085D
:10754000BE016F5F7F4F8CE89FE00E94FF74CE0109
:1075500001960E9438758CE89FE00E9489730E9412
:10756000237C0E94487C6093650C7093660C80932A
:10757000670C9093680C0E94487C6093690C709330
:107580006A0C80936B0C90936C0CCE014C960E940D
:10759000D31F6EE975E0CE0101960E94D775BE013A
:1075A000645E7F4FCE0101960E945374BC01CE01F0
:1075B00082960E94CE75CE0182960E946518CE01F9
:1075C00082960E943875CE0101960E943875CE01D0
:1075D0004C960E94387573CD4BE050E06AEA7FE02C
:1075E000CE0101960E94D108BE016F5F7F4F8CE8EB
:1075F0009FE00E94FF74CE0101960E9438758CE8CE
:107600009FE00E94897360587F488F4F9F4FA7CF9C
:1076100064E077E0CE0101960E94D775BE016F5FEE
:107620007F4FCE01C4960E942274182FCE0101967E
:107630000E943875112309F46CC045E050E06AEAF5
:107640007FE0CE0101960E94D108BE016F5F7F4F9F
:107650008CE89FE00E94FF74CE0101960E9438756D
:107660000E94487C6093650C7093660C8093670C55
:107670009093680C8CE89FE00E9489736093AC0241
:107680007093AD028093AE029093AF0260932D1180
:1076900070932E1180932F119093301120912C1103
:1076A0002093750C672B682B692B11F41092750CC5
:1076B00084EF91E090939B0280939A026DE270E1D7
:1076C0000E94900864E670E080E090E00E94AB7950
:1076D00061E17AE0CE0101960E94C575CE01019666
:1076E0000E947C18CE0101960E9438754091AC0230
:1076F0005091AD026091AE027091AF02CE01019641
:107700000E945173CE0101960E946518CE01019628
:1077100060CF6FEA75E0CE0101960E94D775BE0179
:107720006F5F7F4FCE01C4960E942274182FCE0146
:1077300001960E9438751123D9F14AE050E06AEAB7
:107740007FE0CE0101960E94D108BE016F5F7F4F9E
:107750008CE89FE00E94FF74CE0101960E9438756C
:107760008CE89FE00E948973613071058105910565
:1077700019F481E080932C118CE89FE00E948973BA
:10778000672B682B692B11F410922C1180912C110E
:107790008093750C882309F4B0CD0E94487C6093D7
:1077A000650C7093660C8093670C9093680CA5CD64
:1077B0006AEB75E0CE0101960E94D775BE016F5F3E
:1077C0007F4FCE01C4960E942274182FCE010196DD
:1077D0000E9438751123A1F048E050E06AEA7FE08A
:1077E000CE0101960E94D108BE016F5F7F4F8CE8E9
:1077F0009FE00E94FF74CE0101960E9438758DCDE6
:1078000063EC75E0CE0101960E94D775BE016F5FF3
:107810007F4FCE01C4960E942274182FCE0101968C
:107820000E943875112321F145E050E06AEA7FE0BB
:10783000CE0101960E94D108BE016F5F7F4F8CE898
:107840009FE00E94FF74CE0101960E9438758CE87B
:107850009FE00E9489736130710521F481E080937B
:10786000760C2DCC672B09F02ACC1092760C27CC05
:1078700069EC75E0CE0101960E94D775BE016F5F7D
:107880007F4FCE01C4960E942274182FCE0101961C
:107890000E943875112309F472C066E070E08AEA2C
:1078A0009FE00E94F173682FCE0101960E94A3759C
:1078B000BE016F5F7F4F8CE89FE00E94FF74CE0196
:1078C00001960E9438758CE89FE00E94947360E0F6
:1078D0008CE89FE00E9490748CE89FE00E9489737E
:1078E0006B01CB01181619060CF0E9CB2091A80208
:1078F0003091A902261737070CF4E1CB48E050E09D
:107900006AEA7FE0CE0101960E94D108BE016F5F56
:107910007F4F8CE89FE00E94FF74CE0101960E9489
:1079200038758CE89FE00E9494738091900F90913D
:10793000910F0997A8F028E030E050E040E06CE8B3
:107940007FE0CE0101960E94EC75BE016F5F7F4F14
:107950008CE89FE00E94FF74CE0101960E9438756A
:10796000B601E3E0660F771FEA95E1F76F5B7F4EA4
:1079700048E050E08CE89FE00E949B7290CB63E26D
:1079800074E0CE014C960E94D775BE01645E7F4FB5
:10799000CE01C4960E94227411E0811115C060EDE1
:1079A00075E0CE0101960E94D775BE016F5F7F4FD3
:1079B000CE01C4960E94227411E0811101C010E032
:1079C000CE0101960E943875CE014C960E94387502
:1079D000112309F4D3C16CED75E0CE014C960E94E1
:1079E000D77567ED75E0CE0101960E94D775AE019F
:1079F000445E5F4FBE016F5F7F4FCE01C4960E9411
:107A0000809FCE0101960E943875CE014C960E944F
:107A100038756CED75E0CE014C960E94D77569ED16
:107A200075E0CE0101960E94D775AE01445E5F4FAE
:107A3000BE016F5F7F4FCE01C4960E94809FCE0132
:107A400001960E943875CE014C960E9438756CEDF7
:107A500075E0CE014C960E94D7756BED75E0CE01B6
:107A600001960E94D775AE01445E5F4FBE016F5F05
:107A70007F4FCE01C4960E94809FCE0101960E9446
:107A80003875CE014C960E9438756FED75E0CE01C9
:107A90004C960E94D7756EED75E0CE0101960E945E
:107AA000D775AE01445E5F4FBE016F5F7F4FCE0161
:107AB000C4960E94809FCE0101960E943875CE0127
:107AC0004C960E9438756FED75E0CE014C960E9481
:107AD000D77560E378E0CE0101960E94D775AE01BC
:107AE000445E5F4FBE016F5F7F4FCE01C4960E9420
:107AF000809FCE0101960E943875CE014C960E945F
:107B00003875CE01C4960E9494730E94487C60939D
:107B10004A0C70934B0C80934C0C90934D0C36E0B8
:107B2000E32EF12C44E6442E512C612C712C882438
:107B30008394912C5701F3E0AF0EB11C88AD99AD41
:107B40000197A816B90608F0BACAB701CE01C496C3
:107B50000E94F173682FCE014C960E94A3756701B5
:107B600082E0C80ED11C9FEFE91AF90A9601A7011D
:107B7000BE016C5C7F4FCE0101960E94EC75CE0178
:107B800001960E9489738B01CE0101960E9438757F
:107B90000130110521F40091471110914811033073
:107BA000110521F40091491110914A116CED75E015
:107BB000CE0101960E94D775A601BE016F5F7F4F6F
:107BC000CE01C4960E9479A06C01CE0101960E945C
:107BD000387563ED78E0CE0101960E94D7751C14CC
:107BE0001D0424F59601A501BE016C5C7F4FCE01FA
:107BF00082960E94EC75BE016E5D7F4FCE010196AC
:107C00000E94FF74CE0182960E94387510161106EC
:107C10001CF17601EFEFEE1AFE0ACE0101960E94EA
:107C20003875CE014C960E94387584CFA501BE01EF
:107C30006C5C7F4FCE0182960E94D108BE016E5DC2
:107C40007F4FCE0101960E94FF74CE0182960E9462
:107C50003875101611060CF78091A8029091A902B0
:107C6000801791070CF445C070E060E0CE014C969F
:107C70000E94F173823509F041C0CE0101960E9445
:107C80008973672B682B692B39F4F801EE0FFF1FFE
:107C9000EE55FD4F11821082CE0101960E9489732C
:107CA000613071058105910521F5F801EE0FFF1F87
:107CB000EE55FD4F91828082000F111F000F111FA2
:107CC000F801E55AFD4F80819181A281B381181698
:107CD00019061A061B0624F04082518262827382C2
:107CE0000E94487C015B1D4FF80160837183828391
:107CF00093831C141D040CF48CCF8FCF8634F1F4C5
:107D0000CE0101960E948973672B682B692B39F489
:107D1000F801EE0FFF1FE75BFD4F11821082CE01CD
:107D200001960E948973613071058105910521F6E4
:107D3000F801EE0FFF1FE75BFD4FBCCF843481F4E9
:107D4000CE0101960E948973000F111F000F111FB1
:107D5000F801E95CFD4F6083718382839383C0CF18
:107D6000843539F6CE0101960E948973000F111FE8
:107D7000000F111FF801E55AFD4FEDCF6CE07AE0DE
:107D8000CE0101960E94C575BE016F5F7F4FCE0187
:107D9000C4960E942274082FCE0101960E94387565
:107DA000002309F413C144E050E06AEA7FE0CE0109
:107DB00001960E94D108BE016F5F7F4F8CE89FE063
:107DC0000E94FF74CE0101960E9438758CE89FE0F6
:107DD0000E94947360E08CE89FE00E949074409150
:107DE000900F5091910F6CE07CE08CE89FE00E9436
:107DF0009B726EED78E0CE018E960E94D7756CE88E
:107E00007FE0CE0188960E94CE758CA59DA5892B1A
:107E1000A9F063ED78E0CE0182960E94D7758AA919
:107E20009BA9892B09F05CC0CE0188960E948973BA
:107E30006AAFCE0182960E94387511E0CE01889615
:107E40000E943875CE018E960E943875112309F470
:107E500036C98E01065C1F4F59E5E52E50E1F52E1F
:107E60006E018EE3C80ED11CF80181918F01F701DC
:107E700081937F011D8E1C8E1F8E1E8E19A218A24B
:107E80004AE0BE016F5F7F4F90E00E944CA3BE01AD
:107E90006F5F7F4FCE014C960E941B73CE014C96B4
:107EA0000E946518CE014C960E943875C016D10606
:107EB000D9F684EF91E090939B0280939A026DE251
:107EC00070E10E94900864E670E080E090E00E941B
:107ED000AB7961E07AE0CE0101960E94C57512CCC3
:107EE00050E040E0BE01625D7F4FCE0188960E9467
:107EF00079A08C01892B11F40CA51DA563ED78E008
:107F0000CE014C960E94D7754E01FAE38F0E911C5C
:107F10005401F12CE12C6501C818D908101611067E
:107F200084F59801A701BE01685D7F4FCE010196DF
:107F30000E94EC75BE016F5F7F4FCE014C960E9490
:107F4000FF74CE0101960E943875CE014C960E94B6
:107F50008973F50161935F017801FFEFEF1AFF0A62
:107F6000A701BE01625D7F4FCE0188960E9479A075
:107F70008C018CA59DA5E816F90668F210E000E0DA
:107F8000CACF8CA59DA5E816F906D8F4A701BE01B5
:107F9000685D7F4FCE0101960E94D108BE016F5FE0
:107FA0007F4FCE014C960E94FF74CE0101960E9435
:107FB0003875CE014C960E948973FE01EC0DFD1DB3
:107FC00062AFCE014C960E94387533CF6AEF79E0EC
:107FD000CE0101960E94C575BE016F5F7F4FCE0135
:107FE000C4960E942274182FCE0101960E94387503
:107FF0001123E9F146E050E06AEA7FE0CE01019604
:108000000E94D108BE016F5F7F4F8CE89FE00E9405
:10801000FF74CE0101960E9438758CE89FE00E94A3
:1080200094738091900F9091910F892B09F447C818
:108030008CE89FE00E9489737093561160935511EC
:10804000709336026093350284EF91E090939B0227
:1080500080939A026DE270E10E94900864E670E0FD
:1080600080E090E00E94AB7966EE79E034CF61EE7B
:1080700075E0CE0101960E94D775BE016F5F7F4FFC
:10808000CE01C4960E942274182FCE0101960E9440
:1080900038751123A1F069ED79E0CE0101960E94B7
:1080A000C57564E670E0CE0101960E94F07FCE01B6
:1080B00001960E943875F0E0E0E0199500C868EE7E
:1080C00075E0CE014C960E94D775BE01645E7F4F6D
:1080D0008AEA9FE00E94227411E0811115C060EFCE
:1080E00075E0CE0101960E94D775BE016F5F7F4F8C
:1080F0008AEA9FE00E94227411E0811101C010E021
:10810000CE0101960E943875CE014C960E943875BA
:10811000112389F168EF75E0CE0101960E94D775B1
:108120006BE671E1CE0101960E945374BC0182E9B5
:108130009FE00E94E874CE0101960E9438756CE8B9
:1081400077E0CE0101960E94D77562E97FE0CE010B
:1081500001960E945374BC01CE014C960E94CE75CC
:10816000CE014C960E946518CE014C960E9438753F
:10817000CE0101966BC562E076E0CE014C960E947E
:10818000D775BE01645E7F4F8AEA9FE00E94227429
:1081900011E0811115C069E076E0CE0101960E94E0
:1081A000D775BE016F5F7F4F8AEA9FE00E942274FD
:1081B00011E0811101C010E0CE0101960E943875D6
:1081C000CE014C960E943875112369F06BEC79E072
:1081D00082E99FE00E94C37461E771E182E99FE058
:1081E0000E94BC74ACCF60E176E0CE0101960E94A3
:1081F000D775BE016F5F7F4FCE01C4960E94227477
:10820000182FCE0101960E943875112331F00E947B
:108210000429109234020C945F3869E176E0CE01B3
:108220004C960E94D775BE01645E7F4F8AEA9FE03C
:108230000E94227411E0811115C06EE176E0CE013A
:1082400001960E94D775BE016F5F7F4F8AEA9FE05B
:108250000E94227411E0811101C010E0CE0101964C
:108260000E943875CE014C960E943875112309F48E
:1082700041C06FED75E0CE0101960E94D775409127
:10828000AE0F5091AF0F8D819E81481B590BBE01DF
:108290006F5F7F4F8AEA9FE00E94329FAC014F5F81
:1082A0005F4F6AEA7FE0CE014C960E94D108BE0182
:1082B000645E7F4F8CE89FE00E94FF74CE014C9675
:1082C0000E943875CE0101960E9438758CE89FE0B7
:1082D0000E9489736115710531F481E08093DE029B
:1082E0000E944D9496CF6130710509F092CF1092A3
:1082F000DE02F6CF63E276E0CE0101960E94D775EA
:10830000BE016F5F7F4FCE01C4960E942274182F6A
:10831000CE0101960E943875112309F43AC143E059
:1083200050E06AEA7FE0CE0101960E94D108BE01CA
:108330006F5F7F4F8CE89FE00E94FF74CE01019633
:108340000E9438756CE87FE0CE0101960E94CE75E0
:10835000CE0101960E94691DCE0101960E943875DA
:1083600084EF91E090939B0280939A026CE87FE007
:10837000CE0101960E94CE7560E0CE0101960E946A
:10838000A474BC0187E791E10E94E874CE010196D4
:108390000E9438756CE87FE0CE0101960E94CE7590
:1083A00060E0CE0101960E94A474BC0181E791E1D6
:1083B0000E94E874CE0101960E94387540917B11AD
:1083C00050917C116DEE70E187E791E10E949B7204
:1083D000409175115091761168EF70E181E791E15C
:1083E0000E949B726DE270E180919A0290919B02D3
:1083F0000E94900867E276E0CE0101960E94D77550
:108400006CE87FE0CE0101960E945374BC01CE015E
:1084100082960E94CE75CE0101960E943875809199
:10842000E9109091EA10892B39F4BE016E5D7F4FFF
:108430008CEB9CE00E94267768EB7BE080E090E08C
:108440000E94AB798091E9109091EA10029709F0AF
:1084500087C06CE87FE0CE0188960E94CE756FE2FF
:1084600076E0CE0101960E94D775CE0101960E945A
:108470007994CE0101960E94387564EF71E080E036
:1084800090E00E94AB7962E376E0CE0101960E9413
:10849000D775CE0101960E947994CE0101960E9473
:1084A00038756CED75E080E090E00E94AB796BE38D
:1084B00076E0CE0101960E94D775CE0101960E940A
:1084C0007994CE0101960E94387564EF71E080E0E6
:1084D00090E00E94AB7969E476E0CE0101960E94BB
:1084E000D775CE0101960E947994CE0101960E9423
:1084F000387564EF71E080E090E00E94AB7967E24C
:1085000076E0CE0101960E94D775BE01685D7F4F6F
:10851000CE0101960E945374BC01CE014C960E947C
:10852000CE75CE0101960E943875CE014C960E9400
:108530009473BE01645E7F4FCE0101960E94CE759A
:10854000CE0101960E947994CE0101960E94387561
:10855000CE014C960E943875CE0188960E943875DF
:1085600068EB7BE080E090E00E94AB796DEE70E11B
:10857000CE0101960E94D775CE0101960E94691D19
:10858000CE0101960E94387510923402CE01829677
:1085900020C867E576E0CE0101960E94D775BE013E
:1085A0006F5F7F4FCE01C4960E942274182FCE01B8
:1085B00001960E943875112309F486C044E050E00A
:1085C0006AEA7FE0CE0101960E94D108BE016F5F8A
:1085D0007F4F8CE89FE00E94FF74CE0101960E94BD
:1085E00038756CE576E0CE0101960E94D7756CE88F
:1085F0007FE0CE0101960E945374BC01CE014C96DF
:108600000E94CE75CE0101960E9438758091E910C6
:108610009091EA10892B39F4BE01645E7F4F8CEB98
:108620009CE00E94267768E873E180E090E00E9479
:10863000AB798091E9109091EA10029759F563E6C1
:1086400076E0CE0101960E94D7758091900F9091AF
:10865000910F892B19F56CE676E0CE0101960E9408
:108660001B73BE01645E7F4FCE0182960E94CE7561
:10867000CE0182960E947994CE0182960E9438752E
:1086800068E873E180E090E00E94AB79CE0101964A
:108690000E943875109234020C94E73ABE016F5F65
:1086A0007F4FCE0182960E94CE75CE0182960E94A7
:1086B0007994CE0182960E94387560E777E180E078
:1086C00090E00E94AB79CDCF65E776E0CE010196D0
:1086D0000E94D775BE016F5F7F4FCE01C4960E9486
:1086E0002274182FCE0101960E943875112309F4C7
:1086F00062C06AEA7FE08CE89FE00E94E87481E053
:10870000809334026AEA7FE0CE0101960E94CE7522
:10871000CE0101960E94691DCE0101960E94387516
:108720008091E9109091EA10029709F16CE87FE0DE
:108730008CEB9CE00E94267768EB7BE080E090E089
:108740000E94AB79CE0101960E941295BE016F5F27
:108750007F4F8AEA9FE00E94FF74CE0101960E943B
:10876000387560ED77E080E090E00E94AB79809111
:10877000E9109091EA10029771F46CE87FE0CE0165
:1087800001960E94CE75CE0101960E947994CE0189
:1087900001960E9438758091AE0F9091AF0F892B92
:1087A00009F437CD6CE877E0CE0101960E94D775C9
:1087B0006AEA7FE0CCCC69E776E0CE0101960E94C0
:1087C000D775BE016F5F7F4FCE01C4960E942274A1
:1087D000182FCE0101960E943875112309F492C119
:1087E0008091E9109091EA10019709F012CD6FE79E
:1087F00076E0CE0188960E94D775BE01685D7F4FF6
:108800008CEB9CE00E9426776CE271E080E090E0C7
:108810000E94AB79CE0182960E94129564E670E0C8
:1088200080E090E00E94AB7910E000E035E0C32EDC
:10883000D12C4AE0A42EB12C6AE876E0CE01019654
:108840000E94D77550E040E0BE016F5F7F4FCE01C0
:1088500082960E9479A07C01CE0101960E94387513
:10886000A7014F5F5F4FBE016E5D7F4FCE01019646
:108870000E94D108BE016F5F7F4FCE0188960E9493
:10888000FF74CE0101960E9438758CA59DA5892B99
:1088900009F170E060E0CE0188960E94F173082E25
:1088A000000C990BC0970A97A8F46CE876E0CE010B
:1088B00001960E94D775BE016F5F7F4FCE018896EB
:1088C0000E942274E82ECE0101960E943875FF2482
:1088D000F394E110F12C6AE678E0CE0101960E9453
:1088E000C57564E170E0CE0101960E9495A0CE01AD
:1088F00001960E9438750F5F1F4F62E370E080E0C1
:1089000090E00E94AB79C801B6010E9418AA0197B5
:10891000C1F4CE0101960E94951D8D819E81892B07
:1089200009F4BBC0BE016F5F7F4F8AEA9FE00E94DF
:10893000E8740E944837FF24F394CE0101960E9408
:108940003875CE0101960E941295BE016F5F7F4F70
:10895000CE0182960E94FF74CE0101960E94387566
:1089600062E370E080E090E00E94AB79043611058C
:1089700019F0FF2009F460CF8091D90B8823F1F022
:108980006CE877E0CE014C960E94D775BE01685D19
:108990007F4FCE014C960E945374BC01CE010196CC
:1089A0000E94CE75CE0101960E946518CE010196F7
:1089B0000E943875CE014C960E9438758CA59DA5F5
:1089C000892B69F070E060E0CE0188960E94F17317
:1089D000082E000C990BC0970A9708F477C064E939
:1089E00076E0CE0101960E94D775CE0182960E9454
:1089F0003875CE0188960E9438758D819E810097CA
:108A000009F446C0E981FA812081222309F440C09B
:108A10000797F0F162EC79E0CE014C960E94C575A3
:108A200068EC70E0CE014C960E9495A0CE014C9669
:108A30000E943875BE016F5F7F4FCE014C960E9439
:108A4000CE7560ED77E0CE014C960E94F07FCE01AE
:108A50004C960E94387560EA76E0CE014C960E94F2
:108A6000D7756AEA7FE0CE014C960E945374BC0130
:108A7000CE0182960E94CE75CE0182960E94651824
:108A8000CE0182960E943875CE014C960E943875B0
:108A9000CE0101960E943875BCCB043111050CF44F
:108AA0004CCFC801B5010E9418AA892B09F045CF07
:108AB000BE01685D7F4F8CEB9CE00E94267768ECDE
:108AC00070E080E090E00E94AB7937CF6CE876E010
:108AD000CE0101960E94D775BE016F5F7F4FCE0118
:108AE00088960E942274182FCE0101960E94387534
:108AF000111175CFBE01685D7F4FCE0101960E94B6
:108B0000BC7573CF6EEA76E0CE0101960E94D775F0
:108B1000BE016F5F7F4FCE01C4960E942274182F52
:108B2000CE0101960E943875112309F4E8C025E0B2
:108B300030E044E050E06AEA7FE0CE0101960E9416
:108B4000EC75BE016F5F7F4F8CE89FE00E94FF7461
:108B5000CE0101960E9438756AEA7FE0CE01019647
:108B60000E94CE75CE0101960E94691DCE0101962C
:108B70000E9438758CE89FE00E948973613071050E
:108B800009F067C07093EA106093E91069E978E032
:108B9000CE0101960E94C575CE0101960E94691D05
:108BA000CE0101960E94387563EB76E0CE014C96BB
:108BB0000E94D77561E771E1CE014C960E94537413
:108BC000BC01CE0101960E94CE7548EC50E06FEFDB
:108BD0007FEFCE0101960E948C19CE0101960E9472
:108BE0003875CE014C960E9438750E94159F40E062
:108BF00052EC61E070E08CEB9CE00E94497184EFE4
:108C000091E090939B0280939A026DE270E10E9442
:108C1000900862EC76E0CE014C960E94D7756BE628
:108C200071E1CE014C960E945374BC01CE010196B5
:108C30000E94CE7560ED77E0CE0101960E94F07F34
:108C4000CE0101960E943875CE014C960E9438756F
:108C5000E0CA61157105D1F51092EA101092E91081
:108C60006BE878E0CE0101960E94C575CE010196B1
:108C70000E94691DCE0101960E94387569EB76E06D
:108C8000CE014C960E94D77561E771E1CE014C96FA
:108C90000E945374BC01CE0101960E94CE7548EC2F
:108CA00050E06FEF7FEFCE0101960E948C19CE014C
:108CB00001960E943875CE014C960E9438750E942C
:108CC000159F40E855E260E070E095CF6230710595
:108CD00009F09FCA7093EA106093E9106AE778E0A0
:108CE000CE0101960E94C575CE0101960E94691DB4
:108CF000CE0101960E9438756DEB76E0C1CF67EC2E
:108D000076E0CE0101960E94D775BE016F5F7F4F5E
:108D1000CE01C4960E942274182FCE0101960E94A3
:108D20003875112309F441C047E050E06AEA7FE05A
:108D3000CE0101960E94D108BE016F5F7F4F8CE883
:108D40009FE00E94FF74CE0101960E94387562E98F
:108D500076E0CE0101960E94D775BE016F5F7F4F0E
:108D60008CE89FE00E942274182FCE0101960E9489
:108D7000387511111092740C62EC74E0CE010196FA
:108D80000E94D775BE016F5F7F4F8CE89FE00E9405
:108D90002274182FCE0101960E943875112309F410
:108DA00001CD81E08093740CFDCC6FEC76E0CE01B8
:108DB00001960E94D775BE016F5F7F4FCE01C496AA
:108DC0000E942274182FCE0101960E94387511233B
:108DD00081F146E050E06AEA7FE0CE0101960E9410
:108DE000D108BE016F5F7F4F8CE89FE00E94FF7447
:108DF000CE0101960E9438758CE89FE00E947E7338
:108E00006093311170933211809333119093341128
:108E100084EF91E090939B0280939A026DE270E15F
:108E20000E94900864E670E080E090E00E94AB79D8
:108E3000B9CC66ED76E0CE0101960E94D775BE01F1
:108E40006F5F7F4FCE01C4960E942274182FCE010F
:108E500001960E943875112301F148E050E06AEA5A
:108E60007FE0CE0101960E94D108BE016F5F7F4F67
:108E70008CE89FE00E94FF74CE0101960E94387535
:108E80008CE89FE00E947E736093371170933811D5
:108E90008093391190933A11BBCF6FED76E0CE01FC
:108EA00001960E94D775BE016F5F7F4FCE01C496B9
:108EB0000E942274182FCE0101960E94387511234A
:108EC00001F149E050E06AEA7FE0CE0101960E949C
:108ED000D108BE016F5F7F4F8CE89FE00E94FF7456
:108EE000CE0101960E9438758CE89FE00E947E7347
:108EF00060933B1170933C1180933D1190933E1110
:108F000087CF69EE76E0CE0101960E94D775BE014B
:108F10006F5F7F4FCE01C4960E942274182FCE013E
:108F200001960E9438751123F1F049E050E06AEA99
:108F30007FE0CE0101960E94D108BE016F5F7F4F96
:108F40008CE89FE00E94FF74CE0101960E94387564
:108F50008CE89FE00E947E730E94CCA9709342111E
:108F60006093411155CF63EF76E0CE0101960E94E8
:108F7000D775BE016F5F7F4FCE01C4960E942274E9
:108F8000182FCE0101960E9438751123F1F04AE0A6
:108F900050E06AEA7FE0CE0101960E94D108BE014E
:108FA0006F5F7F4F8CE89FE00E94FF74CE010196B7
:108FB0000E9438758CE89FE00E947E730E94CCA9C5
:108FC0007093401160933F1123CF6EEF76E0CE0196
:108FD00001960E94D775BE016F5F7F4FCE01C49688
:108FE0000E942274182FCE0101960E943875112319
:108FF00011F14BE050E06AEA7FE0CE0101960E9459
:10900000D108BE016F5F7F4F8CE89FE00E94FF7424
:10901000CE0101960E9438758CE89FE00E947E7315
:109020000E94CCA960934311709344118093451121
:1090300090934611EDCE6AE077E0CE0101960E9452
:10904000D775BE016F5F7F4FCE01C4960E94227418
:10905000182FCE0101960E9438751123E1F045E0EA
:1090600050E06AEA7FE0CE0101960E94D108BE017D
:109070006F5F7F4F8CE89FE00E94FF74CE010196E6
:109080000E9438758CE89FE00E94897370933611B6
:1090900060933511BDCE60E177E0CE0101960E946C
:1090A000D775BE016F5F7F4FCE01C4960E942274B8
:1090B000182FCE0101960E943875112359F00E9495
:1090C000487C60934A0C70934B0C80934C0C9093AB
:1090D0004D0C9FC866E177E0CE0101960E94D775DE
:1090E000BE016F5F7F4FCE01C4960E942274182F7D
:1090F000CE0101960E943875112389F143E050E0BA
:10910000BE016C5C7F4FCE0101960E94D108BE016A
:109110006F5F7F4F8CE89FE00E94FF74CE01019645
:109120000E9438758091900F9091910F892B41F09A
:109130008CE89FE00E9489737093AB026093AA024F
:109140008091AA029091AB020197029708F42ACB72
:1091500081E090E09093AB028093AA0223CB67EF6B
:1091600076E0CE014C960E94D775BE01645E7F4FBB
:10917000CE01C4960E94227411E0811115C061E6EF
:1091800077E0CE0101960E94D775BE016F5F7F4FD9
:10919000CE01C4960E94227411E0811101C010E03A
:1091A000CE0101960E943875CE014C960E9438750A
:1091B000112309F468C067EF76E0CE0101960E94A2
:1091C000D775BE016F5F7F4FCE01C4960E94227497
:1091D000182FCE0101960E9438751123A1F046E0A8
:1091E00050E0BE016C5C7F4FCE0101960E94D10819
:1091F000BE016F5F7F4F8CE89FE00E94FF74CE013D
:1092000001960E94387561E677E0CE0101960E94D2
:10921000D775BE016F5F7F4FCE01C4960E94227446
:10922000182FCE0101960E9438751123A1F042E05B
:1092300050E0BE016C5C7F4FCE0101960E94D108C8
:10924000BE016F5F7F4F8CE89FE00E94FF74CE01EC
:1092500001960E9438758091900F9091910F892B03
:1092600009F4A0CA6CE87FE0CE0101960E94CE7599
:1092700061E070E0CE0101960E94522ECE0101966F
:109280000E9438758FCA63E277E0CE0182960E9411
:10929000D775BE016E5D7F4FCE01C4960E942274C9
:1092A00011E0811129C06AE177E0CE014C960E945D
:1092B000D775BE01645E7F4FCE01C4960E942274B2
:1092C00011E0811115C062E277E0CE0101960E94A3
:1092D000D775BE016F5F7F4FCE01C4960E94227486
:1092E00011E0811101C010E0CE0101960E94387595
:1092F000CE014C960E943875CE0182960E94387538
:10930000112309F4E6C063E277E0CE0101960E94E2
:10931000D775BE016F5F7F4FCE01C4960E94227445
:10932000182FCE0101960E943875112309F466C0EA
:1093300046E050E0BE016C5C7F4FCE0101960E947A
:10934000D108BE016F5F7F4F8CE89FE00E94FF74E1
:10935000CE0101960E9438758CE89FE00E947E73D2
:109360006B017C0120E030E0A9010E9402AA1816DE
:109370000CF08EC0A701960160E070E08AE794E4EB
:109380000E945AA90E94CCA96093300270933102C6
:109390008093320290933302809130029091310297
:1093A000A0913202B0913302181619061A061B0654
:1093B00064F081E090E0A0E0B0E080933002909310
:1093C0003102A0933202B09333028091AA029091AD
:1093D000AB028130910509F068C080913002909114
:1093E0003102A0913202B091330280932C0290930B
:1093F0002D02A0932E02B0932F02D4C947E050E073
:10940000BE016C5C7F4FCE0101960E94D108BE0167
:109410006F5F7F4F8CE89FE00E94FF74CE01019642
:109420000E9438756AE674E0CE0101960E94D775F5
:10943000BE016F5F7F4FCE01C4960E942274182F29
:10944000CE0101960E943875112331F081E090E041
:109450009093AB028093AA0260E376E0CE0101967E
:109460000E94D775BE016F5F7F4FCE01C4960E94E8
:109470002274182FCE0101960E943875112309F429
:109480006BCF82E090E09093AB028093AA0264CF0E
:1094900081E090E0A0E0B0E0809330029093310250
:1094A000A0933202B093330277CF029709F07AC9C2
:1094B0008091300290913102A0913202B09133023A
:1094C0008093280290932902A0932A02B0932B0242
:1094D00069C96AE277E0CE014C960E94D775BE0159
:1094E000645E7F4FCE01C4960E94027411E0811128
:1094F00015C06FE277E0CE0101960E94D775BE01DC
:109500006F5F7F4FCE01C4960E94227411E08111DB
:1095100001C010E0CE0101960E943875CE014C9634
:109520000E943875112309F48CC26CEB77E0CE01F0
:1095300001960E94D775BE016F5F7F4FCE01C49622
:109540000E942274182FCE0101960E9438751123B3
:1095500009F4FBC001E010E01093AB020093AA02F3
:10956000109368020093670266E377E08CE89FE05F
:109570000E941B73109368020093670281E090E0E1
:10958000A0E0B0E08093300290933102A0933202C9
:10959000B093330280932C0290932D02A0932E025D
:1095A000B0932F026CE87FE0CE0101960E94CE7549
:1095B00062E070E0CE0101960E94522ECE0101962B
:1095C0000E94387561EB79E0CE0101960E94C57565
:1095D000CE0101960E946518CE0101960E94387551
:1095E00061EA79E0CE0101960E94C575CE0101962F
:1095F0000E94A01FCE0101960E94387562E976E0B4
:109600008CE89FE00E941B736CE87FE0CE0101961E
:109610000E94CE7563E070E0CE0101960E94522E4A
:10962000CE0101960E94387582E090E09093AB02E3
:109630008093AA0260E979E0CE0101960E94C57587
:10964000CE0101960E946518CE0101960E943875E0
:1096500064E879E0CE0101960E94C575CE010196BD
:109660000E94A01FCE0101960E94387566E377E044
:109670008CE89FE00E941B738091531190915411CC
:1096800097FF06C06AE377E08CE89FE00E941B73B7
:109690006CE87FE0CE0101960E94CE7562E070E03A
:1096A000CE0101960E94522ECE0101960E9438757D
:1096B00062E976E08CE89FE00E941B7382E090E014
:1096C0009093AB028093AA026CE87FE0CE010196F2
:1096D0000E94CE7563E070E0CE0101960E94522E8A
:1096E000CE0101960E94387584EF91E090939B0221
:1096F00080939A026DE270E10E94900864E670E047
:1097000080E090E00E94AB7981E090E09093AB0222
:109710008093AA021092A5021092A40282E090E027
:10972000A0E0B0E080935F0290936002A09361029A
:10973000B09362020E94487C60935302709354027B
:1097400080935502909356022DC86AE277E0CE01CD
:1097500001960E94D775BE016F5F7F4FCE01C49600
:109760000E942274182FCE0101960E9438751111A3
:1097700019C86AE674E0CE0101960E94D775BE0151
:109780006F5F7F4FCE01C4960E942274182FCE01C6
:1097900001960E943875112331F081E090E090939A
:1097A000AB028093AA0260E376E0CE0101960E94AC
:1097B000D775BE016F5F7F4FCE01C4960E942274A1
:1097C000182FCE0101960E943875112331F082E0E6
:1097D00090E09093AB028093AA0281E090E0A0E039
:1097E000B0E08093300290933102A0933202B093A4
:1097F00033028091AA029091AB028130910509F069
:1098000099C090936802809367026FE277E0CE017F
:1098100001960E94D775BE016F5F7F4FCE01C4963F
:109820000E942274182FCE0101960E9438751123D0
:1098300019F146E050E0BE016C5C7F4FCE014C96C2
:109840000E94D1086EE377E0CE0101960E94D775A1
:10985000BE01645E7F4FCE0101960E945374BC012D
:109860008CE89FE00E94E874CE0101960E94387552
:10987000CE014C960E943875809130029091310251
:10988000A0913202B091330280932C0290932D026A
:10989000A0932E02B0932F0266E377E08CE89FE05E
:1098A0000E941B736CE87FE0CE0101960E94CE758A
:1098B00062E070E0CE0101960E94522ECE01019628
:1098C0000E94387563E779E0CE0101960E94C57564
:1098D000CE0101960E946518CE0101960E9438754E
:1098E00081E090E0909368028093670262E976E0FD
:1098F0008CE89FE00E941B736CE87FE0CE0101962C
:109900000E94CE7563E070E0CE0101960E94522E57
:10991000CE0101960E94387563E679E0CE0101968A
:109920000E94C575CE0101960E94A01FCE0101962E
:109930000E9438758091AA029091AB02029711F0B3
:109940000C94D24366E377E08CE89FE00E941B739F
:10995000809153119091541197FF06C06AE377E00C
:109960008CE89FE00E941B7301E010E010936802F6
:10997000009367026CE87FE0CE0101960E94CE75ED
:1099800062E070E0CE0101960E94522ECE01019657
:109990000E94387562E976E08CE89FE00E941B73B4
:1099A00062E579E0CE0101960E94C575CE0101966F
:1099B0000E946518CE0101960E9438756CE87FE020
:1099C000CE0101960E94CE7563E070E0CE01019653
:1099D0000E94522ECE0101960E94387566E479E00D
:1099E000CE0101960E94C575CE0101960E94A01F6E
:1099F000CE0101960E9438758091531190915411B7
:109A000091958195910990935411809353111093DE
:109A100068020093670284EF91E090939B02809329
:109A20009A026DE270E10E94900864E670E080E0C6
:109A300090E00E94AB791093AB020093AA020C94C1
:109A4000D24360E477E0CE0188960E94D775BE01CC
:109A5000685D7F4FCE01C4960E94227401E081119F
:109A60003DC061E977E0CE0182960E94D775BE01C4
:109A70006E5D7F4FCE01C4960E94227401E0811179
:109A800029C060E977E0CE014C960E94D775BE01EF
:109A9000645E7F4FCE01C4960E94227401E0811162
:109AA00015C067E477E0CE0101960E94D775BE012C
:109AB0006F5F7F4FCE01C4960E94227401E0811136
:109AC00001C000E0CE0101960E943875CE014C968F
:109AD0000E943875CE0182960E943875CE01889614
:109AE0000E943875002309F41FC260E477E0CE01BC
:109AF00001960E94D775BE016F5F7F4FCE01C4965D
:109B00000E942274082FCE0101960E94387546E00B
:109B100050E0011117C061E977E0CE0101960E9483
:109B2000D775BE016F5F7F4FCE01C4960E9422742D
:109B3000082FCE0101960E943875002309F48BC0CE
:109B400042E050E0BE016C5C7F4FCE0101960E9466
:109B5000D108BE016F5F7F4F8CE89FE00E94FF74C9
:109B6000CE0101960E9438758091900F9091910FCF
:109B7000892B11F40C94D2436EE377E0CE014C961E
:109B80000E94D775BE01645E7F4F8CE89FE00E9403
:109B90002274811114C068E679E0CE0101960E941A
:109BA000D775BE016F5F7F4F8CE89FE00E942274E3
:109BB00011E0811110E0CE0101960E943875CE01AE
:109BC0004C960E943875C12CD12C7601112309F4D2
:109BD0006AC18CE89FE00E947E736B017C018091DA
:109BE000AA029091AB02019709F09FC08CE89FE018
:109BF0000E947E739B01AC016091080C7091090C6E
:109C000080910A0C90910B0C0E94EEA86093080CB6
:109C10007093090C80930A0C90930B0C8090080CA5
:109C20009090090CA0900A0CB0900B0C20E030E052
:109C300044EB53E4C501B4010E9402AA87FD86C02B
:109C400020E030E044EB53E4C501B4010E94EDA8EC
:109C50004B015C01EBCF43E050E0BE016C5C7F4FF9
:109C6000CE0101960E94D108BE016F5F7F4F8CE844
:109C70009FE00E94FF74CE0101960E9438756AE64B
:109C800074E0CE0101960E94D775BE016F5F7F4FD1
:109C9000CE01C4960E942274082FCE0101960E9424
:109CA00038750023B1F081E090E09093AB0280938F
:109CB000AA0280915D0C90915E0CA0915F0CB09116
:109CC000600C8093080C9093090CA0930A0CB0933D
:109CD0000B0C60E376E0CE0101960E94D775BE01C1
:109CE0006F5F7F4FCE01C4960E942274082FCE0171
:109CF00001960E943875002309F436CF82E090E087
:109D00009093AB028093AA028091590C90915A0CC7
:109D1000A0915B0CB0915C0C8093080C9093090CA3
:109D2000A0930A0CB0930B0C1FCF8CE89FE00E940D
:109D30007E739B01AC016091080C7091090C8091BD
:109D40000A0C90910B0C0E94EDA860CF20E030E04F
:109D5000A901C501B4010E9440A787FF0BC020E004
:109D600030E044EB53E4C501B4010E94EEA84B017E
:109D70005C01ECCF8092080C9092090CA0920A0C26
:109D8000B0920B0C20E030E0A901C701B6010E949F
:109D900002AA87FD15C068E679E0CE0101960E940F
:109DA000D7756CE87FE0CE0101960E945374BC0128
:109DB0008CE89FE00E94E874CE0101960E943875FD
:109DC00020E030E0A901C701B6010E9440A787FF4B
:109DD0006AC08091AA029091AB02019799F520E0A8
:109DE00030E0A901C701B6010E9402AA18160CF0C2
:109DF00092C020E030E040E251E4C701B6010E9489
:109E0000EEA822E0AB01BC01CE014C960E94407549
:109E10006EE377E0CE0101960E94D775BE01645EC5
:109E20007F4FCE0101960E945374BC018CE89FE0E5
:109E30000E94E874CE0101960E943875CE014C96BE
:109E40000E9438758091AA029091AB02019759F156
:109E500020E030E0A901C701B6010E9402AAB701C3
:109E6000A60118160CF0705822E0CE014C960E9404
:109E700040756EE377E0CE0101960E94D775BE0172
:109E8000645E7F4FCE0101960E945374BC018CE842
:109E90009FE00E94E874CE0101960E943875CE01C1
:109EA0004C960E94387581E090E090936802809310
:109EB00067026CE87FE0CE0101960E94CE7562E0F9
:109EC00070E0CE0101960E94522ECE0101960E94B2
:109ED000387520E030E0A901C701B6010E9440A713
:109EE00087FD02C00C94D2438091AA029091AB02EC
:109EF000019711F00C94D2436BE477E08CE89FE07B
:109F00000E941B736CE87FE0CE0101960E94CE7523
:109F100062E070E0AFC9A701960160E070E080E206
:109F200091E40E94EDA86DCF60E577E0CE018296C6
:109F30000E94D775BE016E5D7F4FCE01C4960E9410
:109F4000227411E0811129C06FE477E0CE014C96B4
:109F50000E94D775BE01645E7F4FCE01C4960E94F9
:109F6000227411E0811115C066E577E0CE010196FB
:109F70000E94D775BE016F5F7F4FCE01C4960E94CD
:109F8000227411E0811101C010E0CE0101960E94FF
:109F90003875CE014C960E943875CE0182960E948B
:109FA0003875112309F49BC0CE01C4960E949473A6
:109FB00066E377E08CE89FE00E941B736AE674E03A
:109FC000CE0101960E94D775BE016F5F7F4FCE0113
:109FD000C4960E942274182FCE0101960E943875F3
:109FE000112331F081E090E09093AB028093AA02BC
:109FF00060E376E0CE0101960E94D775BE016F5FE7
:10A000007F4FCE01C4960E942274182FCE01019674
:10A010000E943875112391F082E090E09093AB029A
:10A020008093AA02809153119091541197FF06C01A
:10A030006AE377E08CE89FE00E941B7381E090E088
:10A0400090936802809367026CE87FE0CE010196EE
:10A050000E94CE7562E070E0CE0101960E94522E01
:10A06000CE0101960E94387560E577E0CE01019639
:10A070000E94D775BE016F5F7F4FCE01C4960E94CC
:10A080002274182FCE0101960E94387545E050E0E9
:10A09000111102C046E050E0BE016C5C7F4FCE0162
:10A0A00001960E94D108BE016F5F7F4F8CE89FE050
:10A0B0000E94FF74CE0101960E9438758091900F26
:10A0C0009091910F892B11F40C94D2436CE87FE0AE
:10A0D000CE0101960E94CE7563E070E0CBC86EE5BC
:10A0E00077E0CE0182960E94D775BE016E5D7F4FEC
:10A0F000CE01C4960E94227411E0811129C06DE541
:10A1000077E0CE014C960E94D775BE01645E7F4F0A
:10A11000CE01C4960E94227411E0811115C064E63C
:10A1200077E0CE0101960E94D775BE016F5F7F4F29
:10A13000CE01C4960E94227411E0811101C010E08A
:10A14000CE0101960E943875CE014C960E9438755A
:10A15000CE0182960E943875112309F426C16EE55E
:10A1600077E0CE0101960E94D775BE016F5F7F4FE9
:10A17000CE01C4960E942274182FCE0101960E942F
:10A180003875112309F443C045E050E0BE016C5C12
:10A190007F4FCE0101960E94D108BE016F5F7F4FB5
:10A1A0008CE89FE00E94FF74CE0101960E943875F2
:10A1B0008091900F9091910F892B61F08CE89FE036
:10A1C0000E947E736093080C7093090C80930A0CB4
:10A1D00090930B0CC090080CD090090CE0900A0CE6
:10A1E000F0900B0C20E030E044EB53E4C701B601E3
:10A1F0000E9402AA87FD55C020E030E044EB53E402
:10A20000C701B6010E94EDA86B017C01EBCF46E0CF
:10A2100050E0BE016C5C7F4FCE0101960E94D108D8
:10A22000BE016F5F7F4F8CE89FE00E94FF74CE01FC
:10A2300001960E9438756AE674E0CE0101960E948C
:10A24000D775BE016F5F7F4FCE01C4960E94227406
:10A25000182FCE0101960E943875112331F081E04C
:10A2600090E09093AB028093AA0260E376E0CE0187
:10A2700001960E94D775BE016F5F7F4FCE01C496D5
:10A280000E942274182FCE0101960E943875112366
:10A2900009F48ECF82E090E09093AB028093AA0203
:10A2A00087CF20E030E0A901C701B6010E9440A796
:10A2B00087FF0BC020E030E044EB53E4C701B60158
:10A2C0000E94EEA86B017C01ECCFC092080CD092EA
:10A2D000090CE0920A0CF0920B0C8091AA0290916A
:10A2E000AB02019771F4C0925D0CD0925E0CE092CB
:10A2F0005F0CF092600C62E075E082E99FE00E94E2
:10A300001B738091080C9091090CA0910A0CB091DC
:10A310000B0C2091AA023091AB022230310571F46E
:10A320008093590C90935A0CA0935B0CB0935C0CE7
:10A3300062E175E082E99FE00E941B734091080C86
:10A340005091090C60910A0C70910B0C21E0CE0128
:10A350004C960E94407562E97FE0CE0101960E9412
:10A36000CE75BE01645E7F4FCE0101960E9453748C
:10A370006DE075E00E943D74BC0182E99FE00E949F
:10A38000E874CE0101960E943875CE014C960E9469
:10A39000387562E97FE0CE0101960E94CE75CE014C
:10A3A00001960E94A01F0C943E496CE677E0CE0116
:10A3B00082960E94D775BE016E5D7F4FCE01C49616
:10A3C0000E94227411E0811129C06BE677E0CE0172
:10A3D0004C960E94D775BE01645E7F4FCE01C49635
:10A3E0000E94227411E0811115C061E777E0CE016F
:10A3F00001960E94D775BE016F5F7F4FCE01C49654
:10A400000E94227411E0811101C010E0CE0101967A
:10A410000E943875CE014C960E943875CE01829606
:10A420000E943875112309F412C2C0903002D090F6
:10A430003102E0903202F090330267E777E0CE011C
:10A4400001960E94D775BE016F5F7F4FCE01C49603
:10A450000E942274182FCE0101960E943875112394
:10A4600009F465C044E050E0BE016C5C7F4FCE0152
:10A4700001960E94D108BE016F5F7F4F8CE89FE07C
:10A480000E94FF74CE0101960E9438758091AA0245
:10A490009091AB028130910509F093C0C0902C02DD
:10A4A000D0902D02E0902E02F0902F0281E090E0FB
:10A4B000A0E0B0E080932C0290932D02A0932E0296
:10A4C000B0932F028091900F9091910F892B09F0FA
:10A4D00090C06CE777E08CE89FE00E941B7380914E
:10A4E000900F9091910F892B81F06CE87FE0CE0165
:10A4F00001960E94CE7570E060E0CE0101960E9448
:10A50000522ECE0101960E9438758091AA02909138
:10A51000AB028130910509F08CC1C0922C02D0921F
:10A520002D02E0922E02F0922F020C94D24345E0CD
:10A5300050E0BE016C5C7F4FCE0101960E94D108B5
:10A54000BE016F5F7F4F8CE89FE00E94FF74CE01D9
:10A5500001960E9438756AE674E0CE0101960E9469
:10A56000D775BE016F5F7F4FCE01C4960E942274E3
:10A57000182FCE0101960E943875112331F081E029
:10A5800090E09093AB028093AA0260E376E0CE0164
:10A5900001960E94D775BE016F5F7F4FCE01C496B2
:10A5A0000E942274182FCE0101960E943875112343
:10A5B00009F46CCF82E090E09093AB028093AA0202
:10A5C00065CF029709F07ECFC0902802D090290273
:10A5D000E0902A02F0902B0281E090E0A0E0B0E051
:10A5E0008093280290932902A0932A02B0932B0211
:10A5F00069CF62E877E0CE0101960E94D775BE016F
:10A600006F5F7F4F8CE89FE00E940274182FCE018D
:10A6100001960E943875112309F477CF8CE89FE0EA
:10A620000E947E7320E030E0A9010E9440A78111C2
:10A6300028C08091AA029091AB02019731F465E89D
:10A6400077E08CE89FE00E941B738091AA029091B2
:10A65000AB02029731F46CE777E08CE89FE00E9450
:10A660001B738091900F9091910F892B09F44DCF1E
:10A670006CE87FE0CE0101960E94CE7561E070E04B
:10A680003CCF6FED75E0CE0101960E94D775BE01FB
:10A690006F5F7F4F8CE89FE00E940274182FCE01FD
:10A6A00001960E943875112309F42FCF41E050E044
:10A6B0006CE87FE0CE0101960E94D108CE010196A0
:10A6C0000E947E734B015C01CE0101960E94387599
:10A6D00020E030E0A901C501B4010E9440A718168E
:10A6E00034F0812C912C20E8A22E2FE3B22E009181
:10A6F000AA021091AB020130110509F075C0A50145
:10A70000940160E070E48CE995E40E945AA960939A
:10A71000240270932502809326029093270260936F
:10A720004B1170934C1180934D1190934E11609387
:10A730002002709321028093220290932302B80199
:10A74000CE014C960E9425736AE877E0CE0101960F
:10A750000E94D775BE01645E7F4FCE0101960E94B4
:10A760005374BC01CE0182960E94CE75CE018296B2
:10A770000E947C18CE0182960E943875CE01019607
:10A780000E943875CE014C960E94387564E379E0DA
:10A79000CE0101960E94C575CE0101960E947C18DB
:10A7A000CE0101960E9438754091240250912502F5
:10A7B000609126027091270225E0CE0101960E9449
:10A7C0004075CE0101960E946518CE0101960E9447
:10A7D000387584EF91E090939B0280939A026DE22A
:10A7E00070E10E94900891CE0230110509F0A7CFC8
:10A7F000A501940160E070E48CE196E40E945AA9FE
:10A80000609324027093250280932602909327027E
:10A8100060934F1170935011809351119093521186
:10A8200060931C0270931D0280931E0290931F027E
:10A8300086CF029711F00C94D243C0922802D09296
:10A840002902E0922A02F0922B020C94D2436FE884
:10A8500077E0CE0182960E94D775BE016E5D7F4F74
:10A86000CE01C4960E94227411E0811129C06EE8C5
:10A8700077E0CE014C960E94D775BE01645E7F4F93
:10A88000CE01C4960E94227411E0811115C064E9C2
:10A8900077E0CE0101960E94D775BE016F5F7F4FB2
:10A8A000CE01C4960E94227411E0811101C010E013
:10A8B000CE0101960E943875CE014C960E943875E3
:10A8C000CE0182960E943875112309F429C188AD02
:10A8D00099AD059710F40C94D24344E050E0BE01CA
:10A8E0006C5C7F4FCE0101960E94D108BE016F5F64
:10A8F0007F4F8CE89FE00E94FF74CE0101960E947A
:10A9000038756FE877E0CE0101960E94D775BE01D9
:10A910006F5F7F4FCE01C4960E942274182FCE0124
:10A9200001960E943875112309F49BC044E050E061
:10A93000BE016C5C7F4FCE0101960E94D108BE0122
:10A940006F5F7F4F8CE89FE00E94FF74CE010196FD
:10A950000E9438758CE89FE00E947E7320E030E012
:10A96000A9010E9402AA181614F00C94D2438CE894
:10A970009FE00E947E73609324027093250280936F
:10A980002602909327022091AA023091AB02213037
:10A99000310509F0B0C060934B1170934C11809356
:10A9A0004D1190934E116093200270932102809379
:10A9B000220290932302B901CE014C960E94257386
:10A9C0006AE877E0CE0101960E94D775BE01645E09
:10A9D0007F4FCE0101960E945374BC01CE01829636
:10A9E0000E94CE75CE0182960E947C18CE0182967E
:10A9F0000E943875CE0101960E943875CE014C96A2
:10AA00000E94387562E279E0CE0101960E94C57518
:10AA1000CE0101960E947C18CE0101960E943875E5
:10AA200040912402509125026091260270912702E4
:10AA300025E0CE0101960E944075CE0101960E944C
:10AA40006518CE0101960E94387584EF91E09093CD
:10AA50009B0280939A026DE270E10E9490080C9430
:10AA6000D24345E050E0BE016C5C7F4FCE010196C1
:10AA70000E94D108BE016F5F7F4F8CE89FE00E946B
:10AA8000FF74CE0101960E9438756AE674E0CE012B
:10AA900001960E94D775BE016F5F7F4FCE01C496AD
:10AAA0000E942274182FCE0101960E94387511233E
:10AAB00031F081E090E09093AB028093AA0260E3D2
:10AAC00076E0CE0101960E94D775BE016F5F7F4F81
:10AAD000CE01C4960E942274182FCE0101960E94C6
:10AAE0003875112309F436CF82E090E09093AB02E1
:10AAF0008093AA022FCF2230310509F05CCF6093FA
:10AB00004F11709350118093511190935211609393
:10AB10001C0270931D0280931E0290931F024BCF64
:10AB200065E775E0CE014C960E94D775BE01645E64
:10AB30007F4FCE01C4960E94227411E0811115C08E
:10AB40006AE977E0CE0101960E94D775BE016F5F7A
:10AB50007F4FCE01C4960E94227411E0811101C082
:10AB600010E0CE0101960E943875CE014C960E94ED
:10AB70003875112309F463C065E775E0CE010196CD
:10AB80000E94D775BE016F5F7F4FCE01C4960E94B1
:10AB90002274182FCE0101960E943875112399F066
:10ABA00042E050E06AEA7FE0CE0101960E94D108BF
:10ABB000BE016F5F7F4F8CE89FE00E94FF74CE0163
:10ABC00001960E9438756AE977E0CE0101960E94ED
:10ABD000D775BE016F5F7F4FCE01C4960E9422746D
:10ABE000182FCE0101960E943875112399F043E089
:10ABF00050E06AEA7FE0CE0101960E94D108BE01D2
:10AC00006F5F7F4F8CE89FE00E94FF74CE0101963A
:10AC10000E9438758CE89FE00E948973653B71053E
:10AC200010F40C94D2436FE079E0CE0101960E94BB
:10AC3000C575CE0101960E947C180C943E496EE9C0
:10AC400077E0CE0101960E94D775BE016F5F7F4FFE
:10AC5000CE01C4960E942274182FCE0101960E9444
:10AC60003875112309F47EC026E030E044E050E05E
:10AC70006AEA7FE0CE0101960E94EC75BE016F5F2B
:10AC80007F4F8CE89FE00E94FF74CE0101960E94E6
:10AC900038756FED75E0CE0101960E94D775409131
:10ACA000AE0F5091AF0F8D819E81481B590BBE0195
:10ACB0006F5F7F4F8AEA9FE00E94329FAC014F5F37
:10ACC0005F4F6AEA7FE0CE014C960E94D108BE0138
:10ACD000645E7F4F8CE89FE00E94FF74CE014C962B
:10ACE0000E943875CE0101960E9438758CE89FE06D
:10ACF0000E947E7388E2E0EEFBE0A4E0B1E1019007
:10AD00000D928A95E1F784EF91E090939B028093F6
:10AD10009A026DE270E10E9490086EEE78E082E99E
:10AD20009FE00E94C37444E050E06AEA7FE0CE01F5
:10AD300001960E94D108BE016F5F7F4F82E99FE0BC
:10AD40000E94BC74CE0101960E94387562E97FE0D2
:10AD5000CE0101960E94CE75CE0101960E94651823
:10AD60000C94484562EA77E0CE0101960E94D775BF
:10AD7000BE016F5F7F4FCE01C4960E942274182FD0
:10AD8000CE0101960E94387511110C9494466AEA1E
:10AD900077E0CE0101960E94D775BE016F5F7F4FAD
:10ADA000CE01C4960E942274182FCE0101960E94F3
:10ADB0003875112371F141E066EB72E0CE01019626
:10ADC0000E94B68FBE016F5F7F4F89E891E10E94BC
:10ADD000931889E891E10E94638F811104C062EAAF
:10ADE00078E00C946B3F89E891E10E945A70892BBE
:10ADF00051F089E891E10E942989682F89E59DE059
:10AE00000E94836EF0CF89E891E10E946F8F0C94CD
:10AE10005F3861EB77E0CE0101960E94D775BE01E5
:10AE20006F5F7F4FCE01C4960E942274182FCE010F
:10AE300001960E9438751123E9F08DB79EB78A52AA
:10AE400091400FB6F8949EBF0FBE8DBFADB7BEB791
:10AE500011968AE291E0EDE2F0E101900D92019706
:10AE6000E1F70E94282B0FB6F894DEBF0FBECDBFCE
:10AE70000C945F386AEB77E0CE0101960E94D7759B
:10AE8000BE016F5F7F4FCE01C4960E942274182FBF
:10AE9000CE0101960E943875112309F459C08DB76F
:10AEA0009EB78A5291400FB6F8949EBF0FBE8DBFD9
:10AEB000ADB7BEB711968AE291E0EDE2F0E1019004
:10AEC0000D920197E1F70E94CE230FB6F894DEBFF2
:10AED0000FBECDBF6DED78E0CE0101960E94C57525
:10AEE0008DB79EB78A5291400FB6F8949EBF0FBEA1
:10AEF0008DBFADB7BEB711968AE291E0EDE2F0E109
:10AF000001900D920197E1F70E944C1B0FB6F89447
:10AF1000DEBF0FBECDBF8DB79EB78A5291400FB630
:10AF2000F8949EBF0FBE8DBFADB7BEB711968AE233
:10AF300091E0EDE2F0E101900D920197E1F70E94BE
:10AF4000282B0FB6F894DEBF0FBECDBF0C94863B06
:10AF50006CEB77E0CE0101960E94D775BE016F5F62
:10AF60007F4FCE01C4960E942274182FCE01019605
:10AF70000E9438751123B1F06BEC78E0CE01019698
:10AF80000E94C575BE016F5F7F4FCE014C960E9437
:10AF9000CE75CE014C960E946518CE014C960E944B
:10AFA0003875B9CF60EC77E0CE0101960E94D77575
:10AFB000BE016F5F7F4FCE01C4960E942274182F8E
:10AFC000CE0101960E943875112309F4F5C06FEA8D
:10AFD00078E0CE0182960E94C575BE016E5D7F4FFE
:10AFE000CE0101960E94CE75AE014F5F5F4F62E0C9
:10AFF00070E086E792E00E947125182FCE0101963D
:10B000000E943875111122C0BE016E5D7F4FCE01C6
:10B010004C960E94CE7564EC77E0CE014C960E946F
:10B020003D746DED7FE00E945374BC01CE0101962A
:10B030000E94CE75CE0101960E946518CE01019640
:10B040000E943875CE014C960E94387568EE73E008
:10B0500080E090E00E94AB79BE016E5D7F4FCE0133
:10B0600001960E94CE75AE014F5F5F4F63E070E0C6
:10B0700089E692E00E947125182FCE0101960E9468
:10B080003875111122C0BE016E5D7F4FCE014C9606
:10B090000E94CE7564ED77E0CE014C960E943D741F
:10B0A0006DED7FE00E945374BC01CE0101960E94B9
:10B0B000CE75CE0101960E946518CE0101960E94C0
:10B0C0003875CE014C960E94387568EE73E080E0CA
:10B0D00090E00E94AB7961ED7FE0CE0101960E9485
:10B0E000CE75AE014F5F5F4F61E070E080ED92E0A2
:10B0F0000E947125182FCE0101960E9438751111FA
:10B1000021C061ED7FE0CE014C960E94CE7564EDCA
:10B1100077E0CE014C960E943D746DED7FE00E9479
:10B120005374BC01CE0101960E94CE75CE010196EA
:10B130000E946518CE0101960E943875CE014C968A
:10B140000E94387568EE73E080E090E00E94AB7971
:10B150008091740C882311F40C94C64243E160ED95
:10B1600072E0CE0101960E94B68FBE016F5F7F4FE5
:10B170008FEB91E10E9493188FEB91E10E94638F16
:10B18000882311F40C94C64261ED7FE08FEB91E1CE
:10B190000E94347766E970E080E090E00E94AB792D
:10B1A0008FEB91E10E946F8F62E370E080E090E0AE
:10B1B0000E94AB790C94C64260EE77E0CE01019616
:10B1C0000E94D775BE016F5F7F4FCE01C4960E946B
:10B1D0002274182FCE0101960E943875112301F1B7
:10B1E0009AEDE92E9BE0F92E01E010E0F2E0EF0E7F
:10B1F000F11C8091A8029091A9028017910714F484
:10B200000C945F3860E0F70180810E9438786CE22E
:10B2100071E080E090E00E94AB790F5F1F4FE6CFB6
:10B2200064EE77E0CE0101960E94D775BE016F5F94
:10B230007F4FCE01C4960E942274182FCE01019632
:10B240000E943875112301F18AEDE82E8BE0F82E6B
:10B2500001E010E0F2E0EF0EF11C8091A802909165
:10B26000A9028017910714F40C945F3861E0F7018C
:10B2700080810E9438786CE271E080E090E00E946A
:10B28000AB790F5F1F4FE6CF69EE77E0CE010196F5
:10B290000E94D775BE016F5F7F4FCE01C4960E949A
:10B2A0002274182FCE0101960E943875112311F4D3
:10B2B0000C945F3827E030E046E050E06AEA7FE037
:10B2C000CE0101960E94EC75BE016F5F7F4F8CE846
:10B2D0009FE00E94FF74CE0101960E9438758CE8B1
:10B2E0009FE00E948973672B71F41092D90B6AEA70
:10B2F0007FE0CE0101960E94CE75CE0101960E949C
:10B30000691D0C94484581E08093D90BF0CF4F9292
:10B310005F926F927F928F929F92AF92BF92CF92E5
:10B32000DF92EF92FF920F931F93CF93DF93CDB7EE
:10B33000DEB72C970FB6F894DEBF0FBECDBF67E324
:10B3400070E080918302909184020E94010984E15F
:10B35000482E512C612C712CD12CC12CAFEFCA1A64
:10B36000DA0AC301B2010E94AB79E0908302F09047
:10B37000840267E370E0C7010E9401098C01B3E019
:10B38000CB16D10434F08EE1C816D10444F4012B5D
:10B3900051F094E1490E511C611C711CDFCF011565
:10B3A000110509F0AEC08BE0E816F10409F08EC07B
:10B3B00080905B1190905C11A0905D11B0905E1137
:10B3C0008091571190915811A0915911B0915A1133
:10B3D00089879A87AB87BC8764E670E080E090E05D
:10B3E0000E94AB796CE275E0CE0101960E94C575B2
:10B3F000CE0101960E94A01FCE0101960E943875D1
:10B4000061E082E00E94C37F21E0B501A401CE018A
:10B4100001960E944075BE016F5F7F4F8BED91E1F9
:10B420000E942677CE0101960E9438756FED8BED54
:10B4300091E10E949B7F67E275E08BED91E10E94B4
:10B44000487720E049855A856B857C85CE01019639
:10B450000E944075BE016F5F7F4F8BED91E10E94AE
:10B460002677CE0101960E94387560EF77E08BED6C
:10B4700091E10E941E7789829A82AB82BC82898583
:10B480009A85AB85BC858D839E83AF83B8872981E0
:10B490003A814B815C816D817E818F8198852C966C
:10B4A0000FB6F894DEBF0FBECDBFDF91CF911F91D5
:10B4B0000F91FF90EF90DF90CF90BF90AF909F9053
:10B4C0008F907F906F905F904F90089596E1E9166E
:10B4D000F10409F46DCFACE0EA16F10409F07CCF79
:10B4E0008090020B9090030BA090040BB090050B82
:10B4F0008091FE0A9091FF0AA091000BB091010B80
:10B5000067CF0F3F9FEF1907CCF069E175E0CE01DF
:10B5100001960E94C5754AE050E070E060E0CE01FF
:10B5200001960E948C19CE0101960E94387566EF33
:10B5300074E082E99FE00E94C37432C00E3FAFEF17
:10B540001A07B9F168EE74E0CE0101960E94C57544
:10B550004AE050E070E060E0CE0101960E948C1954
:10B56000CE0101960E94387569ED74E082E99FE092
:10B570000E94C374B801CE0101960E942573BE01DA
:10B580006F5F7F4F82E99FE00E94BC74CE010196FD
:10B590000E94387563EC74E082E99FE00E94667453
:10B5A00019821A821B821C821D821E821F821886AB
:10B5B0006ECF68EB74E0CE0101960E94C5754AE03B
:10B5C00050E070E060E0CE0101960E948C19CE013F
:10B5D00001960E94387568E974E0ABCF2F923F92D4
:10B5E0004F925F926F927F928F929F92AF92BF9293
:10B5F000CF92DF92EF92FF920F931F93CF93DF933F
:10B60000CDB7DEB7AC970FB6F894DEBF0FBECDBF97
:10B610008C017B018091570C9091580C019690936E
:10B62000580C8093570C2091560C222341F06AE06D
:10B6300070E00E9418AA181619060CF4BAC281E02C
:10B640008093560C1092580C1092570C50E040E02A
:10B650006AE074E0C8010E94121982E0E816F10461
:10B6600009F4C0C263ED78E08BEC9FE00E941B738D
:10B6700067E370E080918302909184020E94010947
:10B680001C016CE276E0C8010E94C41862EF77E00A
:10B69000C8010E941E7765E671E1CE0101960E9405
:10B6A000CE75BE016F5F7F4FC8010E942677CE0125
:10B6B00001960E9438756BEF77E0C8010E941E77F3
:10B6C00067E176E0C8010E9448776BE671E1CE0140
:10B6D00001960E94CE75BE016F5F7F4FC8010E9428
:10B6E00026776DE076E0C8010E94487765E870E152
:10B6F000CE0109960E94D775BE01675F7F4FC801D2
:10B700000E94267760E076E0C8010E9448776DEEDF
:10B7100070E1CE010F960E94D775BE01615F7F4F29
:10B72000C8010E94267769EF75E0C8010E9448773A
:10B73000CE010F960E943875CE0109960E94387589
:10B74000CE0101960E9438750E94697A28EE33E096
:10B7500040E050E00E948AA829013A016FEE75E0AE
:10B76000C8010E944877CE0101960E94D31FBE01F6
:10B770006F5F7F4FC8010E942677CE0101960E941D
:10B780003875C301B20120E13EE040E050E00E9484
:10B79000ACA84B015C01B901CE0187960E94221A28
:10B7A0004CE3C42ED12CE12CF12CC501B401A7012E
:10B7B00096010E94ACA8B901CE0101960E94221AFE
:10B7C00060EC76E0CE0109960E94D775BE016F5FEE
:10B7D0007F4FCE0109960E945374BC01CE0187961B
:10B7E0000E94BC74CE0109960E943875CE01019664
:10B7F0000E943875C301B201A70196010E94ACA84E
:10B80000CE0101960E94221A60EC76E0CE010996E4
:10B810000E94D775BE016F5F7F4FCE0109960E94CF
:10B820005374BC01CE0187960E94BC74CE01099668
:10B830000E943875CE0101960E94387561E078E06B
:10B84000CE0109960E94D775BE01695D7F4FCE017A
:10B8500009960E94537464E078E00E943D74BC0134
:10B86000CE0101960E94CE75BE016F5F7F4FC80169
:10B870000E942677CE0101960E943875CE01099666
:10B880000E94387562E178E0C8010E941E77CE01FF
:10B8900001960E947D72B801CE0101960E94AA769F
:10B8A0006DE078E0C8010E940A770E9487592983D9
:10B8B0003A834B835C836D837E838F839887498132
:10B8C0005A816B817C8121E0CE010F960E944075E8
:10B8D000BE01615F7F4FCE0109960E94CE756AE17D
:10B8E00078E0CE0109960E943D74BC018BEC9FE08C
:10B8F0000E94E874CE0109960E943875CE010F9619
:10B900000E94387561E278E0CE010F960E94D775EB
:10B910006BEC7FE0CE010F960E945374BC01CE0108
:10B9200009960E94CE75BE01675F7F4FC8010E94D5
:10B930002677CE0109960E943875CE010F960E9497
:10B9400038754D815E816F81788521E0CE01099641
:10B950000E944075BE01675F7F4F8BEC9FE00E94A5
:10B96000FF74CE0109960E94387563E378E0CE013A
:10B970000F960E94D7756BEC7FE0CE010F960E9468
:10B98000537464E478E00E943D74BC01CE010996D2
:10B990000E94CE75BE01675F7F4FC8010E94267767
:10B9A000CE0109960E943875CE010F960E94387517
:10B9B00040915D0C50915E0C60915F0C7091600C39
:10B9C00022E0CE010F960E9440756BE478E0CE0134
:10B9D00045960E94D775BE01615F7F4FCE014596A7
:10B9E0000E9453746DE578E00E943D74BC01CE0165
:10B9F00009960E94CE75BE01675F7F4FC8010E9405
:10BA00002677CE0109960E943875CE0145960E9490
:10BA10003875CE010F960E9438754091590C50919F
:10BA20005A0C60915B0C70915C0C22E0CE010F9679
:10BA30000E94407566E678E0CE0145960E94D77573
:10BA4000BE01615F7F4FCE0145960E9453746DE544
:10BA500078E00E943D74BC01CE0109960E94CE752B
:10BA6000BE01675F7F4FC8010E942677CE0109960D
:10BA70000E943875CE0145960E943875CE010F960A
:10BA80000E943875E6EF2E16EFEF3E062CF46FE1BC
:10BA900077E0C8010E94C4186FEC75E0C8010E94ED
:10BAA000C41822EAC22E22E0D22EEE24E394F12C16
:10BAB000F2E0CF0ED11C8091A8029091A9028E15C0
:10BAC0009F050CF468C0B701CE010F960E94257344
:10BAD0006CE877E0CE0145960E94D775BE01615FA4
:10BAE0007F4FCE0145960E9453746CED75E00E9425
:10BAF0003D74BC01CE0109960E94CE75BE01675F00
:10BB00007F4FC8010E942677B70183E0660F771F39
:10BB10008A95E1F76F5B7F4ECE014B960E94D775F9
:10BB2000BE01655E7F4FC8010E94267764E778E01A
:10BB3000C8010E941E77F60160817181660F771F30
:10BB4000660F771F675C7F4ECE0181960E94D77586
:10BB5000BE016F5D7F4FC8010E94267769E778E0DC
:10BB6000C8010E941E77CE0181960E943875CE01D1
:10BB70004B960E943875CE0109960E943875CE0109
:10BB800045960E943875CE010F960E943875FFEFDA
:10BB9000EF1AFF0A8DCFCE0187960E94387581E09B
:10BBA0008093770C65EE76E0C8010E94C41810926D
:10BBB000560CAC960FB6F894DEBF0FBECDBFDF912A
:10BBC000CF911F910F91FF90EF90DF90CF90BF909A
:10BBD000AF909F908F907F906F905F904F903F902D
:10BBE0002F9008956FE177E0C8010E94C418DACF62
:10BBF000AF92BF92CF92DF92EF92FF920F931F937B
:10BC0000CF93DF93CDB7DEB7A0970FB6F894DEBF22
:10BC10000FBECDBF63ED78E085EF9FE00E941B7300
:10BC200063ED78E089EE9FE00E941B7353E4E52EFC
:10BC300052E0F52E62EAC62E62E0D62E7BE3A72EF6
:10BC400072E0B72E01E010E08091A8029091A90265
:10BC5000801791070CF482C0F50181919191A19117
:10BC6000B1915F01892B8A2B8B2B19F5F60182810B
:10BC70009381F7012281338182179307D1F0880FD6
:10BC8000991FFC01EB52F44FD801AA0FBB1FA6521B
:10BC9000B44F60818C910E943878F6018281938143
:10BCA000F7019383828364E670E080E090E00E9475
:10BCB000AB79F70162817381CE0145960E942573AD
:10BCC000B801CE010F960E942573B80123E0660FDC
:10BCD000771F2A95E1F76F5B7F4ECE0109960E9490
:10BCE000D7756CED75E0CE0101960E94D775BE0147
:10BCF000675F7F4FCE0101960E9453746EE778E034
:10BD00000E943D74BE01615F7F4F0E9453746FEDCE
:10BD100075E00E943D74BE016B5E7F4F0E945374BC
:10BD2000BC0185EF9FE00E94BC74CE0101960E9489
:10BD30003875CE0109960E943875CE010F960E9483
:10BD40003875CE0145960E9438750F5F1F4FF2E09F
:10BD5000EF0EF11C22E0C20ED11C76CFE09147110C
:10BD6000F0914811EE0FFF1FED5BFD4F6081718177
:10BD7000CE0101960E94257346E050E0BE016F5F40
:10BD80007F4FCE0109960E944519BE01675F7F4F24
:10BD900089EE9FE00E94BC74CE0109960E9438751E
:10BDA000CE0101960E943875E0914911F0914A1137
:10BDB000EE0FFF1FED5BFD4F60817181CE0101969B
:10BDC0000E94257346E050E0BE016F5F7F4FCE01B9
:10BDD00009960E944519BE01675F7F4F89EE9FE07B
:10BDE0000E94BC74CE0109960E943875CE0101965E
:10BDF0000E9438756CED75E0CE0145960E94D775AE
:10BE00000E94697A28EE33E040E050E00E948AA860
:10BE100069017A0163ED78E0CE014B960E94D775F7
:10BE200063ED78E08BEF9FE00E941B73CE010196DB
:10BE30000E94D31F44E150E0BE016F5F7F4FCE01EF
:10BE400009960E944519BE01675F7F4F8BEF9FE007
:10BE50000E94FF74CE0109960E943875CE010196AA
:10BE60000E9438752AE0B701A601CE0109960E940A
:10BE7000767548E050E0BE01675F7F4FCE010F96B8
:10BE80000E9445196BEF7FE0CE0101960E94CE75AE
:10BE9000BE01615F7F4FCE0101960E945374BC01C9
:10BEA0008FEE9FE00E94E874CE0101960E943875E3
:10BEB000CE010F960E943875CE0109960E94387502
:10BEC0002AE0B701A601CE0109960E94767561E8C5
:10BED00078E0CE0101960E94D775BE01675F7F4F63
:10BEE000CE0101960E945374BE016B5E7F4F0E948B
:10BEF0005374BC018BEF9FE00E94BC74CE0101968D
:10BF00000E943875CE0109960E94387540915D0CEB
:10BF100050915E0C60915F0C7091600C21E0CE013D
:10BF200001960E944075BE016F5F7F4FCE014B9618
:10BF30000E94FF74CE0101960E94387568E878E08F
:10BF4000CE0101960E94D775BE01655E7F4FCE017E
:10BF500001960E945374BE016B5E7F4F0E94537422
:10BF6000BC018BEF9FE00E94BC74CE0101960E9441
:10BF70003875BE01655E7F4FCE0101960E94CE7579
:10BF800046E050E0BE016F5F7F4FCE0109960E94F0
:10BF90004519BE01675F7F4F8FEE9FE00E94BC7422
:10BFA000CE0109960E943875CE0101960E9438751F
:10BFB0004091590C50915A0C60915B0C70915C0C43
:10BFC00021E0CE0101960E944075BE016F5F7F4F58
:10BFD000CE014B960E94FF74CE0101960E943875E7
:10BFE00066E978E0CE0101960E94D775BE01655ED4
:10BFF0007F4FCE0101960E945374BE016B5E7F4F4E
:10C000000E945374BC018BEF9FE00E94BC74CE0170
:10C0100001960E943875BE01655E7F4FCE01019684
:10C020000E94CE7546E050E0BE016F5F7F4FCE01AB
:10C0300009960E944519BE01675F7F4F8FEE9FE012
:10C040000E94BC74CE0109960E943875CE010196FB
:10C050000E943875009183021091840267E370E0BA
:10C06000C8010E94010990931D0C80931C0C892B20
:10C0700049F067E370E0C8010E94010990931D0C2C
:10C0800080931C0C80911C0C90911D0C8C3F9F4F39
:10C090000CF4EEC00E94875929833A834B835C835A
:10C0A0006D837E838F83988749815A816B817C81E0
:10C0B00021E0CE0109960E944075BE01675F7F4F67
:10C0C000CE014B960E94FF74CE0109960E943875EE
:10C0D00060EA78E0CE0109960E94D775BE01655EE0
:10C0E0007F4FCE0109960E945374BE016B5E7F4F55
:10C0F0000E945374BC018BEF9FE00E94BC74CE0180
:10C1000009960E943875BE01655E7F4FCE01099683
:10C110000E94CE7546E050E0BE01675F7F4FCE01C2
:10C120000F960E944519BE01615F7F4F8FEE9FE021
:10C130000E94BC74CE010F960E943875CE010996FC
:10C140000E9438754D815E816F81788521E0CE0136
:10C1500009960E944075BE01675F7F4FCE014B96E6
:10C160000E94FF74CE0109960E9438756BEA78E050
:10C17000CE0109960E94D775BE01655E7F4FCE0144
:10C1800009960E945374BE016B5E7F4F0E945374E8
:10C19000BC018BEF9FE00E94BC74CE0109960E9407
:10C1A0003875BE01655E7F4FCE0109960E94CE753F
:10C1B00046E050E0BE01675F7F4FCE010F960E94C0
:10C1C0004519BE01615F7F4F8FEE9FE00E94BC74F6
:10C1D000CE010F960E943875CE0109960E943875DF
:10C1E00065EF7FE08BEF9FE00E94BC746CED75E023
:10C1F000CE0101960E94D77569EE7FE0CE010196CF
:10C200000E945374BC018FEE9FE00E94BC74CE016B
:10C2100001960E9438756FEE7FE0CE0101960E9474
:10C22000CE75CE0101960E946518CE0101960E943E
:10C2300038756AE070E080E090E00E94AB79CE0152
:10C240004B960E943875CE0145960E943875A0968F
:10C250000FB6F894DEBF0FBECDBFDF91CF911F9117
:10C260000F91FF90EF90DF90CF90BF90AF90089527
:10C2700061EB78E08BEF9FE00E94B27460EC78E0B5
:10C280008FEE9FE00E94B27467EC78E08BEF9FE046
:10C290000E94B27460EC78E08FEE9FE00E94B2746E
:10C2A0009FCFBF92CF92DF92EF92FF920F931F9397
:10C2B000CF93DF93CDB7DEB7C455D1090FB6F8944D
:10C2C000DEBF0FBECDBF6C018B0165965FAF4EAF79
:10C2D00065978091570C9091580C01969093580C4B
:10C2E0008093570C8091560C81113CC0BB24B394B1
:10C2F000B092560C1092580C1092570C63ED78E0E7
:10C30000CE01895B9F4F0E94D77563ED78E0CE0127
:10C31000835B9F4F0E94D77550E040E06AE074E075
:10C32000C6010E9412190130110509F0A6C063ED83
:10C3300078E08BEF9FE00E941B736596EEADFFAD3A
:10C3400065978081811124C00E94F85DB092770CBE
:10C35000CE01835B9F4F0E943875CE01895B9F4F52
:10C360000E9438750FB6F894DEBF0FBECDBFCC5A11
:10C37000DF4F0FB6F894DEBF0FBECDBFDF91CF9178
:10C380001F910F91FF90EF90DF90CF90BF90089595
:10C390006596EEADFFAD65978081882309F467C08F
:10C3A00000E210E09E012F5F3F4F40E250E0BE01EF
:10C3B0006F5D7F4FCE018D5A9F4F0E94B9710497D8
:10C3C00039F3BE016F5D7F4FCE018F5B9F4F0E949F
:10C3D000D775BE016F5B7F4FCE01895B9F4F0E9477
:10C3E000FF74CE018F5B9F4F0E943875BE016F5F57
:10C3F0007F4FCE018F5B9F4F0E94D775BE016F5B51
:10C400007F4FCE01835B9F4F0E94FF74CE018F5BF5
:10C410009F4F0E943875BE01695B7F4F8BEF9FE095
:10C420000E94BC7463968EAD9FAD6397892B09F40F
:10C43000AFCF6FED75E0CE018F5B9F4F0E94D77538
:10C44000BE01635B7F4FCE018F5B9F4F0E94537491
:10C450006CED75E00E943D74BC018BEF9FE00E9483
:10C46000BC74CE018F5B9F4F0E94387591CF6BEFEC
:10C470007FE087ED9FE00E94E8741092560C68CF31
:10C480002F923F924F925F926F927F928F929F92E4
:10C49000AF92BF92CF92DF92EF92FF920F931F93D2
:10C4A000CF93DF93CDB7DEB7C258D1090FB6F8945A
:10C4B000DEBF0FBECDBF6C015B0188EE482E83E06E
:10C4C000582E612C712C03EE13E09BE5892E912CE4
:10C4D0008C0E9D1E8CE0880E911C1B019FEF291A6B
:10C4E000390AD6015996ED90FC90F701858182308A
:10C4F00008F493C082859385A485B5858F719927AB
:10C50000AA27BB27892B8A2B8B2B09F086C040E2F8
:10C5100050E0BE016F5F7F4FC7010E940B888032E1
:10C5200009F07BC08981882309F477C0853E79F3BF
:10C530008E3269F38C8583FDEACF22961FAE1EAE44
:10C5400022978DE693E09FAF8EAF24961FAE24977F
:10C55000BE016F5F7F4FE0E080E04EE2DB019D9126
:10C56000BD019032A1F0883049F426E730E02C0F6D
:10C570003D1F2E0F311DD9014C93EF5F26E730E0B0
:10C580002C0F3D1F2E0F311DD9019C93EF5F8F5F44
:10C590008B3021F786E790E08C0F9D1F8E0F911D49
:10C5A000FC011082D60159966D917C9121E0AE017B
:10C5B0004A585F4FCE01CE960E94988A882369F12F
:10C5C000BE01625C7F4FCE0181960E94138FAE0147
:10C5D0004A585F4FBE016F5D7F4FCE01855A9F4F16
:10C5E0000E94818FCE01855A9F4F0E94638F8823BE
:10C5F00009F4ACC0F12CFA141B042CF569E0CE014F
:10C6000001960E94A375CE0101960E947C18CE016E
:10C6100001960E943875F394EECF6F961FAE1EAE52
:10C620006F97A3964CAE5DAE6EAE7FAEA3976D9640
:10C630001FAF0EAF6D97E6961FAE1EAEE697A8969B
:10C640001FAEA897CFCFB401CE0101960E94D77537
:10C65000CE0101960E947C18CE0101960E94387589
:10C66000E696EEADFFADE697309709F447C08581B9
:10C67000823008F443C060E474E0CE0101960E9469
:10C68000D775CE0101960E946518CE0101960E94D1
:10C6900038756F968EAD9FAD6F979C838B83A396F5
:10C6A0008CAD9DADAEADBFADA3978D839E83AF83A3
:10C6B000B887A7968CAD9DADAEADBFADA797898766
:10C6C0009A87AB87BC871A8309838DE0F401DE016A
:10C6D0001D9601900D928A95E1F7E6968EAD9FAD7D
:10C6E000E6979B8F8A8FB101CE0101960E9440622E
:10C6F000CE01855A9F4F0E946F8FF3CE61ED78E097
:10C70000CE0101960E94D775CE0101960E947C1839
:10C71000CE0101960E943875E696EEADFFADE69724
:10C7200040E050E0BA01309721F04389548965898F
:10C730007689CE0101960E945173CE0101960E9426
:10C740006518CE0101960E943875D2CFCE57DF4FC3
:10C750000FB6F894DEBF0FBECDBFDF91CF911F9112
:10C760000F91FF90EF90DF90CF90BF90AF909F9090
:10C770008F907F906F905F904F903F902F90089593
:10C780002F923F924F925F926F927F928F929F92E1
:10C79000AF92BF92CF92DF92EF92FF920F931F93CF
:10C7A000CF93DF93CDB7DEB7C954D1090FB6F89454
:10C7B000DEBF0FBECDBF40E052EC61E070E089E526
:10C7C0009DE00E94497140E855E260E070E08CEB2A
:10C7D0009CE00E94497161E088E00E94557961E027
:10C7E00089E00E94557960E08AE30E94557961E012
:10C7F00088E00E94387860E089E00E94387861E043
:10C800008AE00E94557961E08BE00E94557960E0F2
:10C810008BE30E94557961E08AE00E94387860E0FD
:10C820008BE00E9438780E943E7984EF91E09093EB
:10C830009B0280939A0268EE73E080E090E00E9491
:10C84000AB7989E59DE00E941F6EF82E6AE0C62E46
:10C85000D12CF1100BC089E59DE00E941F6EF82ECF
:10C860006EE170E080E090E00E94AB7921E0C21AB6
:10C87000D10879F780919A0290919B020DE210E124
:10C880005801FC01ED52F0414F01C4018A0D9B1D7E
:10C890000E9464A8F50181935F01F7E5AF16F1E10D
:10C8A000BF0699F76091471170914811072E000C4F
:10C8B000880B990B0E9447A79B01AC010E9407AA15
:10C8C000882331F081E090E09093481180934711E4
:10C8D0006091491170914A11072E000C880B990B39
:10C8E0000E9447A79B01AC010E9407AA882331F050
:10C8F00082E090E090934A118093491125E7F21667
:10C90000B1F0609143117091441180914511909163
:10C9100046110E9447A79B01AC010E9407AA811102
:10C9200006C080912D1090912E108197E8F08DB760
:10C930009EB78A5291400FB6F8949EBF0FBE8DBF2E
:10C94000ADB7BEB711968AE291E0EDE2F0E1019059
:10C950000D920197E1F70E94CE230FB6F894DEBF47
:10C960000FBECDBF55E7F52E2DB73EB72A52314049
:10C970000FB6F8943EBF0FBE2DBFADB7BEB7119630
:10C980008AE291E0EDE2F0E101900D920197E1F78A
:10C990000E944C1B0FB6F894DEBF0FBECDBF95E7CB
:10C9A000F91619F0E3E7FE121BC02DB73EB72A5265
:10C9B00031400FB6F8943EBF0FBE2DBFADB7BEB726
:10C9C00011968AE291E0EDE2F0E101900D9201977B
:10C9D000E1F70E94282B0FB6F894DEBF0FBECDBF43
:10C9E0006CEB7BE083EE9FE00E94C37466EA7BE021
:10C9F0008DED9FE00E94C3740E943E7964ED78E063
:10CA000089E59DE00E940A77B12CA12C47E2E42E33
:10CA1000992493949092B80CE092BA0C1092B90CAD
:10CA20001092BB0C81E00E947E7E8111AFC160EE4E
:10CA300078E089E59DE00E941E778E2D0E94937616
:10CA4000E092DF116CEF78E089E59DE00E941E77AF
:10CA50008E2D0E9493769FEFA91AB90AE394E0E421
:10CA6000EE12D8CF61E379E0AB2811F067E479E00A
:10CA700089E59DE00E940A770E943E791092E011BC
:10CA80008091E411823018F098E09093E011909139
:10CA9000E511992339F0813029F48091E011846007
:10CAA0008093E01162E370E080E090E00E94AB7957
:10CAB0006091E6118BED91E10E946E7F68EE73E06C
:10CAC00080E090E00E94AB7960E38BED91E10E9401
:10CAD000827F8BE4A82E86E4B82EC5010197F1F77A
:10CAE00060E38BED91E10E94827FC5010197F1F730
:10CAF00060E38BED91E10E94827F83E592E00197F4
:10CB0000F1F760E28BED91E10E94827F8091E0116C
:10CB100080620E94B27F84E08093E1118CE00E94E9
:10CB2000B27F81E00E94B27F9BE3A92E9FE1B92EE4
:10CB3000C5010197F1F782E08093E21186E00E943F
:10CB4000B27F82E00E94B27FC5010197F1F780E4D5
:10CB50000E94B27F22E9A22E22E0B22E3AE9832E71
:10CB600032E0932EF50161915F018BED91E10E941E
:10CB70009B7F8A149B04B1F70E94DD080E94C108C4
:10CB800064E670E080E090E00E94AB796EE87BE0C4
:10CB9000CE0101960E94C575CE0101960E946518CE
:10CBA000CE0101960E94387561E085E30E945579B7
:10CBB00061E085E30E94387861E08AE00E9455795F
:10CBC00061E08AE00E94387861E089E30E9455794B
:10CBD0008091EE0E803308F052C061E089E30E943C
:10CBE00055798091EE0E282F30E0F901EE0FFF1FEE
:10CBF000E20FF31FE55AF14F9081907C9963908387
:10CC00001092EF0E1092F00E2CE0622F0E940CAAF0
:10CC1000829FB00111249B012C0D3D1DF901EE0FE7
:10CC2000FF1FE20FF31FE55AF14F908196FD19C0E7
:10CC3000FFEFCF1ADF0A2CE0C216D10461F7813072
:10CC400009F0B1C01092800082E0809381001092C0
:10CC5000850010928400B19A80916F008260809369
:10CC60006F00E091EE0E8E2F90E0FC01EE0FFF1FA3
:10CC7000E80FF91FE55AF14F80818064808368ECEA
:10CC800070E080E090E00E94AB7968EE73E080E0B5
:10CC900090E00E94AB796DE77BE0CE0101960E94A7
:10CCA000C5754AE050E06FEF7FEFCE0101960E941C
:10CCB0008C19CE0101960E94387510920F0E1092B9
:10CCC0000D0E10920A0E1092090E84E08093080E49
:10CCD0000E94697A6B0161E08091080E0E9455798B
:10CCE00061E08091080E0E9438780E94081782E562
:10CCF0008093020E1092030E8091020E9091030E0B
:10CD00000E946C0C6AE0E62E8FEF0E94FE0BEA9404
:10CD1000E110FACF84E09EE00E947D8120E030E0C7
:10CD2000A90160E084E09EE00E94BF81E82E80932C
:10CD30000E0E31E0831709F462C00E94697A6C1903
:10CD40007D09613D774050F381E08093090E84E0D6
:10CD50009EE00E9493816FE67BE0CE0101960E94E7
:10CD6000C575CE0101960E946518CE0101960E94FC
:10CD700038756EE57BE0CE0101960E94C5756AE0CC
:10CD800070E0CE0101960E94F07F55C1843009F019
:10CD900065CE66E179E089E59DE00E941E778E2DE3
:10CDA0000E9493765BCE823061F410929000809363
:10CDB0009100109295001092940088BB80937100AE
:10CDC00050CF833069F41092A00082E08093A100DC
:10CDD0001092A5001092A40089BB8093720041CFED
:10CDE00081113FCF1092200182E0809321011092A7
:10CDF0002501109224018ABB8093730032CF2AEA66
:10CE000031E040E050E068E084E09EE00E94BF81B5
:10CE100082FF2AC0E0920F0E80910F0E812C912C80
:10CE20005401823029F4812C912CA12C40E4B42EA1
:10CE300020E030E0A90167E384E09EE00E94BF812A
:10CE4000A501940169E284E09EE00E94BF81809385
:10CE50000E0E8823D1F00E94697A6C197D09613D1C
:10CE6000774030F388E071CF54E0E52E0E94A18135
:10CE700080930E0EEA94E110F9CF8A3A11F082E025
:10CE800064CF82E080930F0EC7CF80910F0E823067
:10CE9000D1F420E030E0A9016AE384E09EE00E9442
:10CEA000BF81882311F086E050CF0E94A181807C51
:10CEB000803C19F483E080930F0E0E94A1810E94B0
:10CEC000A1810E94A18184E09EE00E94938180E57F
:10CED0008093020E1092030E81E00E94C683882385
:10CEE00009F464C18091330E811135CF8091270EF2
:10CEF000803109F062C182E08093330E1092450EBA
:10CF00001092460E1092470E1092480E8091280EF5
:10CF10009091290EB0E0A0E035E0880F991FAA1F7C
:10CF2000BB1F3A95D1F78093410E9093420EA09388
:10CF3000430EB093440E80E19EE090934A0E80939E
:10CF4000490E81E08093320E1092340E1092350E0D
:10CF50001092360E1092370E1092380E1092390E33
:10CF600010923A0E10923B0E10923C0E10923D0E13
:10CF700010923E0E10923F0E1092400E62E57BE042
:10CF8000CE0101960E94C575CE0101960E946518DA
:10CF9000CE0101960E94387541E060E474E0CE0154
:10CFA00001960E94B68FBE016F5F7F4F84EA91E1C8
:10CFB0000E9493188091A6119091A7119C838B8356
:10CFC0008091A8119091A911A091AA11B091AB11D3
:10CFD0008D839E83AF83B8878091AC119091AD1102
:10CFE000A091AE11B091AF1189879A87AB87BC87AA
:10CFF00083EE93E09A8389838DE0E0EBF1E1DE013B
:10D000001D9601900D928A95E1F78091BD11909146
:10D01000BE119B8F8A8F70E060E0CE0101960E9466
:10D0200040626CE47BE0CE0101960E94C575CE01A2
:10D0300001960E946518CE0101960E94387568EE2F
:10D0400073E080E090E00E94AB7943E160ED72E034
:10D05000CE0101960E94B68FBE016F5F7F4F8FEBAE
:10D0600091E10E94931863E17BE081ED9FE00E94D3
:10D07000C37468E07BE081ED9FE00E9466748FEBF3
:10D0800091E10E94638F882309F4B6C069EE7CE8C1
:10D0900080ED92E00E94388C811122C06EE479E02C
:10D0A000CE0101960E94D775CE0101960E947C1890
:10D0B000CE0101960E94387560ED72E0CE010196B6
:10D0C0000E94D775CE0101960E946518CE01019687
:10D0D0000E94387561ED7FE08FEB91E10E9434771B
:10D0E0008FEB91E10E946F8F66E970E080E090E045
:10D0F0000E94AB7960E679E0CE0101960E94D77577
:10D10000CE0101960E946518CE0101960E943875E5
:10D110001092730C6DED7AE0CE0101960E94C575F8
:10D12000CE0101960E946518CE0101960E943875C5
:10D130000E940C935C0168EE73E080E090E00E9436
:10D14000AB79D12CC12CAB2809F037C5EAE0CE165B
:10D15000D10409F4F3C2B601CE0101960E942573F1
:10D16000CE0101960E946518CE0101960E94387585
:10D1700060ED77E080E090E00E94AB790E940C9334
:10D180005C0168EE73E080E090E00E94AB79CE0134
:10D1900001960E947D72BE016F5F7F4F89E59DE021
:10D1A0000E94F476FFEFCF1ADF0ACDCF80E00E9415
:10D1B000C683882309F4CFCD95CE803209F0CBCD3C
:10D1C00083E08093330E40912A0E50912B0E609194
:10D1D0002C0E70912D0E4093450E5093460E609389
:10D1E000470E7093480E21E43EE080E19EE00E94ED
:10D1F00012868111A0CEAFCD63EF7AE0CE01019609
:10D200000E94C575CE0101960E947C18CE01019640
:10D210000E94387560ED72E06FCFF40111821082C8
:10D2200069E370E1CE0188960E94D775B801645E0B
:10D230007F4FCE0182960E94D775B701CE014C96E2
:10D240000E94257366E679E0CE0101960E94D775AB
:10D25000BE01645E7F4FCE0101960E94537460EC64
:10D2600076E00E943D74BE016E5D7F4F0E94537454
:10D270006FED75E00E943D74BE01685D7F4F0E94B6
:10D280005374BC0129968FAD29972A969FAD2A9792
:10D290000E94BC74CE0101960E943875CE014C9656
:10D2A0000E943875CE0182960E943875CE0188960C
:10D2B0000E943875F5011082118212821382F301E7
:10D2C0001082118212821382C7010E943E17FFEF63
:10D2D000EF1AFF0A810191C3CE014C960E94D31F21
:10D2E0006AE679E0CE0101960E94D775BE01645EC0
:10D2F0007F4FCE0101960E9453746CED75E00E9441
:10D300003D74BE01605C7F4F0E945374BC018BEF83
:10D310009FE00E94E874CE0101960E943875CE010C
:10D320004C960E943875CE0101960E94D31F46E1AB
:10D3300050E0BE016F5F7F4FCE014C960E944519B1
:10D34000BE01645E7F4FCE0182960E94CE75BE0103
:10D35000665C7F4FCE0182960E945374BC01CE0161
:10D36000CA960E94E874CE0182960E943875CE015A
:10D370004C960E943875CE0101960E9438756BEF6D
:10D380007FE0CE0101960E94CE75CE0101960E94EB
:10D390006518CE0101960E9438756BEF7FE0CE01D3
:10D3A00001960E94CE75AE014F5F5F4F62E070E064
:10D3B00086E792E00E947125182FCE0101960E9407
:10D3C0003875111121C06BEF7FE0CE0101960E94EC
:10D3D000CE7564ED77E0CE0101960E943D746DED4F
:10D3E0007FE00E945374BC01CE014C960E94CE7522
:10D3F000CE014C960E946518CE014C960E9438755D
:10D40000CE0101960E943875BE01665C7F4FCE0149
:10D4100001960E94CE75AE014F5F5F4F63E070E0F2
:10D4200089E692E00E947125CE0101960E9438752E
:10D43000CE01C4960E943875CE01CA960E943875F6
:10D44000CE01805C9F4F0E94387501E010E0109380
:10D45000AB020093AA02109368020093670266E38E
:10D4600077E08CE89FE00E941B73109368020093A2
:10D4700067026CE87FE0CE0101960E94CE7562E003
:10D4800070E0CE0101960E94522ECE0101960E94BC
:10D49000387564E77AE0CE0101960E94C575CE0129
:10D4A00001960E946518CE0101960E94387564E6C7
:10D4B0007AE0CE0101960E94C575CE0101960E94C8
:10D4C000A01FCE0101960E94387562E976E08CE8D3
:10D4D0009FE00E941B736CE87FE0CE0101960E94E2
:10D4E000CE7563E070E0CE0101960E94522ECE010F
:10D4F00001960E94387582E090E09093AB02809391
:10D50000AA0263E57AE0CE0101960E94C575CE01BC
:10D5100001960E946518CE0101960E94387567E455
:10D520007AE0CE0101960E94C575CE0101960E9457
:10D53000A01FCE0101960E94387566E377E08CE863
:10D540009FE00E941B73809153119091541197FF9B
:10D5500006C06AE377E08CE89FE00E941B736CE8EA
:10D560007FE0CE0101960E94CE7562E070E0CE01B0
:10D5700001960E94522ECE0101960E94387562E9F2
:10D5800076E08CE89FE00E941B7382E090E090932D
:10D59000AB028093AA026CE87FE0CE0101960E9464
:10D5A000CE7563E070E0CE0101960E94522ECE014E
:10D5B00001960E9438758091531190915411919564
:10D5C00081959109909354118093531101E010E0DB
:10D5D000109368020093670284EF91E090939B029E
:10D5E00080939A026DE270E10E94900864E670E018
:10D5F00080E090E00E94AB791093AB020093AA0206
:10D600008EEE9AE59093640F8093630F2091850FBF
:10D61000822F022E000C990B88309105C8F4FC0172
:10D62000EE0FFF1FEE0FFF1FEB59F04F44E759E0DD
:10D63000518340832F5F2093850F880F991F880F98
:10D64000991FFC01E959F04F88E59AE191838083A5
:10D650002091850F822F022E000C990B88309105A6
:10D66000C8F4FC01EE0FFF1FEE0FFF1FEB59F04F48
:10D670004AE759E0518340832F5F2093850F880F3D
:10D68000991F880F991FFC01E959F04F81E591E638
:10D690009183808385EF9EE00E94741465E37AE0B5
:10D6A000CE0101960E94C575CE0101960E946518B3
:10D6B000CE0101960E9438750E94487C60934A0C06
:10D6C00070934B0C80934C0C90934D0C1092560C15
:10D6D0000E94611F0E94487C60936D0C70936E0CD9
:10D6E00080936F0C9093700C80912C118093750C2B
:10D6F000882351F00E94487C6093650C7093660CFF
:10D700008093670C9093680CC75BDF4F0FB6F8945B
:10D71000DEBF0FBECDBFDF91CF911F910F91FF9064
:10D72000EF90DF90CF90BF90AF909F908F907F90C1
:10D730006F905F904F903F902F90089561ED7AE049
:10D74000CE0101960E94C575CE0101960E94651812
:10D75000CE0101960E94387568EE73E080E090E09B
:10D760000E94AB7969EE7CE885E892E00E94388CF3
:10D77000882331F066E17DE885E892E00E94388CEC
:10D7800066E970E080E090E00E94AB7943E165E8F3
:10D7900072E0CE0101960E94B68FBE016F5F7F4F8F
:10D7A0008FEB91E10E94931881E08093730CCE017E
:10D7B00001960E947D72BE016F5F7F4F8FEB91E1FA
:10D7C0000E94F4768FEB91E10E946F8F62E370E02C
:10D7D00080E090E00E94AB791092730C0E940429C3
:10D7E00068EE73E080E090E00E94AB790E9416271B
:10D7F00024E6C22ED12CF1100BC089E59DE00E94D9
:10D800001F6EF82E64E170E080E090E00E94AB793A
:10D8100021E0C21AD10879F764EB7AE0CE010196D3
:10D820000E94C575CE0101960E94A01FCE010196EF
:10D830000E94387532E781E0F31280E00E94FE0713
:10D840006AEA7AE08BEF9FE00E94C374CE010196F2
:10D850000E94D31FBE016F5F7F4F8BEF9FE00E943E
:10D86000BC74CE0101960E94387567E97AE08BEFAF
:10D870009FE00E94667465E87AE0CE0101960E94FE
:10D88000C575CE0101960E94A01FCE0101960E948F
:10D89000387567E370E080918302909184020E9462
:10D8A000010990931D0C80931C0C6BEF7FE0CE015F
:10D8B00001960E94CE75AE014F5F5F4F62E070E04F
:10D8C00086E792E00E947125F82ECE0101960E9413
:10D8D0003875F11021C06BEF7FE0CE0101960E94F8
:10D8E000CE7564ED77E0CE0101960E943D746DED3A
:10D8F0007FE00E945374BC01CE014C960E94CE750D
:10D90000CE014C960E946518CE014C960E94387547
:10D91000CE0101960E9438756BEF7FE0CE01019633
:10D920000E94CE75AE014F5F5F4F63E070E089E605
:10D9300092E00E947125F82ECE0101960E94387562
:10D94000F11021C06BEF7FE0CE0101960E94CE75F1
:10D9500064ED77E0CE0101960E943D746DED7FE0AD
:10D960000E945374BC01CE014C960E94CE75CE012C
:10D970004C960E946518CE014C960E943875CE01D7
:10D9800001960E94387568EE73E080E090E00E9496
:10D99000AB791E0180E4280E311C63ED78E0C101F3
:10D9A0000E94D77563ED78E0CE01CA960E94D775C4
:10D9B00063ED78E0CE01C4960E94D775E091A8028D
:10D9C000F091A9022896FFAFEEAF2897A2EA8A2E1F
:10D9D000A2E09A2EBBE5CB2EB2E0DB2E8FE4482EE0
:10D9E00082E0582E32015601EE24E394F12C299660
:10D9F0002FAE29972A963FAE2A97F2E08F0E911C00
:10DA0000180128E0220E311C34E0A30EB11C84E082
:10DA1000680E711C2896EEADFFAD2897EE15FF0538
:10DA20000CF0FBCB73E4A72E72E0B72EE9E4EE2EE8
:10DA3000E2E0FE2E01E010E0F8EE6F2EF3E07F2E24
:10DA4000812C912C22E0A20EB11C34E0C30ED11C1B
:10DA500082E0E80EF11C94E0490E511C8091A8026E
:10DA60009091A902801791070CF436CCF5016081E2
:10DA70007181CE0188960E94257342E050E0BE017C
:10DA8000685D7F4FCE018E960E944519B801CE0188
:10DA90004C960E94257342E050E0BE01645E7F4FC9
:10DAA000CE0182960E9445196CE877E0CE0101967E
:10DAB0000E94D775BE016E5D7F4FCE0101960E9418
:10DAC0005374BE01625D7F4F0E945374BC01CE014E
:10DAD000C4960E94E874CE0101960E943875CE016A
:10DAE00082960E943875CE014C960E943875CE0100
:10DAF0008E960E943875CE0188960E943875F60180
:10DB00006081718182819381A40193010E94ACA8FC
:10DB1000BA01A90120E0CE0101960E94767548E085
:10DB200050E0BE016F5F7F4FCE014C960E944519B9
:10DB3000BE01645E7F4FCE01C4960E94BC74CE01CC
:10DB40004C960E943875CE0101960E943875F701F7
:10DB500060817181CE0101960E94257343E050E0FF
:10DB6000BE016F5F7F4FCE014C960E944519BE01EA
:10DB7000645E7F4FCE01C4960E94BC74CE014C9669
:10DB80000E943875CE0101960E943875BE016C5C0A
:10DB90007F4FCE01CA960E94BC74F601108211829A
:10DBA00012821382F2011082118212821382C80142
:10DBB0000E943E170F5F1F4F45CF64EC7AE0C0CD47
:10DBC000089508950895AF92BF92CF92DF92EF9299
:10DBD000FF920F931F93CF93DF936C017B018B0117
:10DBE000040F151FEB015E01AE18BF08C017D10767
:10DBF00059F06991D601ED91FC910190F081E02DF1
:10DC0000C6011995892B79F7C501DF91CF911F9135
:10DC10000F91FF90EF90DF90CF90BF90AF9008955D
:10DC2000FC01538D448D252F30E0842F90E0821B22
:10DC3000930B541710F0CF96089501970895FC01A7
:10DC4000918D828D981761F0A28DAE0FBF2FB11DFF
:10DC50005D968C91928D9F5F9F73928F90E0089557
:10DC60008FEF9FEF0895FC01918D828D981731F011
:10DC7000828DE80FF11D858D90E008958FEF9FEF65
:10DC80000895FC01918D228D892F90E0805C9F4F3B
:10DC9000821B91098F73992708958CEB9CE00E9459
:10DCA000416E21E0892B09F420E0822F089589E557
:10DCB0009DE00E94416E21E0892B09F420E0822F33
:10DCC0000895FC01A48DA80FB92FB11DA35ABF4F11
:10DCD0002C91848D90E001968F739927848FA6896B
:10DCE000B7892C93A089B1898C91837080648C93BF
:10DCF000938D848D981306C00288F389E02D80816E
:10DD00008F7D80830895EF92FF920F931F93CF939F
:10DD1000DF93EC0181E0888F9B8D8C8D98131AC066
:10DD2000E889F989808185FF15C09FB7F894EE894D
:10DD3000FF896083E889F9898081837080648083AA
:10DD40009FBF81E090E0DF91CF911F910F91FF90F5
:10DD5000EF900895F62E0B8D10E00F5F1F4F0F739D
:10DD60001127E02E8C8D8E110CC00FB607FCFACF58
:10DD7000E889F989808185FFF5CFCE010E94616E27
:10DD8000F1CFEB8DEC0FFD2FF11DE35AFF4FF08229
:10DD90009FB7F8940B8FEA89FB8980818062CFCF8F
:10DDA000CF93DF93EC01888D8823B9F0AA89BB89D2
:10DDB000E889F9898C9185FD03C0808186FD0DC0BD
:10DDC0000FB607FCF7CF8C9185FFF2CF808185FFDE
:10DDD000EDCFCE010E94616EE9CFDF91CF91089522
:10DDE00080E090E0892B29F00E94576E81110E94FB
:10DDF000000080E090E0892B49F080E090E0892BE2
:10DE000029F00E94000081110E94000080E090E053
:10DE1000892B49F080E090E0892B29F00E940000D6
:10DE200081110E94000080E090E0892B29F00E947F
:10DE30004D6E81110C94000008958150823108F0DC
:10DE40005AC0E82FF0E08827E75DF0498F4F0C9427
:10DE50002CAA496F4D6F3B6F416F456F7B6F506FC1
:10DE6000566F5A6F606F646F686F6E6F726F7B6F03
:10DE7000766F7C6F806F809180008F7780938000B9
:10DE80000895809180008F7DF9CF80918000877FF9
:10DE9000F5CF84B58F7784BD089584B58F7DFBCF92
:10DEA0008091B0008F778093B00008958091B0008A
:10DEB0008F7DF9CF809190008F77809390000895A7
:10DEC000809190008F7DF9CF80919000877FF5CF72
:10DED0008091A0008F778093A00008958091A0008A
:10DEE0008F7DF9CF8091A000877FF5CF80912001B1
:10DEF0008F77809320010895809120018F7DF9CF45
:10DF000080912001877FF5CFCF93DF93282F30E0DA
:10DF1000F901E854F34F8491F901EE58F34FD4918D
:10DF2000F901E45DF34FC491CC23A1F081110E946B
:10DF30001D6FEC2FF0E0EE0FFF1FEE5EF34FA5918B
:10DF4000B491EC91ED2381E090E009F480E0DF9161
:10DF5000CF91089580E090E0FACF20911412260F1F
:10DF60003327331F21323105ECF42091B20CFC0130
:10DF700090E080E0243069F082E00895A0911412CE
:10DF80002191AC014C505E4EA40FB52FB11D2C93C6
:10DF90000196861798F380911412680F60931412FB
:10DFA00080E0089581E008950895E091720C8091D9
:10DFB000710CE81730F4F0E0EF5DF34F808190E0F2
:10DFC00008958FEF9FEF08959091720C8091710CDE
:10DFD0002FEF3FEF981748F4E92FF0E0EF5DF34F94
:10DFE000208130E09F5F9093720CC9010895809169
:10DFF000710C9091720C891B990B0895CF92DF924E
:10E00000EF92FF920F931F93CF93DF937C01CB018D
:10E010008A012091B80C222389F0EB016B01C40E18
:10E02000D51ECC15DD0569F06991D701ED91FC9104
:10E030000190F081E02DC7011995F3CF642F0E9464
:10E04000AD6FC801DF91CF911F910F91FF90EF90BD
:10E05000DF90CF900895CF93DF931F92CDB7DEB7B7
:10E0600069832091B80C2223F9F02091BB0C203257
:10E0700058F021E030E0FC013383228390E080E01F
:10E080000F90DF91CF9108958091B90CE82FF0E0C7
:10E09000E956FA4E998190838F5F8093B90C8093F3
:10E0A000BB0C81E090E0ECCF61E0CE0101960E94D4
:10E0B000AD6FF7CFDC015996ED91FC913097B9F037
:10E0C00083899489A589B689428553856485758538
:10E0D000841B950BA60BB70B811520E89207A105B1
:10E0E000B10538F08FEF9FE7A0E0B0E0089590E031
:10E0F00080E00895CF93DF931F92CDB7DEB7698399
:10E10000DC01ED91FC910280F381E02D41E050E0D3
:10E11000BE016F5F7F4F19950F90DF91CF910895EA
:10E120000E9455AC0F931F93CF93DF93EC0188812E
:10E130009981009759F02A813B812617370730F0E3
:10E1400081E0DF91CF911F910F9108958B016F5F57
:10E150007F4F0E9474AB009759F0998388831B838B
:10E160000A832C813D81232B59F7FC011082E8CFD3
:10E1700080E0E7CFEF92FF920F931F93CF93DF934F
:10E180006115710541F480E0DF91CF911F910F91EE
:10E19000FF90EF90089541155105B1F07B01EC011E
:10E1A0000C811D81040F151FB8010E9492708823F5
:10E1B00051F3288139818C819D81B701820F931F92
:10E1C0000E94A5AC1D830C8381E0DECFCF93DF934B
:10E1D000EC0188819981009711F00E94EBAA1982C5
:10E1E00018821D821C821B821A82DF91CF910895B2
:10E1F000EF92FF920F931F93CF93DF93EC017B017C
:10E200008A01BA010E94927081110BC0CE010E9456
:10E21000E670CE01DF91CF911F910F91FF90EF90AB
:10E2200008951D830C83B701888199810E94A5AC54
:10E23000F0CFCF92DF92EF92FF920F931F93CF9385
:10E24000DF93EC017A018B016C01C40ED51ECC1555
:10E25000DD05A9F00E94FC0B8FE00E94FE0B8D2FC4
:10E260000E94FE0B8C2F0E94FE0B219680E00E94E4
:10E27000FE0BF80181938F010E94FA0BE8CFC701D2
:10E28000DF91CF911F910F91FF90EF90DF90CF9092
:10E290000895CF93DF93EC019A01AB01E889F989E6
:10E2A00082E08083211581EE38074105510581F117
:10E2B00060E079E08DE390E00E948AA82150310966
:10E2C000410951095695479537952795EC85FD8568
:10E2D0001082EE85FF852083188EEC89FD8986E00B
:10E2E0008083EA89FB89808180618083EA89FB8958
:10E2F000808188608083EA89FB898081806880834F
:10E30000EA89FB8980818F7D8083DF91CF91089599
:10E31000E889F989108220E1D9CFCF93C82F462F01
:10E3200061E070E00E94050C61E070E08C2F0E94BB
:10E33000200C8111F9CFCF910895FF920F931F9375
:10E34000CF93DF93F82E10E000E08F2D0E94510C48
:10E35000EC01892B21F08F2D0E94510C8C01C017EC
:10E36000D10799F7CE01DF91CF911F910F91FF90C7
:10E3700008954F925F926F927F928F929F92AF9289
:10E38000BF92CF92DF92EF92FF920F931F93CF93A2
:10E39000DF9300D0CDB7DEB72C015B014A01390114
:10E3A000FC01C080D18070E060E0C5010E948AACB1
:10E3B000A80170E060E0C3010E948AACF601808190
:10E3C000882309F493C07601FFEFEF1AFF0AF601E4
:10E3D00060816632A9F06CF5662389F0653209F434
:10E3E00047C0F2E08F16910444F0F5016083F1E03C
:10E3F0008F1A9108C50101965C016701E4CF76018F
:10E4000081E090E0F201F182E0820F900F900F9096
:10E41000DF91CF911F910F91FF90EF90DF90CF9000
:10E42000BF90AF909F908F907F906F905F904F9034
:10E4300008956B3209F45DC06D3399F681818823AC
:10E44000F9F26701FFEFCF1ADF0AF7016081653249
:10E4500079F144F56623B9F1023011053CF0F3017E
:10E46000608301501109C30101963C017601E9CF97
:10E4700081818983882321F282818A8376018111B7
:10E4800004C0F2E0EF0EF11CBBCF83E0E80EF11CFC
:10E490001B8240E150E070E060E0CE0101960E94F6
:10E4A000A9A19FCF663281F06B32B1F660E2D4CF82
:10E4B000818189838823F9F082818A83811108C050
:10E4C000F2E0EF0EF11C6701760183E090E09ACF55
:10E4D000670183E0C80ED11C1B8240E150E070E070
:10E4E00060E0CE0101960E94A9A1B6CF84E090E041
:10E4F0008CCF60E276CF7601E6CFCF93DF93EC014D
:10E5000081E094E0998388831A821B821C821D8299
:10E5100080E590E00E946C0CBE016E5F7F4F44E08E
:10E5200050E08FE090E00E9419710E946B0CCE01C8
:10E53000DF91CF9108950F931F93CF93DF934115F0
:10E54000510541F0FC01048115810115110539F4D3
:10E55000FB011082DF91CF911F910F9108954150DF
:10E5600051094017510708F48A01EB01FC01608151
:10E570007181A801CE010E94BAACC00FD11F1882D0
:10E58000E9CFAF92BF92CF92DF92EF92FF920F93BB
:10E590001F93CF93DF931F921F92CDB7DEB77A837D
:10E5A0006983BA01A901E981FA81F770082F10E0A7
:10E5B000000F111F0C57134FD8018D919C918E0F96
:10E5C0009F1F9F01240F351F21303840A0F05A01B2
:10E5D0006B0160E078E07B01EE1AFF0AA701B6014B
:10E5E0000E941971A5014E195F09B6016E0D7F1DBC
:10E5F000F801808191810F900F90DF91CF911F9151
:10E600000F91FF90EF90DF90CF90BF90AF900C9460
:10E61000197120E3FC0120833296862F82958F703A
:10E620006F706A3030F4605D6293682F8111F5CFAE
:10E630000895695CF9CFFB0101900020E9F731975B
:10E64000AF01461B570B0C94F8700F931F93CF9399
:10E65000DF93CDB7DEB762970FB6F894DEBF0FBE7B
:10E66000CDBF8C01CB01F80111821082138212827E
:10E67000158214824AE0BE016F5F7F4F0E94F0A2B4
:10E68000BE016F5F7F4FC8010E941B7362960FB679
:10E69000F894DEBF0FBECDBFDF91CF911F910F91D8
:10E6A00008950F931F93CF93DF93CDB7DEB7A19754
:10E6B0000FB6F894DEBF0FBECDBF8C01CB01BA01FF
:10E6C000F8011182108213821282158214822AE0CC
:10E6D000AE014F5F5F4F0E942AA3BE016F5F7F4F65
:10E6E000C8010E941B73A1960FB6F894DEBF0FBE3F
:10E6F000CDBFDF91CF911F910F910895FC018081D3
:10E700009181009711F00C94ACA260E070E0CB0115
:10E710000895FC0180819181009711F00C94B0A2C2
:10E7200060E070E0CB010895AF92BF92CF92DF928C
:10E73000EF92FF920F931F93CF93DF93DC01CD9065
:10E74000DC901197C114D10439F01496CD91DC916D
:10E750008C017601209761F4DF91CF911F910F9189
:10E76000FF90EF90DF90CF90BF90AF90089575012C
:10E770005701BFEFAB1ABB0AF7018081082E000CCE
:10E78000990B0E94D7A2892B91F72197CC0DDD1D03
:10E790008881082E000C990B0E94D7A2892B29F0A2
:10E7A000CE15DF0510F02197F3CFAE014F5F5F4F1D
:10E7B0004E195F09D80115965C934E931497CE14A9
:10E7C000DF0420F4B701C6010E946FACD801ED91BF
:10E7D000FC91119714968D919C91E80FF91F10826E
:10E7E000BBCFFC01248135816217730748F4808117
:10E7F0009181009729F0860F971FFC018081089571
:10E8000080E00895FC0124813581FB01448155811C
:10E8100024173507A0F0FC0180819181009779F0E1
:10E82000FB01608171816115710549F0241B350B75
:10E83000820F931F0E949CAC21E0892B09F020E0FD
:10E84000822F0895FB0144815581FC01248135818B
:10E850002417350778F080819181009759F0FB01EA
:10E86000608171816115710529F00E94ACAC21E0D5
:10E87000892B09F020E0822F0895CF93DF93EC01DC
:10E88000FB0101900020E9F73197AF01461B570BC0
:10E890000E94BA70811103C0CE010E94E670CE01C1
:10E8A000DF91CF910895CF93DF93EC01FB01448179
:10E8B0005581608171810E94BA70811103C0CE01BF
:10E8C0000E94E670CE01DF91CF910895EF92FF9202
:10E8D0000F931F93CF93DF93EC017B01CB010E9439
:10E8E000E7A20097A9F00C811D81080F191FB8013C
:10E8F000CE010E949270882361F0288139818C8139
:10E900009D81B701820F931F0E94E0A21D830C839B
:10E9100081E0DF91CF911F910F91FF90EF900895CB
:10E92000CF93DF931F921F92CDB7DEB769831A8210
:10E9300041E050E0BE016F5F7F4F0E94BA700F90C0
:10E940000F90DF91CF910895CF93DF93EC010E9458
:10E950009074811103C0CE010E94E670CE01DF9158
:10E96000CF910895FB0101900020E9F73197AF01A5
:10E97000461B570B0C94BA70FB0144815581608192
:10E9800071810C94BA70EF92FF920F931F93CF9303
:10E99000DF93EC018B01CB010E94E7A27C01BC015B
:10E9A000CE010E94927081110BC0CE010E94E670D0
:10E9B000CE01DF91CF911F910F91FF90EF900895BD
:10E9C000FD82EC82B801888199810E94E0A2F0CF9B
:10E9D000CF93DF93EC01FB018617970749F0608125
:10E9E00071816115710541F0448155810E94F87073
:10E9F000CE01DF91CF9108950E94E670F9CF0F9379
:10EA00001F93CF93DF938C01EB01FC0180819181F7
:10EA10000097E1F06881798161157105A9F0428163
:10EA200053812C813D814217530770F00E94A5ACA1
:10EA30008C819D81F801958384831D821C82DF91E6
:10EA4000CF911F910F9108950E94EBAA888199811F
:10EA5000F801918380838A819B81938382838C8157
:10EA60009D8195838483198218821B821A82E5CF47
:10EA7000FC0180819181009711F00C94EBAA08951C
:10EA8000EF92FF920F931F93CF93DF93CDB7DEB733
:10EA9000A1970FB6F894DEBF0FBECDBF7C01CB01AE
:10EAA000BA01F70111821082138212821582148238
:10EAB00042E0420F8E010F5F1F4F0E94E7A00097B8
:10EAC00089F0BC01C7010E941B73A1960FB6F89490
:10EAD000DEBF0FBECDBFDF91CF911F910F91FF9091
:10EAE000EF900895C7010E94E670EFCF0F931F9338
:10EAF000CF93DF93CDB7DEB7A2970FB6F894DEBF02
:10EB00000FBECDBF8C01CB01BA01F801118210827A
:10EB1000138212821582148230E0AE014F5F5F4F84
:10EB20000E94FBA2BE016F5F7F4FC8010E941B7352
:10EB3000A2960FB6F894DEBF0FBECDBFDF91CF9186
:10EB40001F910F910895CF93DF931F921F92CDB71E
:10EB5000DEB7FC01118210821382128215821482A8
:10EB600069831A82BE016F5F7F4F0E941B730F90F3
:10EB70000F90DF91CF910895FC01118210821382D2
:10EB80001282158214820C94FF74FC01118210828F
:10EB900013821282158214820C94C374FC011182B8
:10EBA000108213821282158214820C94E874FC0184
:10EBB00011821082138212821582148261157105EE
:10EBC00051F0FB0101900020E9F73197AF01461B9E
:10EBD000570B0C94F8700895AF92BF92CF92DF92CA
:10EBE000EF92FF920F931F93CF93DF936C015B0122
:10EBF0007A0189012417350720F48F2D7901042F1C
:10EC0000182F63ED78E0C6010E94D775D5011496E0
:10EC1000CD91DC91EC16FD06E0F40C171D0708F40D
:10EC2000E801D501ED91FC911197EC0FFD1F1081CA
:10EC300010826D917C916E0D7F1DC601611571056D
:10EC4000A1F00E941B73F50180819181C80FD91F2B
:10EC50001883C601DF91CF911F910F91FF90EF9024
:10EC6000DF90CF90BF90AF9008950E94E670EBCFF9
:10EC7000FB0101900020E9F73197AF01461B570BCC
:10EC8000DC01ED91FC910280F381E02D19948F92CB
:10EC90009F92AF92BF92EF92FF920F931F93CF93E9
:10ECA000DF93CDB7DEB7A1970FB6F894DEBF0FBEE6
:10ECB000CDBF7C01FA01CB0119A2223008F42AE071
:10ECC0008E010F5D1F4F822E912CB12CA12CBF0104
:10ECD000A50194010E948AA8F901CA016A300CF5C5
:10ECE000605DD8016E938D01232B242B252B79F7A2
:10ECF00090E080E0109721F0BD01C7010E943876B6
:10ED0000A1960FB6F894DEBF0FBECDBFDF91CF91B5
:10ED10001F910F91FF90EF90BF90AF909F908F90B9
:10ED20000895695CDECFCF93DF93482F50E070E009
:10ED300060E020E189E59DE00E944776EC0167EE06
:10ED400079E089E59DE00E9438768C0F9D1FDF9168
:10ED5000CF9108958F929F92AF92BF92CF92DF9200
:10ED6000EF92FF920F931F93CF93DF937C01EB0100
:10ED70006C0182E0C80ED11C4701E5E08E0E911CAB
:10ED800010E000E0F60141916F0150E070E060E0BA
:10ED90002AE0CE010E9447765C01E881F98101906A
:10EDA000F081E02D6EE2CE0119958A0D9B1D080FB2
:10EDB000191FC814D90431F7F701458150E070E0FC
:10EDC00060E02AE0CE010E944776800F911FDF911C
:10EDD000CF911F910F91FF90EF90DF90CF90BF9058
:10EDE000AF909F908F9008950F931F93CF93DF93D1
:10EDF000EC01CB01BE010E94AA768C0167EE79E09E
:10EE0000CE010E943876800F911FDF91CF911F9124
:10EE10000F9108950F931F93CF93DF93EC010E94FE
:10EE200038768C0167EE79E0CE010E943876800F4B
:10EE3000911FDF91CF911F910F9108956115710579
:10EE400011F00C94387690E080E00895DB01149680
:10EE50004D915C9115976D917C91DC01ED91FC9148
:10EE60000280F381E02D19940F931F93CF93DF93CA
:10EE7000EC010E9426778C0167EE79E0CE010E94BA
:10EE80003876800F911FDF91CF911F910F910895D8
:10EE9000EF92FF920F931F93CF93DF938C017B012F
:10EEA000D0E0C0E0F701EC0FFD1F6491662361F034
:10EEB000D801ED91FC910190F081E02DC8011995E8
:10EEC000892B11F02196EECFCE01DF91CF911F91CA
:10EED0000F91FF90EF900895DC0181E094E08D9315
:10EEE0009D9384E0FB0101900D928A95E1F70895CE
:10EEF0001F920F920FB60F9211240BB60F922F9301
:10EF00003F934F935F936F937F938F939F93AF93B1
:10EF1000BF93EF93FF938CEB9CE00E94616EFF9197
:10EF2000EF91BF91AF919F918F917F916F915F9181
:10EF30004F913F912F910F900BBE0F900FBE0F90EE
:10EF40001F9018951F920F920FB60F9211240BB6B7
:10EF50000F922F938F939F93EF93FF93E091CC0C9D
:10EF6000F091CD0C8081E091D20CF091D30C82FD18
:10EF70001DC090818091D50C8F5F8F732091D60C2E
:10EF8000821741F0E091D50CF0E0E454F34F958FF7
:10EF90008093D50CFF91EF919F918F912F910F90BE
:10EFA0000BBE0F900FBE0F901F9018958081F2CF6F
:10EFB0001F920F920FB60F9211240BB60F922F9340
:10EFC0003F934F935F936F937F938F939F93AF93F1
:10EFD000BF93EF93FF9389E59DE00E94616EFF91DF
:10EFE000EF91BF91AF919F918F917F916F915F91C1
:10EFF0004F913F912F910F900BBE0F900FBE0F902E
:10F000001F9018951F920F920FB60F9211240BB6F6
:10F010000F922F938F939F93EF93FF93E091690D3E
:10F02000F0916A0D8081E0916F0DF091700D82FD7D
:10F030001DC090818091720D8F5F8F732091730D31
:10F04000821741F0E091720DF0E0E75AF24F958F90
:10F050008093720DFF91EF919F918F912F910F905F
:10F060000BBE0F900FBE0F901F9018958081F2CFAE
:10F070001F93CF93DF93282F30E0F901E854F34F2B
:10F080008491F901EE58F34FD491F901E45DF34F07
:10F09000C491CC23A9F0162F81110E941D6FEC2F73
:10F0A000F0E0EE0FFF1FE850F44FA591B4918FB739
:10F0B000F894EC91111108C0D095DE23DC938FBF3A
:10F0C000DF91CF911F910895DE2BF8CFAF92BF92C1
:10F0D000CF92DF92EF92FF920F931F93CF93DF9324
:10F0E0006B017A01EC01C65EDC4E28813CE0389F62
:10F0F0008001399F100D1124A090D515B12C27FF48
:10F100001FC0FB011182108288818F5F88838881F4
:10F110009801280F311D87FD3A95F6012A153B0508
:10F120001CF488818C30C4F18081918104968034F4
:10F130009C4908F473C0F60180819181049670C0E7
:10F1400088819801280F311D87FD3A952A153B05C6
:10F15000DCF68881A801480F511D87FD5A95FA01F8
:10F16000EE0FFF1FE40FF51FE55AF14F808186FF78
:10F17000CBCF8881F801E80FF11D87FDFA95CF010B
:10F18000EE0FFF1FE80FF91FE55AF14F808160E095
:10F190008F730E943878B8CF808191812881A8012F
:10F1A000420F511D27FD5A959A01FA01EE0FFF1FDC
:10F1B000E20FF31FE55AF14F21813281820F931F35
:10F1C000F7019183808388819801280F311D87FD85
:10F1D0003A95F901EE0FFF1FE20FF31FE55AF14FC9
:10F1E000808186FF22C08881080F111D87FD1A9536
:10F1F000F801EE0FFF1FE00FF11FE55AF14F80817C
:10F2000061E08F73DF91CF911F910F91FF90EF908D
:10F21000DF90CF90BF90AF900C94387880E49CE959
:10F22000F701918380838FEF8883DF91CF911F91C6
:10F230000F91FF90EF90DF90CF90BF90AF90089527
:10F240001092B20C81E08093B10C10928C0C61E0B2
:10F2500084E10E94387861E085E10E943878E9EB2A
:10F26000F0E080818E7F808380818D7F808388E441
:10F270008093B80085E48093BC0008951092720CCE
:10F280001092710C1092B90C1092BB0C0E94207954
:10F2900080EE9DE690932C1380932B1381EE9DE6D8
:10F2A00090932A13809329130895CF93DF9390E0CE
:10F2B000FC01EE58F34F2491845D934FFC0184913F
:10F2C0008823D1F090E0880F991FFC01E252F44F9F
:10F2D000A591B491FC01E850F44FC591D49161110E
:10F2E0000EC09FB7F8948C91E22FE0958E238C93FB
:10F2F0002881E223E8839FBFDF91CF9108958FB7E4
:10F30000F894EC91E22BEC938FBFF6CF3FB7F894D3
:10F310008091231390912413A0912513B09126136B
:10F3200026B5A89B05C02F3F19F00196A11DB11D60
:10F330003FBFBA2FA92F982F8827BC01CD01620F9C
:10F34000711D811D911D42E0660F771F881F991F57
:10F350004A95D1F708958F929F92AF92BF92CF9224
:10F36000DF92EF92FF926B017C010E9486794B0144
:10F370005C01C114D104E104F104B9F00E94867962
:10F38000681979098A099B09683E734081059105CE
:10F3900080F321E0C21AD108E108F10888EE880E56
:10F3A00083E0981EA11CB11CE4CFFF90EF90DF908A
:10F3B000CF90BF90AF909F908F900895AF92BF92E3
:10F3C000CF92DF92EF92FF920F931F93CF93DF9331
:10F3D000C82FD62F10925F111092601110926111F8
:10F3E000109262111092631161E00E94557960E001
:10F3F0008C2F0E9438786D2F70E090E080E00E94A2
:10F40000AB7960E08C2F0E9455798BE990E00197F1
:10F41000F1F700E911E08C2F0E94846F892B81F4B1
:10F4200001501109C1F78EEF9FEFDF91CF911F912E
:10F430000F91FF90EF90DF90CF90BF90AF90089525
:10F4400000E911E08C2F0E94846F019721F4015094
:10F450001109C1F7E8CF18E2D0E800E090E9E92E01
:10F46000FF24F3948C2F0E94846F892B29F481E070
:10F47000E81AF108B9F7D7CF0E9486796B017C01B1
:10F4800080E9A82EBB24B3948C2F0E94846F01972F
:10F4900029F481E0A81AB108B9F7C5CF0E9486798E
:10F4A0006C197D098E099F096932710581059105E5
:10F4B00038F0E02FF0E0E95AFE4E80858D2B8087F2
:10F4C000D69511F40F5FD0E8115041F690E080E03E
:10F4D000ACCF2FB7F89460911F13709120138091D7
:10F4E0002113909122132FBF0895CF92DF92EF92B4
:10F4F000FF92CF93DF938091070F843051F4CFEFC9
:10F50000DFEFCE01DF91CF91FF90EF90DF90CF90B2
:10F510000895E0912A0FE1113EC00E94697A6B01C3
:10F520007C0128EEC20E23E0D21EE11CF11C8BEF01
:10F530009EE00E94350F882311F38091600F88238D
:10F5400031F080912B0F90912C0F892BC1F28BEF12
:10F550009EE00E94060EEC01CF3FDC0771F0809127
:10F56000600F882371F280912B0F90912C0F0197DF
:10F5700090932C0F80932B0FC4CF0E94697AC616EC
:10F58000D706E806F90698F610922A0F8BEF9EE050
:10F590000E94E014B6CFE150E0932A0F0E2E000C2B
:10F5A000FF0BEF50F14FC18DD0E0ABCF0F931F9306
:10F5B000CF93DF93EC018C01F80181918F018823B7
:10F5C000C1F10E94757AF8012291022E000C330BD2
:10F5D0008217930789F38F3F980791F0A0912A0F24
:10F5E00091E09A0F90932A0F0A2E000CBB0BAF509C
:10F5F000B14F59968C93903219F48FE180932A0F72
:10F600002FE1EC17FD07D9F092919F3FD1F3A09124
:10F610002A0F81E08A0F80932A0F0A2E000CBB0B61
:10F62000AF50B14F59969C93803259F720932A0FCF
:10F63000E8CF81E0DF91CF911F910F91089580E095
:10F64000F9CF1F920F920FB60F9211242F933F9371
:10F650008F939F93AF93BF9380911F13909120132B
:10F66000A0912113B091221330911E1323E0230F98
:10F670002D3758F50196A11DB11D20931E138093BF
:10F680001F1390932013A0932113B0932213809102
:10F69000231390912413A0912513B0912613019662
:10F6A000A11DB11D8093231390932413A0932513C0
:10F6B000B0932613BF91AF919F918F913F912F915E
:10F6C0000F900FBE0F901F90189526E8230F0296FB
:10F6D000A11DB11DD2CF1F920F920FB60F92112410
:10F6E0000BB60F922F933F934F935F936F937F933C
:10F6F0008F939F93AF93BF93EF93FF9348E251E0B3
:10F7000064E271E090E080E00E946678FF91EF9102
:10F71000BF91AF919F918F917F916F915F914F9129
:10F720003F912F910F900BBE0F900FBE0F901F9027
:10F7300018951F920F920FB60F9211240BB60F92CD
:10F740002F933F934F935F936F937F938F939F93E9
:10F75000AF93BF93EF93FF9348EA50E064EA70E001
:10F7600083E090E00E946678FF91EF91BF91AF91A6
:10F770009F918F917F916F915F914F913F912F91C9
:10F780000F900BBE0F900FBE0F901F9018951F92F9
:10F790000F920FB60F9211240BB60F922F933F9337
:10F7A0004F935F936F937F938F939F93AF93BF9389
:10F7B000EF93FF9348E950E064E970E082E090E065
:10F7C0000E946678FF91EF91BF91AF919F918F91C9
:10F7D0007F916F915F914F913F912F910F900BBE51
:10F7E0000F900FBE0F901F9018951F920F920FB69B
:10F7F0000F9211240BB60F922F933F934F935F9369
:10F800006F937F938F939F93AF93BF93EF93FF93E8
:10F8100048E850E064E870E081E090E00E9466789B
:10F82000FF91EF91BF91AF919F918F917F916F91D8
:10F830005F914F913F912F910F900BBE0F900FBE94
:10F840000F901F9018956093161370931713809361
:10F85000181390931913645D7E4F8F4F9F4F6093E1
:10F86000121370931313809314139093151382E063
:10F8700090E090931113809310130E94697A609323
:10F880000C1370930D1380930E1390930F13089520
:10F89000CF92DF92EF92FF920F931F930E94697AAB
:10F8A0008B019C01C0900C13D0900D13E0900E13AF
:10F8B000F0900F1360911613709117138091181325
:10F8C000909119130C191D092E093F09083E134088
:10F8D00021053105E0F0DC01CB010196A11DB11D30
:10F8E0008093161390931713A0931813B0931913C2
:10F8F000B701A60148515C4F6F4F7F4F40930C13E7
:10F9000050930D1360930E1370930F13C7CF1F9175
:10F910000F91FF90EF90DF90CF9008954F925F92FC
:10F920006F927F928F929F92AF92BF92CF92DF920F
:10F93000EF92FF920F931F93CF93DF934B015C01E4
:10F940008091081390910913A0910A13B0910B13A1
:10F9500088159905AA05BB0509F4C6C08CE3C82E15
:10F96000D12CE12CF12CC501A70196010E948AA897
:10F970006093410CCA01B901A70196010E948AA8AF
:10F980006093420CC501B40120E13EE040E050E04C
:10F990000E948AA8CA01B90128E130E040E050E0A5
:10F9A0000E948AA86093430CC501B40120E831E5A8
:10F9B00041E050E00E948AA869017A01CA01B901B8
:10F9C0006C5F7F4F8F4F9F4F27E030E040E050E06B
:10F9D0000E948AA86F5F6093440C412C512C320125
:10F9E00040E004E610E0C0E9D1E0242F30E02E54DE
:10F9F000384FF901E370FF273097F9F4C901B801D6
:10FA00000E9418AA892B31F4C901BE010E9418AACC
:10FA1000892B99F48EE691E0A0E0B0E0480E591EE3
:10FA20006A1E7B1ED301C201AA27BB27C816D906AE
:10FA3000EA06FB0638F04F5FD8CF8DE691E0A0E0F4
:10FA4000B0E0ECCF4093470CC90164E670E00E943F
:10FA500018AAEC01C90160E971E00E9418AA309768
:10FA600021F42097D9F40097C9F04DE651E060E009
:10FA700070E0441A550A660A770AC418D508E608E1
:10FA8000F708A3E2B3E020E0213069F43097E9F50C
:10FA9000209711F40097C9F54DE106C04EE651E0FC
:10FAA00060E070E0E6CF4C9150E070E060E031E063
:10FAB000320FC416D506E606F70640F0C41AD50A7A
:10FAC000E60AF70A1196232F3C30F1F62F5F2093B8
:10FAD000460CC394C092450C80920813909209136F
:10FAE000A0920A13B0920B13DF91CF911F910F9147
:10FAF000FF90EF90DF90CF90BF90AF909F908F904E
:10FB00007F906F905F904F9008954CE1CDCF0E9411
:10FB1000487C0E948E7C8091470C90E08E54984FD8
:10FB200008950E94487C0E948E7C8091460C90E053
:10FB300008950E94487C0E948E7C8091450C90E044
:10FB400008950E94487C0E948E7C8091420C90E037
:10FB500008950E94487C0E948E7C8091430C90E026
:10FB600008951F920F920FB60F9211240BB60F92A9
:10FB70002F933F934F935F936F937F938F939F93B5
:10FB8000AF93BF93EF93FF93809138120E94846FDD
:10FB900020913B1230913C122F5F3F4F30933C122B
:10FBA00020933B1290913A12953618F096E090937C
:10FBB000371290913712943009F46EC0F8F49230F5
:10FBC00031F1933009F44CC090913912992319F016
:10FBD000811171C02F9AFF91EF91BF91AF919F91C9
:10FBE0008F917F916F915F914F913F912F910F90E6
:10FBF0000BBE0F900FBE0F901F901895953009F413
:10FC000057C0963009F791E0909307134FC08111C8
:10FC1000DBCF20913B1230913C122436310528F481
:10FC200010923C1210923B12CFCF109207131092F9
:10FC30003A12E0913A1291E09E0F90933A12F0E05E
:10FC400020913B1230913C12EE0FFF1FE35CFD4E02
:10FC50003183208310923C1210923B1293E019C022
:10FC6000813009F0B1CFE0913A1291E09E0F90936C
:10FC70003A12F0E020913B1230913C12EE0FFF1F40
:10FC8000E35CFD4E3183208310923C1210923B12B4
:10FC900094E09093371298CF882359F220913B1229
:10FCA00030913C122536310508F48ECF95E0F1CF26
:10FCB00081118ACFB5CF2F988ECFCF93DF9391E06C
:10FCC0009093F3118823B9F0C091B800D091BA0095
:10FCD0008091BC008A7B8093BC0060E084E10E943C
:10FCE000387860E085E10E9438780E942079D093CE
:10FCF000BA00C093B800DF91CF9108958F929F9280
:10FD0000AF92BF92CF92DF92EF92FF920F931F9329
:10FD1000CF93DF93D091BB0CD13208F0D7C0182F0E
:10FD2000C091BA0C0E9486796B017C018091B20C63
:10FD300081116BC082E08093B20C1093B10C8FEFF5
:10FD40008093B00C1092AF0CD093AE0CA7E9B5E144
:10FD5000EEE8FCE080E0D81391C010928D0C809109
:10FD60008D0CCC0FC82BC0938D0C80918C0C8130E6
:10FD700009F088C010928C0C0E9486796B017C017E
:10FD800080918D0C8093BB008091B40C9091B50C48
:10FD9000A091B60CB091B70C892B8A2B8B2BA1F0BC
:10FDA0000E9486790091B40C1091B50C2091B60C8C
:10FDB0003091B70C6C197D098E099F09061717073A
:10FDC0002807390708F442C08091BC0083FDD8CFD2
:10FDD00085EC8093BC000E9486796B017C01809148
:10FDE000B20C823009F450C08091B00C8F3F09F4FE
:10FDF0006FC08091B00C803209F46CC08091B00C5F
:10FE0000803309F469C084E026C08091B40C9091DD
:10FE1000B50CA091B60CB091B70C892B8A2B8B2B0B
:10FE200009F484CF0E9486798090B40C9090B50C30
:10FE3000A090B60CB090B70C6C197D098E099F0983
:10FE400086169706A806B90608F070CF8091B30C05
:10FE50000E945D7E85E01092B90C1092BB0C10924E
:10FE6000B80CDF91CF911F910F91FF90EF90DF9031
:10FE7000CF90BF90AF909F908F9008959D91919358
:10FE80008F5F69CF85EEA5CF8091B40C9091B50CB2
:10FE9000A091B60CB091B70C892B8A2B8B2B09F44F
:10FEA0009ECF0E9486790091B40C1091B50C2091E0
:10FEB000B60C3091B70C6C197D098E099F09061795
:10FEC00017072807390708F08ACFC0CF81E0C3CFD2
:10FED00080E0C1CF82E0BFCF83E0BDCFFC012481B1
:10FEE00031E03093B80C2093BA0C1092B90C1092F8
:10FEF000BB0C8385682B86EF9DE00E942B7081E010
:10FF00000C947E7E0F931F93CF938C01C62F0E947B
:10FF10006E7F6C2F6460C8010E946E7F6C2F6B7FB8
:10FF2000C8010E946E7F83EC90E00197F1F7CF91BA
:10FF30001F910F9108950F931F93CF938C01C62F9C
:10FF4000607F61600E94827F80E1C89FB0011124C0
:10FF50006160C8010E94827F81E090E0CF911F9193
:10FF60000F910895CF93C82F682F607F8BED91E19B
:10FF70000E94827F80E1C89FB00111248BED91E146
:10FF8000CF910C94827FCF93DF9300D000D01F924B
:10FF90001F92CDB7DEB798E0E9E1F3E0DE011196FC
:10FFA00001900D929A95E1F79091E411961708F45B
:10FFB0006FEF70E0660F771F21E030E02C0F3D1FE0
:10FFC000620F731FFB019081890F806828960FB61E
:10FFD000F894DEBF0FBECDBFDF91CF910C94B27FFE
:10FFE0000F931F93CF93DF932091DE02222321F101
:10FFF0002091DD02222301F1EB018C0161E080E020
:020000040001F9
:100000000E94C37FB8018BED91E10E94267765E2E3
:100010007EE08BED91E10E94487761E0F8018481F8
:100020000E94C37FBE01DD0F880B990BDF91CF913A
:100030001F910F910C94AB79DF91CF911F910F918C
:10004000089585ED8093BC008091B40C9091B50C1F
:10005000A091B60CB091B70C0796A11DB11D23E07D
:10006000B695A795979587952A95D1F72091BC00CD
:1000700024FD03C01092B20C08954091B40C50912D
:10008000B50C6091B60C7091B70C452B462B472BE5
:1000900069F30097A105B10541F025E32A95F1F731
:1000A00000000197A109B109E1CF8091B30C0C9434
:1000B0005D7E1F920F920FB60F9211240BB60F9216
:1000C0002F933F934F935F936F937F938F939F9360
:1000D000AF93BF93EF93FF938091B900887F8036F1
:1000E00009F44DC008F040C0883209F4A9C028F5D1
:1000F000803109F49DC0C8F4882309F4FBC088301E
:1001000009F496C0FF91EF91BF91AF919F918F91AC
:100110007F916F915F914F913F912F910F900BBE07
:100120000F900FBE0F901F901895883109F488C06A
:10013000803241F78093B00C14C0803409F49DC024
:1001400040F48033B9F38833E9F68093B00C85EC42
:10015000B0C0803509F485C0883509F496C088346C
:1001600089F60E942180CECF883909F48CC038F5F9
:10017000883729F050F4883611F0803719F683E07B
:100180008093B20C1092361257C0883809F47BC0A5
:10019000803919F0803809F0B5CF8091361280325D
:1001A00008F071C0E091361281E08E0F8093361214
:1001B0008091BB00F0E0EA5EFD4E80833DC0803B55
:1001C00039F0E0F4803A09F479C0883A09F09ACF1E
:1001D00084E08093B20C1092151210921412E091E8
:1001E0002B13F0912C1319958091141281110FC0CB
:1001F00081E0809314121092F41109C0803C09F43C
:10020000A6CF883C09F4A3CF883B09F07BCFE091CF
:10021000151281E08E0F80931512F0E0EC50FE4E27
:1002200080818093BB00909115128091141229C097
:1002300080918D0C8093BB0085EC8093BC0062CFD5
:100240009091AF0C8091AE0C981758F5E091AF0CDF
:1002500081E08E0F8093AF0CF0E0E257F34F808186
:10026000E9CFE091AF0C81E08E0F8093AF0C8091CD
:10027000BB00F0E0E257F34F80839091AF0C809188
:10028000AE0C9817C8F285E8D8CFE091AF0C81E0AA
:100290008E0F8093AF0C8091BB00F0E0E257F34FDC
:1002A00080838091B10C81115CCF81E080938C0CB4
:1002B00084EA8093BC001092B20C24CF85EC80932A
:1002C000BC001092B20C80913612803230F4E09172
:1002D0003612F0E0EA5EFD4E10826091361270E058
:1002E000E0912913F0912A1386E192E11995109279
:1002F000361208CF1092B00C34CFCF93DF93EC01BD
:100300008091ED11811109C081E08093ED11809100
:10031000020E9091030E0E946C0C60E08C81DF91C4
:10032000CF910C94387861E0FC0184810E94387888
:100330008091ED11882321F01092ED110C946B0C3B
:1003400008958FEF0C94FE0B0F931F93CF93DF93C1
:10035000EC010E94697A8B010E94A1818F3F69F0B4
:100360000E94697A601B710B6C177D07A8F380E00F
:10037000DF91CF911F910F91089581E0F9CF8F9276
:100380009F92AF92BF92FF920F931F93CF93DF93F1
:10039000EC01F62E49015A018E81882389F08F8164
:1003A00098859C012F5F3F4F38872F838230924082
:1003B00018F40E94A181F3CFCE010E9493811E8286
:1003C000CE010E947D818CE291E00E94A4818F2D5C
:1003D00080640E94FE0B08E110E0D501C401002EEC
:1003E00004C0B695A795979587950A94D2F70E9471
:1003F000FE0B08501109083F8FEF180771F785E9C8
:10040000FF2021F028E087E8F2128FEF0E94FE0B18
:1004100010E00E94A1818A8787FF04C01F3F11F06E
:100420001F5FF7CFDF91CF911F910F91FF90BF908A
:10043000AF909F908F900895AF92BF92CF92DF922E
:10044000EF92FF920F931F93CF93DF93EC0169011B
:10045000C801820F931F8130924050F58E8188230E
:1004600079F088819981AA81BB8184179507A607B5
:10047000B70731F48F819885C816D90608F042C0B5
:10048000488359836A837B838B85833039F089E085
:10049000440F551F661F771F8A95D1F79A01AB014C
:1004A00061E1CE010E94BF81882389F083E08D83C2
:1004B000CE010E94938180E0DF91CF911F910F9137
:1004C000FF90EF90DF90CF90BF90AF9008950E9483
:1004D000697A5B010E94A1818A878F3F69F40E943B
:1004E000697A6A197B096D327140A0F38FE08D83C0
:1004F000CE010E949381DCCF8E3F89F418861F8243
:1005000081E08E838F8198858C159D0550F40E9423
:10051000A1818F819885019698878F83F3CF8DE095
:10052000E6CF6701E00EF11E0E94A181F6018193E2
:100530006F01EE15FF05C1F78F819885080F191F10
:1005400018870F838985882319F001151240A0F0C0
:100550008E81882389F08F8198859C012F5F3F4F82
:1005600038872F838230924018F40E94A181F3CF04
:10057000CE010E9493811E8281E09ECFEF92FF9276
:100580000F931F93CF93DF93EC01790182E1411523
:1005900051056105710599F08B85833039F089E04B
:1005A000440F551F661F771F8A95D1F79A01AB013B
:1005B00068E1CE010E94BF81882319F084E08D8319
:1005C00030C08EEF0E94FE0B87018EEFF81AF80103
:1005D00081918F010E94FE0B0E151F05C1F78FEF51
:1005E0000E94FE0B8FEF0E94FE0B0E94A1818A8762
:1005F0008F71853089F488E592E00E94A481882378
:10060000A9F020E030E0A9016DE0CE010E94BF8199
:10061000882371F084E1D3CF81E18D83CE010E94E4
:100620009381CE010E94938180E00AC085E1C7CF0B
:100630000E94A1818111EECFCE010E94938181E0C1
:10064000DF91CF911F910F91FF90EF900895CF937D
:10065000DF938091EE118823A9F1C0912D13D091E1
:100660002E1340919E0250919F026091A0027091C2
:10067000A10227E933E1CE010E94BE82811104C0AC
:1006800080E0DF91CF9108954091EF115091F011EA
:100690006091F1117091F2114115510561057105DB
:1006A00079F027E933E1CE010E94BE82882341F32D
:1006B0001092EF111092F0111092F1111092F211AC
:1006C0001092EE1181E0DDCF8F929F92AF92BF9298
:1006D000EF92FF920F931F93CF934B015C01C42FB6
:1006E00080919E0290919F02A091A002B091A102E0
:1006F00088159905AA05BB0549F10E942783811138
:100700000BC080E0CF911F910F91FF90EF90BF90B1
:10071000AF909F908F90089587E9E82E83E1F82E9F
:1007200000E012E030E020E0B501A40180912D133B
:1007300090912E130E941C82882319F380929E02AE
:1007400090929F02A092A002B092A1024091EE115D
:100750004C2B4093EE1181E0D5CFCF93DF93EC018A
:100760006E857F858889998941E00E94648388230A
:1007700051F08A8920E2829FC001112489569C4E43
:10078000DF91CF91089590E080E0FACF8F929F9211
:10079000AF92BF92CF92DF92EF92FF92CF9324E07D
:1007A0003EE030932E1320932D13882309F46DC05F
:1007B00040E060E070E0CB010E94648381110BC0D7
:1007C00080E0CF91FF90EF90DF90CF90BF90AF90FF
:1007D0009F908F900895809155158F7789F780911C
:1007E000611590916215A0916315B09164158436DE
:1007F0009105A105B10520F3C0905D15D0905E155F
:10080000E0905F15F0906015C114D104E104F1048B
:10081000B9F240E0C701B6010E946483882381F2E7
:100820008091A2139091A3138115924049F6A09153
:10083000A713AA2329F26091A5137091A61361153D
:10084000710509F4BDCF2091A413222309F4B8CF78
:10085000A093220E2093140E90E080E030E0E1E0BF
:10086000F0E0C82FAF01082E02C0440F551F0A94B4
:10087000E2F72417350769F041E0480F0196893007
:10088000910579F740931D0E9BCFC12CD12C760199
:10089000C0CF80931D0E2091AD133091AE1350E068
:1008A00040E02115310541F42091BB133091BC1378
:1008B0004091BD135091BE132093150E3093160E28
:1008C0004093170E5093180E46015701860E971E3F
:1008D000A11CB11C8092230E9092240EA092250E92
:1008E000B092260EE091A813F091A913F093290E6F
:1008F000E093280EB0E00E94CBA8DC01CB01880D6C
:10090000991DAA1DBB1D80932A0E90932B0EA093B8
:100910002C0EB0932D0E25E0EE0FFF1F2A95E1F768
:10092000E150FE4FEF2FFF27E6958E0F9F1FA11D71
:10093000B11D80931E0E90931F0EA093200EB093B6
:10094000210E8090AA139090AB13B12CA12C81148E
:10095000910441F48090B7139090B813A090B9130C
:10096000B090BA13C81AD90AEA0AFB0AC80CD91CF3
:10097000EA1CFB1C04C0F694E794D794C794CA956C
:10098000D2F7C092190ED0921A0EE0921B0EF0927E
:100990001C0E85EFC8168FE0D806E104F10428F498
:1009A0008CE08093270E81E00CCF80E125EFC2160A
:1009B0002FEFD206E104F104A0F38091C3139091CC
:1009C000C413A091C513B091C61380932A0E9093BF
:1009D0002B0EA0932C0EB0932D0E80E2E2CF4F92FF
:1009E0005F926F927F928F929F92AF92BF92CF92BF
:1009F000DF92EF92FF920F931F93CF93DF93EC015F
:100A0000423051056105710590F480E0DF91CF918E
:100A10001F910F91FF90EF90DF90CF90BF90AF901C
:100A20009F908F907F906F905F904F9008958985F1
:100A30009A85AB85BC850196A11DB11D84179507CC
:100A4000A607B70710F3CB88DC88ED88FE888F896E
:100A5000803109F042C0BB27A72F962F852F480170
:100A600059012A013B01C80ED91EEA1EFB1E8091C6
:100A70009E0290919F02A091A002B091A102C8167F
:100A8000D906EA06FB0699F58F898031C1F5B301D5
:100A9000A201552766277727440F551F49565C4EFC
:100AA000FA01918280828091EE1181608093EE1133
:100AB0008A89823080F08D819E81AF81B8858C0DCE
:100AC0009D1DAE1DBF1D8093EF119093F011A0935B
:100AD000F111B093F21181E099CFDB01CA01E7E097
:100AE000B695A79597958795EA95D1F7B8CF40E049
:100AF000C701B6010E9464838111C6CF86CFB301BE
:100B0000A2014F77552766277727440F551F440FBB
:100B1000551F49565C4EFA0180829182A282B382AF
:100B2000C2CF8F929F92AF92BF92CF92DF92EF92FD
:100B3000FF920F931F93CF93DF93FC0181859285E2
:100B4000A385B4850196A11DB11D84179507A6073D
:100B5000B70770F480E0DF91CF911F910F91FF9064
:100B6000EF90DF90CF90BF90AF909F908F900895BF
:100B700083889488A588B6888789803189F5BB27C2
:100B8000A72F962F852FE9016A017B018F01BC01F8
:100B9000CD01680D791D8A1D9B1D80909E0290904D
:100BA0009F02A090A002B090A10286169706A80608
:100BB000B90601F5F8018789803111F5DD24EE24AD
:100BC000FF24F601EE0FFF1FE956FC4E8081918154
:100BD000B0E0A0E088839983AA83BB8381E0BBCF88
:100BE000DB01CA01C7E0B695A79597958795CA9589
:100BF000D1F7C9CF40E00E9464838111DBCFAACF37
:100C0000E894C7F8DD24EE24FF24F601EE0FFF1F61
:100C1000EE0FFF1FE956FC4E80819181A281B381C6
:100C2000BF70D8CF4F925F926F927F92AF92BF9278
:100C3000CF92DF92EF92FF920F931F93CF93DF93A8
:100C400000D01F92CDB7DEB78C0149835A836B83E6
:100C50007C835901C12CD12C7601412C82E0582E85
:100C6000612C712C49815A816B817C819E012F5F9F
:100C70003F4FC8010E949185882339F1F80185858D
:100C8000A301920104C0220F331F441F551F8A95F0
:100C9000D2F7DA01C901C80ED91EEA1EFB1E49812E
:100CA0005A816B817C818789803111F188EF9FEFB8
:100CB000AFEFBFE0481759076A077B0798F2F501C5
:100CC000C082D182E282F38281E00F900F900F9078
:100CD0000F90DF91CF911F910F91FF90EF90DF90D8
:100CE000CF90BF90AF907F906F905F904F9008959E
:100CF00088EF9FEFA0E0B0E0DDCF8F929F92AF92A0
:100D0000BF92CF92DF92EF92FF920F931F93CF93F8
:100D1000DF93EC018D8181110EC080E0DF91CF91D6
:100D20001F910F91FF90EF90DF90CF90BF90AF9009
:100D30009F908F9008950B891C892D893E890417F7
:100D400015072607370748F34A015B01823031F463
:100D50008A869B86AC86BD8681E0E0CF81149104B3
:100D6000A104B10449F41E821F82188619861A86CE
:100D70001B861C861D86F0CF0A851B852C853D852C
:100D8000EB8DFC8D858590E00996B901A801415055
:100D9000510961097109082E04C076956795579528
:100DA00047950A94D2F775016401E1E0CE1AD108A3
:100DB000E108F10804C0F694E794D794C7948A95A3
:100DC000D2F7C416D506E606F70620F0012B022B53
:100DD000032B11F58F89988DA98DBA8D8E839F83F2
:100DE000A887B9878E010A5F1F4FC114D104E1049F
:100DF000F10409F4ADCF4E815F8168857985980152
:100E00008B8D9C8D0E94918591E0C91AD108E108D3
:100E1000F1088111EACF81CFC41AD50AE60AF70A90
:100E2000E1CF3F924F925F926F927F928F929F920B
:100E3000AF92BF92CF92DF92EF92FF920F931F93E8
:100E4000CF93DF93CDB7DEB72C970FB6F894DEBF04
:100E50000FBECDBF5C01DC015B968D909C905C97D2
:100E600016964D905D906D907C90199741145104A9
:100E70006104710409F468C0BFEF4B1A5B0A6B0A86
:100E80007B0A312CF40181859285A385B4859C0170
:100E9000AD012F5F3F4F4F4F5F4F29873A874B87F9
:100EA0005C87730162011D821E821F821886F40115
:100EB00081859285A385B4852D813E814F8158859A
:100EC000281739074A075B0708F056C089859A85B5
:100ED000AB85BC858C159D05AE05BF0550F482E041
:100EE000C82ED12CE12CF12C92E0492E512C612CF2
:100EF000712C9E012F5F3F4FB701A601C4010E94D4
:100F000091858823C9F189819A81AB81BC81892B24
:100F10008A2B8B2B09F1260137019FEF491A590AB9
:100F2000690A790A2D813E814F8158852F5F3F4F95
:100F30004F4F5F4F2D833E834F8358873FEFC31A38
:100F4000D30AE30AF30AB3CFF401408051806280F0
:100F500073803324339496CFC414D504E604F70485
:100F600009F70FEF1FEF2FEF3FE0B701A601C40114
:100F70000E94EF84811119C080E02C960FB6F8947E
:100F8000DEBF0FBECDBFDF91CF911F910F91FF90BC
:100F9000EF90DF90CF90BF90AF909F908F907F9019
:100FA0006F905F904F903F900895F5014681578173
:100FB00060857185411551056105710539F097010D
:100FC0008601C4010E94EF848823B1F2D5011696F0
:100FD000CD92DD92ED92FC921997332051F0D7011A
:100FE000C6010196A11DB11DF40180839183A283E6
:100FF000B383F5018789908DA18DB28D892B8A2BC2
:101000008B2B39F4C78AD08EE18EF28E8481806872
:10101000848381E0B2CF2F923F924F925F926F9282
:101020007F928F929F92AF92BF92CF92DF92EF9278
:10103000FF920F931F93CF93DF93EC015B012A0183
:101040008D81811115C08FEF9FEFDF91CF911F919F
:101050000F91FF90EF90DF90CF90BF90AF909F9057
:101060008F907F906F905F904F903F902F9008955A
:101070008C8180FFE8CF0B891C892D893E894A85A8
:101080005B856C857D85C201B0E0A0E068017901D7
:10109000C41AD50AE60AF70AC816D906EA06FB06F4
:1010A00018F42801441A550A42011E0126E0220EB6
:1010B000311C8114910409F4B3C04A855B856C85A9
:1010C0007D856A0181E0D8228B8D9C8D8A019B01F0
:1010D000E9E03695279517950795EA95D1F7ED81C3
:1010E000E230E1F5FC01628D738D848D958D600F8A
:1010F000711F821F931F612C22E0722E6C187D08D5
:101100008614970408F434012C8126FD04C0611470
:10111000F2E07F0671F400919E0210919F022091EF
:10112000A0023091A102061717072807390709F016
:1011300053C040E00E946483882309F484CFC60131
:1011400089569C4ED5019C01260D371DFC012E179A
:101150003F0709F460C041914D93F9CFFC017480C1
:101160007A947022C114D10471F471100CC0452B13
:10117000462B472B39F58F89988DA98DBA8D8E8393
:101180009F83A887B987EB8DFC8D6E817F818885D1
:1011900099856250710981099109258504C0660FFE
:1011A000771F881F991F2A95D2F7068517852089F2
:1011B0003189600F711F821F931F670D711D811D83
:1011C000911D99CF4E815F816885798591010E943B
:1011D00091858111D8CF37CF750183019601AB017D
:1011E000BC0180912D1390912E130E941C828823A4
:1011F00009F429CFA60CB71C8A859B85AC85BD85D3
:10120000860D971DA11DB11D8A879B87AC87BD8761
:10121000861897084ECF281B390BA20EB31EECCFB1
:10122000C20113CFCF93DF931F92CDB7DEB741E05A
:1012300050E0BE016F5F7F4F0E940B88019731F431
:10124000898190E00F90DF91CF9108958FEF9FEF0C
:10125000F9CFFC01818D928D009711F00C941289C9
:101260008FEF9FEF08950F931F93CF93DF93EC01C0
:10127000898D9A8D10E000E0009799F00E94128904
:101280008C010F3F100769F0898D9A8DFC01428512
:1012900053856485758541505109610971090E9422
:1012A0007D86C801DF91CF911F910F910895CF9353
:1012B000DF93EC018D81882329F18C8187FF1EC08B
:1012C000CE010E94AD83FC01892BE1F08D8182303B
:1012D00040F48B899C89AD89BE89848F958FA68FB8
:1012E000B78F8F89988D938F828F8F89988DA98DD5
:1012F000BA8DB58BA48B8C818F778C83DF91CF9146
:101300000C94278380E0DF91CF9108958F929F9274
:10131000AF92BF92CF92DF92EF92FF920F931F9303
:10132000CF93DF9300D01F92CDB7DEB7FC0185814C
:10133000813091F080E00F900F900F900F90DF912F
:10134000CF911F910F91FF90EF90DF90CF90BF90C2
:10135000AF909F908F900895848181FFEBCF838918
:101360009489A589B689892B8A2B8B2B09F45EC0B9
:101370007F0140E050E0BA01CF010E947D868823C2
:10138000C9F2F701C38CD48C8788908CA18CB28C65
:1013900082E090E0A0E0B0E0F60180839183A28338
:1013A000B3839E012F5F3F4FB501A401C6010E9488
:1013B0009185882309F4BECF00E010E09801B501C3
:1013C000A401C6010E94EF84882309F4B3CF898069
:1013D0009A80AB80BC80F6018789803111F188EF5B
:1013E0009FEFAFEFBFE088169906AA06BB06C8F2CA
:1013F000F701178A108E118E128E138A148A158A9D
:10140000168A848180688483C7010E945789882353
:1014100009F490CF40E050E0BA01C7010E947D86F8
:101420008ACF88EF9FEFA0E0B0E0DDCF81E083CFEF
:10143000CF92DF92EF92FF921F93CF93DF93EC0155
:1014400080E2689FF0011124E956FC4E938591716A
:1014500061F0842F827449F080E0DF91CF911F9179
:10146000FF90EF90DF90CF900895142F6A8B8091BA
:101470009E0290919F02A091A002B091A1028E873E
:101480009F87A88BB98BC488D588F12CE12C760175
:10149000DD24CC24CF8AD88EE98EFA8E828D938D6E
:1014A000B0E0A0E0AC01BD014C295D296E297F2987
:1014B0004F8B588F698F7A8F83858871B1F4848DB3
:1014C000958DA68DB78D8B8B9C8BAD8BBE8B81E064
:1014D0008D831F701C831E821F82188619861A86B0
:1014E0001B861C861D8681E0B8CF803109F0B4CF01
:1014F0009E012D5E3F4F8B8D9C8D0E94128688230E
:1015000009F4AACF84E0E4CFCF93DF93EC010E94EB
:101510005789882311F01D8281E0DF91CF910895D2
:10152000FC01818D928D009711F00C9457890895DC
:101530003F924F925F926F927F928F929F92AF9263
:10154000BF92CF92DF92EF92FF920F931F93CF93B0
:10155000DF9300D000D000D01F921F92CDB7DEB72E
:101560007C01DC0115968C91811115C0FE0131962C
:10157000CE010C966F0130E23193E817F907E1F7DD
:10158000DA0130E087E09D91B92E992329F19E324E
:1015900039F48A3011F480E0D9C038E08AE0F3CF22
:1015A000EEECFBE04491442321F031969413FACF02
:1015B000F2CF831780F34FED490F4E3560F74FE9B7
:1015C000490F4A3118F440EEB42EB90EF601E30F7C
:1015D000F11DB0823F5FD7CF89818032E1F2322E98
:1015E0008B01FB01838D948DD7015C969C938E9328
:1015F0005B971682178210861186128613861486D0
:101600001586F80182859385A485B585438954891B
:101610006589768984179507A607B70708F04DC036
:1016200025E0B695A795979587952A95D1F7F82F38
:10163000FF70AF2ED80115968C91823008F4ABCF95
:10164000C8010E94128997FDA6CFF8018285938573
:10165000A485B5854F96A11DB11D82879387A48768
:10166000B587F0E2AF9EB001112469567C4E61153A
:10167000710509F490CFDB018C91882341F0853E00
:1016800009F057C0BB2029F0BB24B394BACFB110E6
:101690000EC0F701A28A80919E0290919F02A091B4
:1016A000A002B091A10286879787A08BB18BDB0146
:1016B0008C918111E9CFBB24B394832D8271823147
:1016C00009F069CFBB2009F459C0C7010E94AD835E
:1016D000009709F460CF20E2FC0111922A95E9F706
:1016E0002BE0F601DC0101900D922A95E1F721E251
:1016F00038E2DC0151963C932E93509740E058E03D
:101700001F965C934E931E9753963C932E9352973D
:1017100059963C932E93589757965C934E935697B1
:101720000E942783882309F436CF432DF70162896D
:101730000AC04BE050E0C6010E9462AC892B09F060
:1017400060CF432D6A2DC7010E94188A2B960FB6D1
:10175000F894DEBF0FBECDBFDF91CF911F910F91E7
:10176000FF90EF90DF90CF90BF90AF909F908F90C1
:101770007F906F905F904F903F900895F801858122
:10178000823009F408CFC8010E941187882309F428
:1017900002CFD8015B96ED91FC915C9716968D90E7
:1017A0009D90AD90BC901997B2E08B1A9108A1085A
:1017B000B108858504C0880C991CAA1CBB1C8A959D
:1017C000D2F786859785A089B189880E991EAA1EB1
:1017D000BB1E848124013501480E511C611C711C03
:1017E00084149504A604B70401F1E1E04E1A5108EF
:1017F000610871080E942783882309F4CCCEE7E9A9
:10180000F3E1119287E995E18E179F07D1F7409296
:101810009E0250929F026092A0027092A10280915B
:10182000EE1181608093EE11DBCFD8015B96ED91D4
:10183000FC91258580E092E0A0E0B0E004C0880F34
:10184000991FAA1FBB1F2A95D2F7F8014389548913
:1018500065897689840F951FA61FB71F838B948B8C
:10186000A58BB68BD70152961C9287E993E133CFB3
:101870005F926F927F928F929F92AF92BF92CF9220
:10188000DF92EF92FF920F931F93CF93DF93CDB729
:10189000DEB7C754D1090FB6F894DEBF0FBECDBF77
:1018A0005C013B0119A218A28DE693E09F8F8E8FF9
:1018B0001BA21C821B829A8389831E8210E000E097
:1018C0006E018EE1C80ED11C8EE2E82E8EE0F82E5D
:1018D000F501E00FF11F80818F3211F40F5F1F4F70
:1018E000D501A00FB11FFE01FB9690E080E04F01F3
:1018F0002D912F3249F0222339F00F5F1F4F0196AF
:1019000021938C309105A1F7880D991DFC0110825F
:10191000F501E00FF11F80818F3211F40F5F1F4F2F
:10192000F501E00FF11F508041E0511040E030E040
:1019300020E0B401C701F3011995811121C0FEE235
:10194000EF16FEE0FF06C1F480E0C95BDF4F0FB683
:10195000F894DEBF0FBECDBFDF91CF911F910F91E5
:10196000FF90EF90DF90CF90BF90AF909F908F90BF
:101970007F906F905F900895C7010E94848AE4CFA2
:10198000552091F021E0A401B701C6010E94988A78
:10199000982E8EE2E8168EE0F80681F0C7010E94CC
:1019A000848A911010C0D0CF9EE2E9169EE0F9061D
:1019B00019F0C7010E94848A81E0C7CF992021F2E3
:1019C000FE0131967F019E2D8F2D7601C92ED82ED6
:1019D0007FCF1F93CF93DF93CDB7DEB76D970FB651
:1019E000F894DEBF0FBECDBFAB011C821B822DE67B
:1019F00033E03A8329831E8221E0BC01CE010196A7
:101A00000E94988A11E081110CC010E0812F6D9620
:101A10000FB6F894DEBF0FBECDBFDF91CF911F91FF
:101A20000895CE0101960E94848AF0CFCF93DF9370
:101A3000CDB7DEB76D970FB6F894DEBF0FBECDBF42
:101A4000442391F1AB01BC011C821B828DE693E023
:101A50009A8389831E8222E0CE0101960E94988A91
:101A600081110EC090E081E0911101C080E06D967F
:101A70000FB6F894DEBF0FBECDBFDF91CF910895B2
:101A8000CE0101960E948689882361F3CE010196DA
:101A90000E94AD83009731F325EEFC0120831E8266
:101AA0000E942783982FDFCF81E0E1CF2F923F92D2
:101AB0004F925F926F927F928F929F92AF92BF925E
:101AC000CF92DF92EF92FF920F931F93CF93DF930A
:101AD00000D01F92CDB7DEB78C015B011A01DC018B
:101AE00015968C911597813009F0C8C014968C9189
:101AF00081FFC4C082FDAEC06101D8011A964D912C
:101B00005D916D917C911D97C114D10409F429C197
:101B10005B968D919C915C97FC0174802FEF270D53
:101B20002A013B0139E076946794579447943A959B
:101B3000D1F7722E74207A01F1E0FF22711020C0DB
:101B4000E114F104E9F416964D915D916D917C914B
:101B50001997411551056105710509F098C057960F
:101B60008D919D910D90BC91A02D0097A105B1057F
:101B700009F0AFC0C8010E941187882309F47EC014
:101B800080E092E08E199F0946018C159D0508F4AE
:101B90004C01D8015B964D915C915C9716968D91A6
:101BA0009D910D90BC91A02D0297A109B109FA0158
:101BB000258504C0880F991FAA1FBB1F2A95D2F73D
:101BC0004685578560897189840F951FA61FB71FA9
:101BD0009C01AD01270D311D411D511D29013A0107
:101BE000811432E0930609F07AC080919E029091B0
:101BF0009F02A091A002B091A10284159505A605AF
